:100000000C94F9230C942A240C942A240C942A246A
:100010000C942A240C9465560C942A240C942A24BB
:100020000C942A240C942A240C942A240C9438BA74
:100030000C942A240D9443AE0C942A240C942A2464
:100040000C942A240D94ED260C942A240C942A2432
:100050000C942A240C942A240D94333D0D9472A6FA
:100060000C942A240C949D320C942A240C942A2457
:100070000C942A240C942A240C942A240C942A24C8
:100080000C942A240C942A240C942A240C942A24B8
:100090000C942A240C942A240C942A240C942A24A8
:1000A0000C942A240C942A240C942A240C942A2498
:1000B0000C942A240C942A240C942A240C942A2488
:1000C0000C942A240C942A240C942A240C94E632AE
:1000D0000C942A240C942A240C942A240C942A2468
:1000E0000C942A24810193017B01A901AB01C50174
:1000F000790151015301EB01E701E5018B01630136
:10010000A101E9013B016D01470173017F01590123
:1001100055014B016901C10197016B01D901AF0183
:10012000C701AD016701B3015D018701D1019D01E7
:10013000AF01A501B9017D01D501DF0143019101A5
:100140006101D70141014501330189015B018F0143
:100150003F01B501D701A701A3019901036EDB3669
:100160003D9A9999993DABAAAA2A3E000000803F8A
:10017000084AD73B3BCE016E84BCBFFDC12F3D6C0E
:1001800074319ABD56833DDA3D00C77F11BED9E474
:10019000BB4C3E916BAAAABE000000803F072C7AA0
:1001A000A5BA6CC590DA3B9365FC8BBC53F810FD87
:1001B0003C5692834DBD879D3AB63DCBC9BF5BBED1
:1001C00073DA0FC93F05A84CCDB2D44EB93836A961
:1001D000020C50B9918688083CA6AAAA2ABE000043
:1001E00000803F07634236B79BD8A71A3968561874
:1001F000AEBAAB558C1D3CB7CC5763BD6DEDFD75EC
:100200003EF6177231BF000000803F08000000BEBC
:10021000922449123EABAAAA2ABECDCCCC4C3E00B9
:10022000000080BEABAAAAAA3E00000000BF0000EA
:1002300000803F0000000000084178D3BB4387D115
:10024000133D190E3CC3BD4282AD2B3E68EC827655
:10025000BED98FE1A93E4C80EFFFBE01C4FF7F3FB6
:100260000000000000000D947DA80D94626D0D94B7
:100270001D4A0D9408530D940B700D94CF290D94C5
:100280008FA80D9473A80D945EA80D9477A80D9473
:1002900033700D942F7F0D9482700D9441950D94C1
:1002A000527B0D94363E0D94383E0D9472700D9431
:1002B000C7750D9462700D9485A80D94FFA70D94D9
:1002C00090610D9468A80D94743E0D94B86C0D94D3
:1002D000EBA70D94B3A70D94C7A70D941E700D94B2
:1002E0004D660D94C38C0D9458700D94A66C0D94AE
:1002F0008E6F0D94323E0D94E23D0D9440A80D9406
:100300005D700D94B83D0D949D6C0D948A4E0D94C6
:1003100009A80D9481A80D94663E0D94AF6C0D94C0
:100320008BA80D9462A80D94C63D0D94C84D0D94F4
:10033000BDA70D94A1A80D94015B0D9422A80D9466
:100340004F040D94943E0D949DA80D942CA80D94EB
:1003500099A80D94F03D0D940A3E0D94E3A70D94D9
:100360004AA80D948E6E0D94F5A70D9493A80D9444
:100370003DA90D9436A80D94FB4F0D9489640D94FE
:100380001E5E0D94B8A70D94009C0D94183E0D941C
:10039000DBA70D94E4720D94B34D0D941C870D945E
:1003A00007610D9418A80D94C67D0D946CA80D944A
:1003B000A6A80D94D1A70D942A4D0D94C24D0D946D
:1003C0006FA80D94316B0D94724B0D944C3E0D94AF
:1003D0003E3E0D94FB6F0D943C3E48617264636F2A
:1003E0006465642044656661756C7420536574743B
:1003F000696E6773204C6F616465640053746F723B
:1004000065642073657474696E67732072657472B5
:10041000696576656400202020452F44203D20003A
:100420002020204D393030204B004C696E656172C0
:1004300020616476616E63652073657474696E67AC
:10044000733A0046696C616D656E742073657474EF
:10045000696E67733A2044697361626C6564002059
:1004600020204D32303020440046696C616D656E4D
:10047000742073657474696E67733A002020204D90
:100480003230392053004175746F2D52657472619A
:1004900063743A20533D3020746F20646973616245
:1004A0006C652C203120746F20696E7465727072D7
:1004B000657420657874727564652D6F6E6C792033
:1004C0006D6F7665732061732072657472616374F9
:1004D00073206F72207265636F7665726965730051
:1004E0002046002020204D323038205300526563D2
:1004F0006F7665723A20533D4578747261206C6561
:100500006E67746820286D6D2920463A53706565C2
:100510006420286D6D2F6D2900205A002046002090
:1005200020204D323037205300526574726163745D
:100530003A20533D4C656E67746820286D6D292004
:10054000463A537065656420286D6D2F6D29205AD9
:100550003A205A4C69667420286D6D2900204400A9
:100560002049002020204D33303420500050494491
:1005700020686561746265642073657474696E6770
:10058000733A002044002049002020204D333031B0
:100590002050005049442073657474696E67733A43
:1005A00000205A0020590020204D323036205800BB
:1005B000486F6D65206F666673657420286D6D29C0
:1005C0003A00204500205A002059002058002042BF
:1005D0000020540020204D323035205300416476F5
:1005E000616E636564207661726961626C65733AFD
:1005F00020533D4D696E20666565647261746520A7
:10060000286D6D2F73292C20543D4D696E20747216
:100610006176656C20666565647261746520286D1D
:100620006D2F73292C20423D6D696E696D756D20AB
:100630007365676D656E742074696D6520286D73D0
:10064000292C20583D6D6178696D756D20585920B1
:100650006A65726B20286D6D2F73292C20205A3DFE
:100660006D6178696D756D205A206A65726B2028FE
:100670006D6D2F73292C2020453D6D6178696D7556
:100680006D2045206A65726B20286D6D2F732900DF
:1006900020540020204D32303420530041636365E4
:1006A0006C65726174696F6E3A20533D6163636576
:1006B0006C65726174696F6E2C20543D7265747242
:1006C00061637420616363656C65726174696F6EE8
:1006D00000204500205A0020590020204D323031A2
:1006E0002058004D6178696D756D20416363656CBC
:1006F00065726174696F6E20286D6D2F7332293AAF
:1007000000204500205A0020590020204D3230336F
:100710002058004D6178696D756D2066656564725D
:100720006174657320286D6D2F73293A0020450090
:10073000205A0020590020204D393220580053748F
:100740006570732070657220756E69743A00536528
:100750007474696E67732053746F726564004545E5
:1007600050524F4D204572726F72000020006D652F
:10077000736820626564206C6576656C696E673AA3
:10078000200029002C20002C2000706879736963F8
:10079000616C20636F6F7264696E617465733A2077
:1007A000280029002C20002C2000776F726C642018
:1007B000636F6F7264696E617465733A20280020FC
:1007C00046002045004731205A004D3234004D325A
:1007D000362053256C75004D31303620530047319B
:1007E000204625640047312045312046343830000A
:1007F0004731205A0020463230303000205900471F
:10080000312058004D383300506F736974696F6E32
:1008100020726561642066726F6D20656570726F0D
:100820006D3A004D3233202573002E67636F00460A
:10083000656564726174653A007265636F766572AE
:100840005F6D616368696E655F73746174655F6134
:10085000667465725F706F7765725F70616E6963F1
:100860002C20696E697469616C20007265636F7613
:1008700065725F6D616368696E655F7374617465ED
:100880005F61667465725F706F7765725F70616ECD
:1008900069632C20696E697469616C2000726563FC
:1008A0006F7665725F6D616368696E655F737461B1
:1008B00074655F61667465725F706F7765725F7093
:1008C000616E69632C20696E697469616C200063D4
:1008D000757272656E745F706F736974696F6E5B49
:1008E0005A5F415849535D3A0043757272656E74A0
:1008F00020706F736974696F6E20595F4158495356
:100900003A0043757272656E7420706F7369746912
:100910006F6E20585F415849533A004166746572C2
:100920002077616974696E6720666F722074656DE7
:10093000703A00473120452D312046343830004789
:10094000312045352046313230004D3833004D31AD
:10095000393020532564004D31303920532564004F
:1009600047323820582059004731205A3235204626
:10097000383030004D31343020532564004D313053
:10098000342053256400494E54340055564C4F20B2
:100990002D20656E6400737470730055564C4F00C3
:1009A00020423A0020453A00543A005A206C6976B9
:1009B000652061646A757374206F7574206F66209A
:1009C00072616E67652E2053657474696E6720745A
:1009D0006F20302E20436C69636B20746F20636F2F
:1009E0006E74696E75652E005A206C69766520619B
:1009F000646A757374206F7574206F662072616EFF
:100A000067652E2053657474696E6720746F20309B
:100A10000020573A0020453A00543A004B494C4CCC
:100A20003A20004175746F0020452F443D00416419
:100A300076616E6365204B3D0022283229004431E7
:100A400030303000473238205900473238205800C3
:100A50005400496E76616C6964205420636F64654C
:100A60002E00496E76616C6964204D20636F646569
:100A70002E004D3232302053256900203A200000EC
:100A80004C414E472053454C20464F52434544006D
:100A9000222831290020453A00205A3A0020593AAC
:100AA0000020453A00205A3A0020593A00583A00AE
:100AB00020002E0020423A0020453A00543A0020FF
:100AC000413A0020503A002042403A0020403A008B
:100AD000202F003A00205400202F0020423A00200E
:100AE0002F006F6B20543A002569206D696E2C2011
:100AF00025692073656300496E76616C6964204DD9
:100B000020636F6465004D65736820626564206CC6
:100B10006576656C696E67206E6F742061637469B9
:100B200076652E000A002020000A4D6561737572FB
:100B3000656420706F696E74733A000A5A20736599
:100B400061726368206865696768743A20002C00E8
:100B50004E756D20582C593A2000476F20686F6DF4
:100B6000652066696E6973686564004D6573682009
:100B7000626564206C6576656C696E67206163747C
:100B800069766174656400557073616D706C652081
:100B900066696E697368656400426564206C657699
:100BA000656C696E6720636F7272656374696F6EDE
:100BB0002066696E697368656400206D6963726F91
:100BC0006E7300457863657373697665206265644A
:100BD000206C6576656C696E6720636F7272656301
:100BE00074696F6E3A200042656420636F727265AB
:100BF0006374696F6E2064617461206E6F74207617
:100C0000616C69640A0042656420636F7272656397
:100C100074696F6E20646174612076616C69640A26
:100C2000006261627973746570206170706C6965CF
:100C30006400636C65616E2075702066696E69730F
:100C400068656420004D4553485F484F4D455F5AE5
:100C50005F5345415243483A20004D657368206216
:100C60006564206C6576656C696E67207768696C71
:100C700065206C6F6F702066696E69736865642E9D
:100C80000000206F66667365743A20006D657368B6
:100C900020626564206C6576656C696E673A200039
:100CA0000A00593A200000583A20003A206E6F207E
:100CB000787920636C616D70696E670A003A2078FC
:100CC0007920636C616D7065642E0A00002C2063CE
:100CD000616C6962726174696F6E207A3A200042B9
:100CE0006564206C6576656C696E672C20706F6931
:100CF0006E743A2000005A206A6974746572206428
:100D00006174612066726F6D205A2063616C2E20C1
:100D10006E6F742076616C69642E0A005A206A69CD
:100D20007474657220646174612066726F6D205AFC
:100D30002063616C2E2076616C69642E0A004E6F10
:100D400020636C616D70696E6720666F72206669E2
:100D50007273742063616C6962726174696F6E2072
:100D6000706F696E742E0A00466972737420636135
:100D70006C6962726174696F6E20706F696E742045
:100D8000636C616D7065642E0A00473238205730FD
:100D9000003A200054656D7065726174757265204B
:100DA00063616C6962726174696F6E20646F6E65F5
:100DB0002E20436F6E74696E7565207769746820A4
:100DC0007072657373696E6720746865206B6E6FEF
:100DD000622E0000205A20736869667420286D6DA9
:100DE000293A0050494E44412074656D7065726126
:100DF000747572653A2000002F3600537465703A9E
:100E0000200000205A20736869667420286D6D29BF
:100E10003A0050494E44412074656D7065726174AA
:100E20007572653A20002F362028736B69707065E3
:100E3000642900537465703A2000005A45524F3AB5
:100E400020000073746172742074656D7065726146
:100E5000747572653A200050494E44412070726F9B
:100E600062652063616C6962726174696F6E207380
:100E70007461727400473238205730000A00205ADB
:100E80003A200020593A200020583A2000473238B2
:100E90002C2066696E616C20004732382C20666910
:100EA0006E616C20004732382C2066696E616C20C0
:100EB000004732382C20696E697469616C200047E4
:100EC00032382C20696E697469616C2000443939AC
:100ED00039004D3239002055706C6F616420696EA5
:100EE0002070726F677265737300696E69746961EF
:100EF0006C207A73746570732061667465722072F9
:100F0000657365743A2000696E697469616C207A52
:100F10007374657073206F6E20706F7765722075C3
:100F2000703A2000466163746F72792052455345D0
:100F3000540020202020334420205072696E7465B4
:100F4000727320202020002020204F726967696E74
:100F5000616C205072757361202020004F637420F3
:100F60003232203230313700436F6D70696C656406
:100F70003A2000286E6F6E652C2064656661756C82
:100F80007420636F6E66696729004F637420323284
:100F900020323031372032323A33373A343400732A
:100FA0007461727400202020203344202050726924
:100FB0006E7465727320202020002020204F7269FB
:100FC00067696E616C205072757361202020002566
:100FD000002020202020200020202020202000454C
:100FE000524153494E4720616C6C2064617461002A
:100FF000466163746F727920524553455400FFFF78
:10100000FF0000A0400000A0400000004000007F62
:101010004300005E439AD9514300000000000040A5
:10102000C19A99193E00007F4300005243000052CC
:101030004300000000000040C19A99193E656368B2
:101040006F3A004572726F723A0000002110422020
:1010500063308440A550C660E770088129914AA199
:101060006BB18CC1ADD1CEE1EFF131121002733210
:101070005222B5529442F772D662399318837BB3E9
:101080005AA3BDD39CC3FFF3DEE3622443342004A0
:101090000114E664C774A44485546AA54BB5288539
:1010A0000995EEE5CFF5ACC58DD5533672261116F0
:1010B0003006D776F6669556B4465BB77AA7199789
:1010C0003887DFF7FEE79DD7BCC7C448E558866878
:1010D000A7784008611802282338CCC9EDD98EE9D9
:1010E000AFF9488969990AA92BB9F55AD44AB77A50
:1010F000966A711A500A333A122AFDDBDCCBBFFB29
:101100009EEB799B588B3BBB1AABA66C877CE44C5F
:10111000C55C222C033C600C411CAEED8FFDECCD78
:10112000CDDD2AAD0BBD688D499D977EB66ED55E2F
:10113000F44E133E322E511E700E9FFFBEEFDDDFC8
:10114000FCCF1BBF3AAF599F788F8891A981CAB154
:10115000EBA10CD12DC14EF16FE18010A100C23086
:10116000E3200450254046706760B9839893FBA341
:10117000DAB33DC31CD37FE35EF3B1029012F322D6
:10118000D2323542145277625672EAB5CBA5A89591
:1011900089856EF54FE52CD50DC5E234C324A01426
:1011A00081046674476424540544DBA7FAB7998721
:1011B000B8975FE77EF71DC73CD7D326F236910676
:1011C000B01657667676154634564CD96DC90EF969
:1011D0002FE9C899E9898AB9ABA9445865480678C6
:1011E0002768C018E1088238A3287DCB5CDB3FEB81
:1011F0001EFBF98BD89BBBAB9ABB754A545A376A16
:10120000167AF10AD01AB32A923A2EFD0FED6CDD50
:101210004DCDAABD8BADE89DC98D267C076C645C65
:10122000454CA23C832CE01CC10C1FEF3EFF5DCF60
:101230007CDF9BAFBABFD98FF89F176E367E554EB5
:10124000745E932EB23ED10EF01E7C3C3E5E2B3D72
:101250003F2F5B5D3B2C2A225C004D383420582008
:1012600059205A2045004D3234004D323320257329
:10127000006175746F25692E67000A002F000A004F
:101280002E0044656C6574696F6E206661696C65DB
:10129000642C2046696C653A200046696C652064C0
:1012A000656C657465643A002E002E002E002E00D9
:1012B0004E6F772066726573682066696C653A20A8
:1012C000004E6F7720646F696E672066696C653ABF
:1012D00020002220706F73002220706172656E748E
:1012E0003A2200535542524F5554494E45204341EE
:1012F0004C4C207461726765743A2200747279698B
:101300006E6720746F2063616C6C207375622D674B
:10131000636F64652066696C657320776974682003
:10132000746F6F206D616E79206C6576656C732EBD
:10133000204D4158206C6576656C2069733A002514
:101340006920686F757273202569206D696E7574E8
:1013500065730054494D454F55543A004D31313075
:101360000046756C6C2052582042756666657200A6
:1013700022206661696C65643A2042756666657212
:101380002066756C6C2100456E717565696E67200D
:10139000746F207468652066726F6E743A20220044
:1013A0002200456E717565696E6720746F207468E0
:1013B000652066726F6E743A202200222066616991
:1013C0006C65643A204275666665722066756C6C61
:1013D000210022004D363030005043494E54320037
:1013E0005072757361206933204D4B3320726561F3
:1013F00064792E007A5F6D696E3A20007A5F6D61C4
:10140000783A20005A204F666673657400795F6DE4
:10141000696E3A2000795F6D61783A2000596573F2
:1014200000785F6D696E3A2000785F6D61783A20D0
:1014300000205761746368646F6720526573657438
:1014400000496E666F2073637265656E005761694F
:1014500074696E6720666F72206E6F7A7A6C652091
:10146000616E642062656420636F6F6C696E6700F3
:101470005761697420666F7220757365722E2E2E07
:10148000005573656420647572696E6720707269B7
:101490006E7400556E6C6F61642066696C616D6579
:1014A0006E7400556E6C6F6164696E672066696C5E
:1014B000616D656E7400556E6B6E6F776E20636F35
:1014C0006D6D616E643A20220054756E6500534460
:1014D0002063617264205B466C73684169725D00D1
:1014E00053442063617264205B6E6F726D616C5D4A
:1014F0000054656D702E2063616C2E205B4F4E5D35
:101500000054656D702E2063616C2E205B4F464643
:101510005D0054656D7065726174757265206361FC
:101520006C6962726174696F6E2069732066696E9E
:1015300069736865642E20436C69636B20746F2047
:10154000636F6E74696E75652E0054656D702E2024
:1015500063616C2E20202020202020202020005499
:10156000656D706572617475726500537570706F2A
:1015700072740053746F70207072696E74005354EB
:101580004F505045442E200053746570726174654D
:1015900020746F6F20686967683A2000546F746127
:1015A0006C207072696E742074696D65203A005405
:1015B0006F74616C2066696C616D656E74203A00B1
:1015C0005072696E742074696D653A202000466916
:1015D0006C616D656E7420757365643A20200053EC
:1015E0007461746973746963732020004572726F4B
:1015F00072202D20737461746963206D656D6F7244
:101600007920686173206265656E206F76657277F8
:1016100072697474656E0053706565640020536F61
:10162000667477617265205265736574004D6F64EE
:101630006520202020205B73696C656E745D004D11
:101640006F6465205B6869676820706F7765725D9D
:101650000053686F7720656E642073746F70730039
:101660005365742074656D70657261747572653A46
:101670000053657474696E677300576972696E67A9
:10168000206572726F720053656C662074657374A6
:10169000207374617274202000506C656173652042
:1016A000636865636B203A0053656C6620746573EC
:1016B00074204F4B004E6F7420636F6E6E656374C1
:1016C0006564004D6F746F72004865617465722FB8
:1016D000546865726D6973746F720046616E207430
:1016E0006573740053656C66746573742066616914
:1016F0006C65642020004C65667420686F74656EAC
:10170000642066616E3F0053656C66746573742077
:101710006572726F72202100456E6473746F702061
:101720006E6F742068697400456E6473746F7073B3
:1017300000456E6473746F700046726F6E74207033
:1017400072696E742066616E3F00436865636B6901
:101750006E67205A206178697320200043686563B2
:101760006B696E6720592061786973202000436897
:1017700065636B696E67205820617869732020006B
:10178000436865636B696E6720686F74656E64207B
:101790002000436865636B696E6720656E647374CF
:1017A0006F707300436865636B696E672062656480
:1017B000202020202000416C6C20636F72726563D2
:1017C0007420202020202000426564202F204865BE
:1017D000617465720041786973206C656E67746826
:1017E00000417869730053656C66746573742020DA
:1017F000202020202020200057726974696E672005
:10180000746F2066696C653A2000766F6C756D6543
:101810002E696E6974206661696C65640020536985
:101820007A653A2000436172642072656D6F766557
:1018300064005344207072696E74696E6720627927
:10184000746520006F70656E206661696C65642C3C
:101850002046696C653A20006F70656E526F6F7438
:10186000206661696C6564004361726420696E730F
:10187000657274656400534420696E697420666102
:10188000696C0046696C652073656C65637465649A
:101890000046696C65206F70656E65643A2000656E
:1018A00072726F722077726974696E6720746F202C
:1018B00066696C650053442063617264206F6B003D
:1018C00043616E6E6F7420656E746572207375620D
:1018D0006469723A2000526573756D696E67207095
:1018E00072696E7400526573756D696E67207072EF
:1018F000696E7400526573756D65207072696E74DF
:1019000000526573656E643A2000426C61636B6FD0
:101910007574206F636375727265642E20526563FF
:101920006F766572207072696E743F005265636FE6
:10193000766572696E67207072696E74202020204F
:1019400000686F77746F2E707275736133642E63E5
:101950006F6D00666F72756D2E7072757361336492
:101960002E636F6D00707275736133642E636F6DDB
:10197000005072696E7420706175736564005072F6
:10198000696E742061626F72746564005072696E72
:1019900074657220646973636F6E6E6563746564E9
:1019A00000616E6420707265737320746865206BCB
:1019B0006E6F62005072656865617420746865209E
:1019C0006E6F7A7A6C65210050726568656174008B
:1019D000506F776572557000506C65617365207744
:1019E000616974002020506C616E6E65724275668C
:1019F00066657242797465733A200050494E4441DD
:101A00002048656174696E67005049442063616CC9
:101A10002E2020202020202020202020005049445B
:101A20002063616C2E2066696E697368656400507E
:101A300049442063616C6962726174696F6E005021
:101A400061757365207072696E7400506C616365B6
:101A50002061207368656574206F66207061706511
:101A60007220756E64657220746865206E6F7A7A74
:101A70006C6520647572696E6720746865206361A7
:101A80006C6962726174696F6E206F66206669723C
:101A90007374203420706F696E74732E2049662031
:101AA000746865206E6F7A7A6C6520636174636810
:101AB0006573207468652070617065722C20706F8A
:101AC000776572206F666620746865207072696E33
:101AD00074657220696D6D6564696174656C792ED9
:101AE000006F6B004F6666004E6F206D6F76652E3F
:101AF000004E6F2053442063617264004E6F7A7A07
:101B00006C650046696C616D656E74206E6F742043
:101B10006C6F6164656400436F6C6F72206E6F74EC
:101B200020636C656172004E6F00506C6561736577
:101B300020757067726164652E004E657720666956
:101B4000726D776172652076657273696F6E206160
:101B50007661696C61626C653A004D6F7665205AFA
:101B6000004D6F76652059004D6F76652058004511
:101B700078747275646572004D6F7665206178695E
:101B800073004D65736820426564204C6576656C12
:101B9000696E670043616C6962726174696F6E009F
:101BA000206F662039004D6561737572696E67201C
:101BB0007265666572656E636520686569676874DD
:101BC000206F662063616C6962726174696F6E2058
:101BD000706F696E74004D61696E004D3232312054
:101BE000496E76616C69642065787472756465729B
:101BF00020004D32313820496E76616C6964206571
:101C00007874727564657220004D32303020496EF0
:101C100076616C6964206578747275646572200001
:101C20005265706F7274696E6720656E6473746F4D
:101C30007020737461747573004649524D57415258
:101C4000455F4E414D453A4D61726C696E2056318B
:101C50002E302E323B20537072696E7465722F677E
:101C600072626C206D617368757020666F72206798
:101C7000656E36204649524D574152455F55524C8C
:101C80003A68747470733A2F2F6769746875622E9E
:101C9000636F6D2F707275736133642F507275733B
:101CA000612D69332D506C75732F2050524F544F56
:101CB000434F4C5F56455253494F4E3A312E3020D8
:101CC0004D414348494E455F545950453A5072750D
:101CD0007361206933204D4B33204558545255448D
:101CE00045525F434F554E543A3120555549443A79
:101CF00030303030303030302D303030302D3030EA
:101D000030302D303030302D3030303030303030D9
:101D1000303030300A004D31303920496E76616CF8
:101D2000696420657874727564657220004D313085
:101D30003520496E76616C696420657874727564CB
:101D4000657220004D31303420496E76616C6964D3
:101D500020657874727564657220004C6F6F7365CE
:101D60002070756C6C6579004C6F61642066696CDD
:101D7000616D656E74004C6F6164696E67206669A1
:101D80006C616D656E74004C6F6164696E67206391
:101D90006F6C6F720053656C656374206C616E6765
:101DA00075616765004B494C4C45442E2000496ED7
:101DB00076616C6964206578747275646572004937
:101DC0006E736572742066696C616D656E74005027
:101DD00072696E742046414E3A20004E6F7A7A6CDA
:101DE000652046414E3A00457874727564657220EC
:101DF000696E666F00206F66203900496D70726FE2
:101E000076696E67206265642063616C69627261E5
:101E100074696F6E20706F696E740043616C6962E3
:101E2000726174696E67205A0043616C6962726105
:101E300074696F6E20646F6E650043616C696272D5
:101E4000617465205A0048656174696E6720646F2B
:101E50006E652E0048656174696E670046696C2E78
:101E60002073656E736F7220205B6F6E5D00466934
:101E70006C2E2073656E736F72205B6F66665D00FB
:101E80002046726565204D656D6F72793A20004677
:101E90006C6F770046696E697368696E67206D6F55
:101EA00076656D656E747300206F6620340053652F
:101EB00061726368696E67206265642063616C6942
:101EC00062726174696F6E20706F696E740049741C
:101ED00065726174696F6E2000446F6E6520736176
:101EE00076696E672066696C652E00446F6E6520AA
:101EF0007072696E74696E672066696C65004973FB
:101F000020636F6C6F7220636C6561723F00436881
:101F1000616E67652066696C616D656E740046610F
:101F20006E20737065656400656E717565696E67B6
:101F300020220045787472756465720020457874BB
:101F400065726E616C205265736574005072696EC3
:101F50007465722073746F70706564206475652099
:101F6000746F206572726F72732E204669782074C8
:101F70006865206572726F7220616E64207573658A
:101F8000204D39393920746F207265737461727411
:101F90002E202854656D70657261747572652069B4
:101FA000732072657365742E2053657420697420E4
:101FB00061667465722072657374617274696E67AC
:101FC00029004E6F204C696E65204E756D626572FA
:101FD000207769746820636865636B73756D2C2066
:101FE0004C617374204C696E653A20004E6F20433B
:101FF0006865636B73756D2077697468206C696EB2
:1020000065206E756D6265722C204C617374204C76
:10201000696E653A200020746F6F206C6F6E6720C8
:10202000657874727573696F6E2070726576656E0F
:10203000746564004C696E65204E756D6265722032
:102040006973206E6F74204C617374204C696E65E7
:10205000204E756D6265722B312C204C617374209B
:102060004C696E653A20005072696E746572206822
:10207000616C7465642E206B696C6C282920636127
:102080006C6C6564210020636F6C642065787472E9
:102090007573696F6E2070726576656E7465640025
:1020A000636865636B73756D206D69736D617463CF
:1020B000682C204C617374204C696E653A20004591
:1020C00052524F523A00456E642066696C65206C2E
:1020D000697374006F70656E0054524947474552EA
:1020E000454400656E6473746F7073206869743A58
:1020F0002000536C6565702E2E2E0044697361625A
:102100006C652073746570706572730043757272CC
:10211000656E74004372617368206465742E2020BC
:10212000205B6F6E5D004372617368206465742E7E
:1021300020205B6F66665D0020436F756E742058CB
:102140003A20004368616E67656420636F72726550
:1021500063746C793F00436F6F6C646F776E00201F
:102160004C61737420557064617465643A20004357
:10217000686F6F73652065787472756465723A0074
:102180004368616E676520737563636573732100CF
:102190005072696E742066726F6D205344005465EE
:1021A0006D702E2063616C6962726174696F6E007C
:1021B00043616C6962726174696E67205A2E2E2EBB
:1021C0000043616C69627261746500526573657485
:1021D0002058595A2063616C6962722E0043616C09
:1021E0006962726174652058595A002042726F7793
:1021F0006E206F757420526573657400426567695F
:102200006E2066696C65206C6973740058595A2099
:1022100063616C6962726174696F6E20636F6D7067
:10222000726F6D697365642E204C656674206672EA
:102230006F6E742063616C6962726174696F6E2085
:10224000706F696E74206E6F74207265616368616F
:10225000626C652E0058595A2063616C6962726124
:1022600074696F6E20636F6D70726F6D69736564F2
:102270002E2046726F6E742063616C6962726174A5
:10228000696F6E20706F696E7473206E6F74207248
:102290006561636861626C652E0058595A206361FC
:1022A0006C6962726174696F6E20616C6C20726916
:1022B0006768742E20582F592061786573206172E9
:1022C0006520736C696768746C7920736B657765DA
:1022D000642E20476F6F64206A6F62210058595A3C
:1022E0002063616C6962726174696F6E20616C6CED
:1022F0002072696768742E20536B65772077696C4C
:102300006C20626520636F7272656374656420611E
:1023100075746F6D61746963616C6C792E005859C6
:102320005A2063616C6962726174696F6E206661C4
:10233000696C65642E204265642063616C69627219
:102340006174696F6E20706F696E7420776173209D
:102350006E6F7420666F756E642E0058595A206334
:10236000616C6962726174696F6E206F6B2E2058A8
:102370002F592061786573206172652070657270D5
:10238000656E646963756C61722E20436F6E67724F
:102390006174756C6174696F6E73210058595A20AD
:1023A00063616C6962726174696F6E206661696CE9
:1023B00065642E20506C6561736520636F6E737564
:1023C0006C7420746865206D616E75616C2E0058A8
:1023D000595A2063616C6962726174696F6E20661C
:1023E00061696C65642E204C6566742066726F6E40
:1023F000742063616C6962726174696F6E20706FC2
:10240000696E74206E6F7420726561636861626CBE
:10241000652E0058595A2063616C69627261746953
:102420006F6E206661696C65642E2046726F6E74F3
:102430002063616C6962726174696F6E20706F698C
:102440006E7473206E6F7420726561636861626C74
:10245000652E00426564206C6576656C696E672048
:102460006661696C65642E2053656E736F722064BB
:102470006973636F6E6E6563746564206F72206349
:1024800061626C652062726F6B656E2E20576169A8
:1024900074696E6720666F722072657365742E00B2
:1024A000426564206C6576656C696E67206661695B
:1024B0006C65642E2053656E736F72206469646E60
:1024C0007420747269676765722E20446562726950
:1024D00073206F6E206E6F7A7A6C653F205761694A
:1024E00074696E6720666F722072657365742E0062
:1024F000426564206C6576656C696E67206661690B
:102500006C65642E2053656E736F722074726967F8
:10251000676572656420746F6F20686967682E2034
:1025200057616974696E6720666F722072657365A2
:10253000742E004265642048656174696E670042CC
:10254000656420646F6E6500526967687420736902
:1025500064655B756D5D00526573657400526561FD
:10256000722073696465205B756D5D00426564204F
:102570006C6576656C20636F7272656374004C6580
:1025800066742073696465205B756D5D0046726FCB
:102590006E7420736964655B756D5D0042656400EF
:1025A00044697374616E6365206265747765656EF6
:1025B00020746970206F6620746865206E6F7A7A67
:1025C0006C6520616E6420746865206265642073A8
:1025D00075726661636520686173206E6F74206236
:1025E00065656E20736574207965742E20506C6566
:1025F00061736520666F6C6C6F7720746865206D01
:10260000616E75616C2C2063686170746572204620
:10261000697273742073746570732C2073656374AE
:10262000696F6E204669727374206C6179657220DF
:1026300063616C6962726174696F6E2E004C6976B9
:10264000652061646A757374205A0041646A757309
:1026500074696E67205A004175746F20686F6D65EC
:1026600000207C20417574686F723A2000416C6CC8
:10267000004163746976652045787472756465728B
:102680003A2000E013F413FC1304140D1415141D68
:102690001421142914311441144D1470148114930D
:1026A00014A314B614C914CE14E014F114011512B5
:1026B000154A155F156B1573157E1588159C15AF9A
:1026C00015C015CE15DF15EC1517161D162D163F66
:1026D000165116601671167A1687169916A816B531
:1026E00016C316C916DB16E416F6160717181728B0
:1026F00017311739174A175C176E1780179217A4EE
:1027000017B617C817D517E117E617F8170A181DD7
:102710001825183218441858186818761883189114
:10272000189F18B518C018D618E518F41801190A1A
:10273000192C1941195319651971197E198C19A190
:1027400019B419C819D019D819E419FB19091A1D97
:102750001A2F1A3F1A4B1AE11AE41AE81AF11AFC56
:102760001A031B171B271B2A1B3A1B5A1B611B68CA
:102770001B6F1B781B821B941BA01BA61BD61BDB8D
:102780001BF21B091C201C391C161D2D1D441D5B32
:102790001D681D761D871D951DA51DAE1DBF1DCF76
:1027A0001DDB1DE71DF51DFB1D1B1E291E3A1E46C8
:1027B0001E541E5C1E6E1E801E8F1E941EA81EAE12
:1027C0001ECE1ED91EEB1EFE1E0E1F1E1F281F33FF
:1027D0001F3C1F4C1FC21FEC1F1620342067208691
:1027E00020A020BF20C620D420D920E320F220FB47
:1027F000200C21142126213821432156215F216FED
:1028000021802190219E21B021C121CB21DD21EB0E
:1028100021FC210C2255229A22DD221E235B239CBF
:1028200023CF2313245324A024F02433253F254809
:102830002557255D256C257E258D259C25A0253DCC
:10284000264B26572661266D267126457872656DC2
:1028500065207370616E206F6620746865205A2051
:1028600076616C7565732100626F74746F6D0074AE
:102870006F700000506F696E7420686569676874D6
:1028800020746F6F20736D616C6C3A200072696701
:102890006874006C6566740000506F696E74207710
:1028A0006964746820746F6F20736D616C6C3A207A
:1028B00000002C20003A200046696E616C206361A4
:1028C0006C63756C617465642062656420706F6907
:1028D0006E74200000793A000044697374616E637D
:1028E000652066726F6D206D696E3A000043616C01
:1028F00063756C6174696F6E206F66207468652003
:102900006D616368696E6520736B657720616E64C5
:10291000206F6666736574206661696C65642E005D
:10292000002C20003A200046696E616C206D6561C4
:1029300073757265642062656420706F696E7420BF
:102940000000206661696C65642E204C6F776572AB
:10295000696E67207A20746F20002C20697465727C
:102960006174696F6E2000496D70726F76696E6771
:102970002062656420706F696E742000002C207ADC
:10298000002C20697465726174696F6E2000496D56
:1029900070726F76696E672062656420706F696E11
:1029A000742000006C6F776572207468616E205926
:1029B0006D696E2E205920636F6F7264696E617449
:1029C0006520636C616D70696E6720776173207537
:1029D0007365642E0043616C6962726174696F6E25
:1029E00020706F696E742000417420595F4D494E0C
:1029F0005F504F5300417420593000496D70726F21
:102A000076696E6720626564206F66667365742000
:102A1000616E6420736B657700002C20002C200011
:102A200020004D656173757265642000002C2000E4
:102A300041646A757374656420706F736974696F3B
:102A40006E3A2000002C20683A002C20646D6178DA
:102A50003A005061727469616C20706F696E742005
:102A6000657374696D6174656420726164697573FE
:102A700020746F6F20736D616C6C3A2000005061A0
:102A8000727469616C20706F696E74206469616D25
:102A90006574657220746F6F20736D616C6C3A2081
:102AA00000746F70007269676874006C656674000A
:102AB0007269676874006C65667400746F70006694
:102AC00061696C6564202D206E6F7420666F756E71
:102AD000640A007269676874006C65667400002C93
:102AE0002000496E697469616C20706F7369746944
:102AF0006F6E3A200066696E642062656420696EBC
:102B000064756374696F6E2073656E736F72207085
:102B10006F696E74207A0059207365617263686909
:102B20006E67207261646975732068696768657291
:102B3000207468616E20585F4D41582E20436C61AF
:102B40006D70696E672077617320646F6E652E000B
:102B50005920736561726368696E67207261646988
:102B60007573206C6F776572207468616E20595F91
:102B70004D494E2E20436C616D70696E6720776100
:102B80007320646F6E652E005820736561726368F0
:102B9000696E67207261646975732068696768652A
:102BA00072207468616E20585F4D41582E20436C2E
:102BB000616D70696E672077617320646F6E652E3A
:102BC000005820736561726368696E672072616482
:102BD000697573206C6F776572207468616E205818
:102BE0005F4D494E2E20436C616D70696E67207792
:102BF000617320646F6E652E00536176696E672085
:102C00006265642063616C6962726174696F6E20D1
:102C1000766563746F727320746F20454550524F10
:102C20004D0050657270656E646963756C617269A0
:102C30007479005A65726F20706F696E7420636FCB
:102C40007272656374696F6E3A00592076656374B9
:102C50006F72206C656E6774683A00582076656301
:102C6000746F72206C656E6774683A00203C2000B7
:102C70005741524E494E473A2046726F6E7420704B
:102C80006F696E74206E6F74207265616368616233
:102C90006C652E205920636F6F7264696E61746574
:102CA0003A000070745B315D3A0070745B305D3ADD
:102CB00000004D656173757265643A00006375725A
:102CC00072656E745F706F736974696F6E5B5A5F63
:102CD000415849535D3A000063757272656E745FC6
:102CE000706F736974696F6E5B595F415849535DCA
:102CF0003A000063757272656E745F706F73697409
:102D0000696F6E5B585F415849535D3A00417420CA
:102D1000592D340041742059300000636E74725B89
:102D2000315D3A0000636E74725B305D3A0000768C
:102D300065635F795B315D3A00007665635F795B5F
:102D4000305D3A00007665635F785B315D3A000084
:102D50007665635F785B305D3A00566563746F72C9
:102D6000733A2000497465726174696F6E3A20008D
:102D7000496E76616C69642062656420636F72726B
:102D8000656374696F6E206D61747269782E20526C
:102D90006573657474696E6720746F206964656E0D
:102DA000746974792E00496E76616C69642062657D
:102DB0006420636F7272656374696F6E206D6174F5
:102DC0007269782E20582F592061786573206172BE
:102DD00065206661722066726F6D206265696E673C
:102DE0002070657270656E646963756C61722E0027
:102DF000496E76616C69642062656420636F7272EB
:102E0000656374696F6E206D61747269782E2053EA
:102E100068696674206F7574206F662072616E67D2
:102E2000652E005A65726F20706F696E7420636F33
:102E30007272656374696F6E3A00496E76616C698F
:102E4000642062656420636F7272656374696F6E7B
:102E5000206D61747269782E204C656E67746820ED
:102E60006F6620746865205920766563746F7220E0
:102E70006F7574206F662072616E67652E00592031
:102E8000766563746F72206C656E6774683A00498A
:102E90006E76616C69642062656420636F7272652E
:102EA0006374696F6E206D61747269782E204C6551
:102EB0006E677468206F6620746865205820766598
:102EC00063746F72206F7574206F662072616E6715
:102ED000652E005820766563746F72206C656E678E
:102EE00074683A00556E646566696E656420626553
:102EF0006420636F7272656374696F6E206D6174B4
:102F00007269782E00000043616C63756C617465B2
:102F1000206F666673657420616E6420736B6577DD
:102F20002072657475726E696E6720726573756C58
:102F3000743A000000292C206572726F723A2000EA
:102F40002C2000293B207461726765743A202800A8
:102F50002C2000293B206D656173757265642D63BB
:102F60006F727265637465643A2028002C20006DCE
:102F7000656173757265643A202800706F696E74BC
:102F8000202300446966666572656E63652061662C
:102F900074657220636F7272656374696F6E3A2034
:102FA00000002C200063656E7465722C2061646AD9
:102FB00075737465643A2000002C200059207665F2
:102FC00063746F722C2061646A75737465643A204F
:102FD00000002C20005820766563746F722C2061ED
:102FE000646A75737465643A200000636E74725B82
:102FF000315D3A0000636E74725B305D3A00466981
:103000006E616C20636E74722076616C7565733AC4
:103010000000000077793A0000636E74725B315DE6
:103020003A00005765696768745F793A00007778FD
:103030003A0000636E74725B305D3A000057656958
:103040006768745F783A000056657279206C69741D
:10305000746C6520736B6577206465746563746553
:10306000642E204F7274686F676F6E616C697A6945
:103070006E672074686520617865732E00004D616D
:10308000782E206572726F72206575636C69646951
:10309000616E3A004D61782E206572726F72205910
:1030A0003A004D61782E206572726F7220583A0096
:1030B0004D61782E206572726F72733A0000002C99
:1030C000206572726F7220593A20002C206572724E
:1030D0006F7220583A20006572726F723A20002990
:1030E000002C2000293B207461726765743A202807
:1030F000002C2000293B20636F7272656374656445
:103100003A2028002C20006D656173757265643A61
:10311000202800002C206572726F72203E206D61A5
:10312000782E206572726F72206575636C696469B0
:10313000616E00506F696E74206E6F74206F6E2028
:10314000666972737420726F77002C206572726FDB
:10315000722059203E206D61782E206572726F7248
:103160002059002C206572726F722058203E206D0D
:1031700061782E206572726F722058002C2077655E
:103180006967746820593A2000506F696E74206F27
:103190006E20666972737420726F77003A00706FE8
:1031A000696E742023004572726F722061667465C7
:1031B0007220636F7272656374696F6E3A200000EB
:1031C0002C200063656E746572206E65772C206913
:1031D0006E7665727465643A2000002C20005920D8
:1031E000766563746F72206E65772C20696E7665E4
:1031F000727465643A2000002C20005820766563C4
:10320000746F72206E65772C20696E7665727465B6
:10321000643A2000002C2000636F72726563746949
:103220006F6E20616E676C65733A2000002C200081
:10323000636F7272656374656420616E676C657339
:103240003A2000002C2000636F727265637465641D
:1032500020782F793A2000002C20002C20002C20F0
:10326000003B20636F7272656374696F6E207665D0
:1032700063746F723A2000697465726174696F6E6D
:103280003A200000292C206572726F723A20002CBF
:103290002000293B207461726765743A2028002C55
:1032A0002000206D656173757265643A2028007096
:1032B0006F696E74202300002C200063656E7465B6
:1032C000722C20696E697469616C3A2000002C20B0
:1032D000005920766563746F722C20696E69746979
:1032E000616C3A2000002C20005820766563746FD2
:1032F000722C20696E697469616C3A200063616C9C
:1033000063756C617465206D616368696E652073B7
:103310006B657720616E64206F6666736574204C00
:1033200053000000E442000000000000574300008A
:10333000C0420000E4420000404300004041000061
:10334000C04200004041000000000000E4420000D4
:103350000000000057430000000000005743000039
:10336000C0420000E4420000C042000040410000B2
:10337000C04200004041000040430000E442000021
:10338000404300005743000040435A00205A3A008F
:10339000590020593A00580020583A0024F4D430FB
:1033A00050C38E20C2A24017828B7011127A910DE9
:1033B000816CD90AA861E108C758660761514306C4
:1033C0001E4B5D05C145A7041A411104093D980330
:1033D000713931034036DB0265339102D430540237
:1033E000802E1D02632CEE01752AC501B028A001B4
:1033F000102781018F2564012B244B01E022340129
:10340000AC211F018D200D01801FFC00841EED00EA
:10341000971DDF00B81CD200E61BC600201BBC00B5
:10342000641AB200B219A8000A19A0006A1899001B
:10343000D117910040178B00B516840031167E001D
:10344000B31579003A157300C7146F0058146A0059
:10345000EE1366008813630025135E00C7125B003D
:103460006C12570015125400C111510070114F0019
:1034700021114B00D61049008D1047004610440022
:1034800002104200C00F4000800F3E00420F3C007F
:10349000060F3B00CB0E3800930E37005C0E350054
:1034A000270E3400F30D3200C10D3100900D3000B5
:1034B000600D2E00320D2D00050D2C00D90C2B00B7
:1034C000AE0C2900850C29005C0C2700350C270068
:1034D0000E0C2600E80B2400C40B2400A00B2300D4
:1034E0007D0B23005A0B2100390B2100180B200003
:1034F000F80A1F00D90A1E00BB0A1E009D0A1D0003
:10350000800A1D00630A1C00470A1B002C0A1B00CE
:10351000110A1A00F7091A00DD091900C409190077
:10352000AB091900920917007B09180063091700FD
:103530004C09160036091600200916000A09150064
:10354000F5081500E0081400CC081400B8081400B1
:10355000A4081400900813007D0812006B081300E3
:103560005808120046081200340811002308110000
:103570001208110001081100F0071000E007100008
:10358000D0071000C0071000B0070F00A1071000FF
:1035900091070E0083070F0074070F0065070E00E8
:1035A00057070E0049070E003B070D002E070E00BF
:1035B00020070D0013070D0006070D00F9060C008B
:1035C000ED060D00E0060C00D4060C00C8060C0049
:1035D000BC060C00B0060C00A4060B0099060C00FB
:1035E0008D060B0082060B0077060B006C060B00A5
:1035F00061060A0057060B004C060A0042060A0044
:1036000038060A002E060A0024060A001A060A00D6
:103610001006090007060A00FD050900F405090067
:10362000EB050900E2050900D9050900D0050900EC
:10363000C7050900BE050900B5050800AD0508006D
:10364000A50509009C050800940508008C050800E4
:10365000840508007C050800740508006C05070057
:10366000650508005D050700560508004E050700C2
:103670004705070040050800380507003105070029
:103680002A050700230507001C050600160507008C
:103690000F0507000805060002050700FB040600E9
:1036A000F5040700EE040600E8040600E204070043
:1036B000DB040600D5040600CF040600C90406009A
:1036C000C3040600BD040600B7040600B1040500EB
:1036D000AC040600A6040600A00405009B04060036
:1036E00095040500900406008A0405008504050081
:1036F000800406007A0405007504050070040500C6
:103700006B04050066040500610405005C04050007
:1037100057040500520405004D0405004804050047
:10372000430405003E0404003A0405003504050086
:10373000300404002C0405002704040023040500C1
:103740001E0404001A0404001604050011040400F9
:103750000D0404000904050004040400000404002E
:10376000FC030400F8030400F4030400F003040065
:10377000EC030400E8030400E4030400E003040095
:10378000DC030400D8030400D4030400D0030400C5
:10379000CC030400C8030300C503030024F404D9C8
:1037A000201BC40C5C0E9804C4095F0265077101FC
:1037B000F405F900FB04B30048048700C103690065
:1037C0005803550003034500BE023A00840231004D
:1037D00053022A002902250004022000E4011C00F3
:1037E000C8011900AF0117009801140084011300EB
:1037F000710110006101100051010E0043010D0024
:1038000036010B002B010B0020010B0015010900F4
:103810000C01090003010800FB000800F300080088
:10382000EB000700E4000600DE000600D8000600FA
:10383000D2000600CC000500C7000500C20005004C
:10384000BD000400B9000400B5000400B10004008C
:10385000AD000400A9000400A5000300A2000300BD
:103860009F0004009B0003009800030095000200E5
:1038700093000300900003008D0002008B00030002
:10388000880002008600020084000300810002001C
:103890007F0002007D0002007B0002007900020030
:1038A000770001007600020074000200720001003F
:1038B000710002006F0002006D0001006C00020048
:1038C0006A00010069000200670001006600010053
:1038D0006500010064000200620001006100010057
:1038E000600001005F0002005D0001005C0001005B
:1038F0005B0001005A00010059000100580001005E
:10390000570001005600010055000100540001005D
:10391000530000005300010052000100510001005B
:10392000500001004F0001004E0000004E00010059
:103930004D0001004C0001004B0000004B00010055
:103940004A00010049000100480000004800010051
:10395000470001004600000046000100450000004D
:103960004500010044000100430000004300010045
:10397000420000004200010041000000410001003F
:10398000400001003F0000003F0001003E00000039
:103990003E0001003D0000003D0001003C00000031
:1039A0003C0000003C0001003B0000003B00010027
:1039B0003A0000003A00010039000000390001001F
:1039C0003800000038000000380001003700000017
:1039D000370001003600000036000000360001000C
:1039E0003500000035000000350001003400000003
:1039F00034000000340001003300000033000000F8
:103A000033000100320000003200000032000100EB
:103A100031000000310000003100010030000000E2
:103A200030000000300001002F0000002F000000D7
:103A30002F0000002F0001002E0000002E000000CB
:103A40002E0001002D0000002D0000002D000000C0
:103A50002D0001002C0000002C0000002C000000B4
:103A60002C0001002B0000002B0000002B000000A8
:103A70002B0001002A0000002A0000002A0000009C
:103A80002A00010029000000290000002900000090
:103A90002900000029000100280000002800000083
:103AA0002800000028000000280001002700000076
:103AB0002700000027000000270000002700010069
:103AC000260000002600000026000000260000005E
:103AD0002600010025000000250000002500000050
:103AE0002500000025000000250001002400000042
:103AF0002400000024000000240000002400010035
:103B00002300000023000000230000002300000029
:103B10002300000023000000230001002200000019
:103B2000220000002200000022000000220000000D
:103B300022000100210000002100000021000000FF
:103B400021000000210000002100000021000100F0
:103B500020000000200000002000000020000000E5
:103B600020000000200000002000000020000100D4
:103B70001F0000001F0000001F0000001F000000C9
:103B80001F0000001F0000001F0001001E000000B9
:103B90001E0000001E0000001E0000004572723A68
:103BA000204D494E54454D50204245440054656DCA
:103BB00070657261747572652068656174656420F2
:103BC000626564207377697463686564206F6666F4
:103BD0002E204D494E54454D5020747269676765DB
:103BE0007265642021004572723A204D4158544557
:103BF0004D50204245440054656D70657261747586
:103C000072652068656174656420626564207377FD
:103C1000697463686564206F66662E204D41585450
:103C2000454D502074726967676572656420210094
:103C30004572723A204D494E54454D50003A204548
:103C400078747275646572207377697463686564EB
:103C5000206F66662E204D494E54454D502074729B
:103C6000696767657265642021004572723A204D6C
:103C7000415854454D50003A20457874727564653A
:103C800072207377697463686564206F66662E209E
:103C90004D415854454D502074726967676572658F
:103CA0006420210020484F54454E4420544845523A
:103CB0004D414C2052554E415741590020484541F5
:103CC0005442454420544845524D414C2052554E93
:103CD0004157415900544845524D414C2052554E90
:103CE000415741590042454420544845524D414CAA
:103CF0002052554E415741590020544845524D419C
:103D00004C2052554E415741592028205052454889
:103D100045415420484F54454E44290020544845BD
:103D2000524D414C2052554E415741592028205068
:103D30005245484541542048454154424544290094
:103D400050524548454154204552524F5200424539
:103D5000442050524548454154204552524F52004C
:103D60004572723A205052494E542046414E2045E9
:103D700052524F52004552524F523A205072696E81
:103D8000742066616E207370656564206973206CB1
:103D90006F776572207468656E20657870656374EE
:103DA0006564004572723A20455854522E204641AF
:103DB0004E204552524F52004552524F523A2045E2
:103DC000787472756465722066616E2073706565C3
:103DD00064206973206C6F776572207468656E204B
:103DE000657870656374656400202D20496E766186
:103DF0006C6964206578747275646572206E756D87
:103E0000626572202100504944204175746F7475B9
:103E10006E652066696E69736865642120507574EB
:103E200020746865206C617374204B702C204B6982
:103E300020616E64204B6420636F6E7374616E74D6
:103E4000732066726F6D2061626F766520696E7493
:103E50006F20436F6E66696775726174696F6E2E4D
:103E60006800504944204175746F74756E65206612
:103E700061696C6564212074696D656F75740020DB
:103E8000403A006F6B20543A006F6B20423A00506A
:103E90004944204175746F74756E65206661696C64
:103EA0006564212054656D7065726174757265205A
:103EB000746F6F206869676800204B643A200020A7
:103EC0004B693A2000204B703A200020436C61730C
:103ED0007369632050494420002054753A20002023
:103EE0004B753A2000206D61783A2000206D696E94
:103EF0003A200020643A200020626961733A200071
:103F000010137D002015780060177300C0196E0033
:103F1000401C6900E01E640080215F0040245A00BC
:103F2000F026550090295000202C4B00802E460092
:103F3000C0304100D0323C00B0343700503632003F
:103F4000C0372D0000392800103A2300F03A1E0037
:103F5000B03B1900503C1400D03C0F00303D0A002B
:103F6000803D0500C03D0000F03DFBFF103EF6FF28
:103F7000303EF1FF403EECFF503EE7FF603EE2FF87
:103F8000703EDDFF703ED8FF1000C90210012C0109
:103F90004001220170011801B0010E01F00104017D
:103FA0005002FA00B002F0003003E600D003DC005B
:103FB0009004D2007005C800A006BE000008B4003E
:103FC000B009AA00D00BA000600E960060118C0012
:103FD0000015820020197800C01D6E00A022640028
:103FE000B0275A00902C500000314600E0343C00CD
:103FF00010383200903A2800603C1E00A03D1400AA
:10400000803E0A00203F000070012C019001270132
:10401000B0012201C0011D01F001180110021301BD
:1040200030020E016002090190020401C002FF008B
:104030000003FA004003F5008003F000D003EB001A
:104040002004E6007004E100E004DC004005D70035
:10405000C005D2004006CD00D006C8008007C300CE
:104060003008BE00F008B900C009B400B00AAF00C3
:10407000B00BAA00D00CA500000EA000500F9B00B2
:10408000C01096005012910000148C00C0158700DB
:10409000B0178200B0197D00D01B7800001E73009D
:1040A00040206E0090226900F024640040275F00E9
:1040B00090295A00E02B5500102E500020304B0064
:1040C00010324600E033410090353C001037370095
:1040D00070383200A0392D00B03A2800A03B2300F0
:1040E000603C1E00103D1900903D1400103E0F0072
:1040F000703E0A00C03E0500003F0000544D4320C2
:10410000445249564552204F56455254454D502031
:1041100000436F6E74696E756520776974682061FD
:104120006E6F7468657220626F7764656E3F0047DA
:104130003736004D3435205A004D3435004738307D
:104140000020003E003E0020003E003E000053657F
:104150007665726520736B65773A0000536C69670A
:10416000687420736B65773A002D2D2D2D2D2D2D24
:104170002D2D2D2D2D2D2D2D2D2D2D2D2D004E2F79
:1041800041004D6561737572656420736B65773AA4
:1041900020004E2F41006D6D000052696768743A2F
:1041A0000043656E7465723A004C6566743A005956
:1041B0002064697374616E63652066726F6D206D33
:1041C000696E3A004D373031004D373032004D3591
:1041D0003030004731205A313520463135303000FB
:1041E0004739310047312058353020593139302096
:1041F000453020463730303000473930004D3730B9
:1042000032004D3730322043004D373032205500D8
:104210004D373032004731205A3135204631353064
:104220003000473931004731205835302059313975
:1042300030204530204637303030004D383300478D
:104240003930004D3834004D313034205330004780
:104250003930004731204531004D3832004D383378
:10426000004D31303620532564004D32323020531A
:104270002564003A2000202020202020202020201B
:1042800020202020202020202000203A2000202054
:10429000202020202020202020202020202020201E
:1042A000202000202020202020202020202020202E
:1042B000002573002020002D2D3A2D2D00200020F8
:1042C0000020004C002020002046002D2D2D003E17
:1042D000555342005344002D2D002520202020203E
:1042E000002020002020000120002020202D2D2D46
:1042F000200020205A002020000120004D363030C0
:1043000000464C4558202D20203233302F353000C8
:1043100050502020202D20203235342F31303000D5
:1043200048495053202D20203232302F3130300078
:1043300050455420202D20203234302F3930005069
:104340004C4120202D20203231352F35350041427F
:104350005320202D20203235352F313030004D3282
:1043600034004D323320257300052E2E005800599D
:10437000005A0045787472756465720047393900D7
:1043800044697361626C65206661726D206D6F6453
:10439000653F0044697361626C65206661726D20DF
:1043A0006D6F6465004661726D206E756D62657239
:1043B000004D3834005072696E742066616E3A00A8
:1043C00045787472756465722066616E3A00417852
:1043D0006973206C656E67746820646966666572CF
:1043E000656E63653A004D65617375726564206141
:1043F000786973206C656E6774683A004D383400D4
:104400004732382057005A30005A3100593000598D
:104410003100583000583100456E642073746F705D
:10442000732064696167004D343400473238205787
:10443000004175746F207265636F766572206372D8
:1044400061736800436865636B2066616E73205B0F
:104450004449535D00436865636B2066616E732059
:104460005B454E5D0054656D706572617475726573
:10447000730058595A2063616C2E20646574616919
:104480006C73002D2D2D2D2D2D2D2D2D2D2D2D0031
:10449000466C6173684169722049502041646472BE
:1044A0003A002D2D2D2D2D2D2D2D2D2D2D2D004F67
:1044B0006374203232203230313700446174653AFF
:1044C00020002D2D2D2D2D2D2D2D2D2D2D2D00456B
:1044D0003344763666756C6C0045494E595F30340E
:1044E0006100315F37356D6D5F4D4B33002D2D2DE4
:1044F0002D2D2D2D2D2D2D2D2D0020332E302E3117
:10450000322D5243322062313032004669726D776B
:104510006172653A0025642E25642E25642E25647B
:10452000004661696C207374617473004661726D3A
:10453000206E756D62657200007263006265746161
:1045400000616C706861006465760050525553419B
:104550003344465700332E302E31322D5243320031
:1045600000000A0B02090C0D0E08070304010000ED
:10457000000000000000000000000000000000003B
:1045800000000000000000000000000012111000F8
:10459000000000000000000000000000000000001B
:1045A000000000000000000000000000000000000B
:1045B0000000000000000102102020080810204028
:1045C00010204080020102010804020101020408D7
:1045D0001020408080402010080402018004020165
:1045E00080402010080402010804020101020408AE
:1045F00010204080010204081020408010080408A8
:1046000080102040044080102040048005050505EE
:10461000070508080808020202020A0A080804043A
:104620000404010101010101010103030303030368
:104630000303040707070C0C0C0C0C0C0C0C0202F7
:10464000020206060606060606060B0B0B0B0B0BF4
:104650000B0B07070A0A0A0A0A0A050505040404DF
:104660000808000020002300260029002C002F004D
:1046700032000001000003010601090100002200D0
:10468000250028002B002E0031003400020100001C
:10469000050108010B0100002100240027002A0069
:1046A0002D003000330001010000040107010A0160
:1046B000024E414E494E495459494E46CDCCCC3D0F
:1046C0000AD7233C17B7D13877CC2B329595E624FF
:1046D0001FB14F0A000020410000C84200401C46A4
:1046E00020BCBE4CCA1B0E5AAEC59D7400407A1049
:1046F000F35A00A0724E18090010A5D4E80000E893
:104700007648170000E40B54020000CA9A3B0000F0
:1047100000E1F505000080969800000040420F007F
:104720000000A08601000000102700000000E80340
:10473000000000006400000000000A00000000000B
:104740000100000000002C76D888DC674F0823DFCA
:10475000C1DFAE59E1B1B796E5E3E453C63AE6519D
:10476000997696E8E6C28426EB898C9B62ED407CC4
:104770006FFCEFBC9C9F40F2BAA56FA5F490055A60
:104780002AF75C936B6CF9676DC11BFCE0E40D4785
:10479000FEF520E6B500D0ED902E030094357705A8
:1047A0000080841E080000204E0A000000C80C3360
:1047B0003333330F986E12831141EF8D2114893BEF
:1047C000E65516CFFEE6DB18D1844B381BF77C1D6F
:1047D000901DA4BBE424203284725E228100C9F1C2
:1047E00024ECA1E53D275693DFB99F013D01E1018E
:1047F0007D9311241FBECFEFD1E2DEBFCDBF00E01D
:104800000CBF1AE0A0E0B2E0ECEFFCE703E00BBF66
:1048100002C007900D92AE30B107D9F72CE1AEE09F
:10482000BAE001C01D92A135B207E1F717E4C0EF6D
:10483000D7E400E006C022970109FE010BBF0F94E8
:10484000EEB4C63ED10780E00807A9F70F94A3AEE7
:104850000D946CBE0C940000CF92DF92EF92FF9209
:104860000F931F93CF93DF938C01D42EC62FD72F96
:10487000D60EDC1671F1F801E080F180C990C70115
:104880000F9430BBC816F1F06C2DC7010F9460BBBC
:10489000C7010F9430BB8C15A9F0EEE5F7E08491C9
:1048A000882341F09091C00095FFFCCF8093C60013
:1048B0003196F5CF8091C00085FFFCCF8AE08093D0
:1048C000C60007C0F80180819181019691838083A1
:1048D000D0CFDF91CF911F910F91FF90EF90DF909C
:1048E000CF900895EF92FF920F931F93CF93DF9392
:1048F0001F92CDB7DEB78C017B01460FF801808196
:10490000918149830F9430BBF70181937F01F801B6
:104910008081918101969183808349814E11EECFF0
:104920000F90DF91CF911F910F91FF90EF9008951D
:10493000FF920F931F93CF93DF93CDB7DEB72C97E2
:104940000FB6F894DEBF0FBECDBF8C01F62E80E30C
:1049500090E3A0E3B0E08D839E83AF83B8871C878C
:104960000B8744E0BE016B5F7F4FCE010B9674DF77
:1049700040E16DEA79E1CE010B966EDF40E16DEB2F
:1049800079E1CE010B9668DF40E16DE979E1CE0176
:104990000B9662DF44E065E979E1CE010B965CDFBE
:1049A00044E061E979E1CE010B9656DF44E069E924
:1049B00079E1CE010B9650DF44E06DE779E1CE015D
:1049C0000B964ADF44E06DEC79E1CE010B9644DFB3
:1049D00044E061E879E1CE010B963EDF44E065E812
:1049E00079E1CE010B9638DF44E069E879E1CE0148
:1049F0000B9632DF44E06DE879E1CE010B962CDFB7
:104A00004CE069E47BE0CE010B9626DF44E062E4F3
:104A10007BE0CE010B9620DF44E06DE972E0CE0131
:104A20000B961ADF44E069E972E0CE010B9614DFC1
:104A300044E065E972E0CE010B960EDF44E06DE8DC
:104A400072E0CE010B9608DF44E069E872E0CE0127
:104A50000B9602DF44E065E872E0CE010B96FCDEC7
:104A600080E290E09A87898742E0BE01675F7F4FCE
:104A7000CE010B96F1DE41E06EE37BE0CE010B96BA
:104A8000EBDE44E06DE172E0CE010B96E5DE44E042
:104A900065E172E0CE010B96DFDE44E069E37BE086
:104AA000CE010B96D9DE44E065E37BE0CE010B96A8
:104AB000D3DE44E061E172E0CE010B96CDDE41E051
:104AC00065E67BE0CE010B96C7DE44E06DE372E065
:104AD000CE010B96C1DE89E08F1560F444E06CECEA
:104AE00073E1CE010B96B8DE44E068EC73E1CE01D1
:104AF0000B96B2DE46E551E360E070E049835A83ED
:104B00006B837C831C870B8744E0BE016F5F7F4F04
:104B1000CE010B96A1DEEDE3F0E18491882341F014
:104B20009091C00095FFFCCF8093C6003196F5CFE1
:104B3000EEE4F7E08491882341F09091C00095FF66
:104B4000FCCF8093C6003196F5CF8091C00085FFE1
:104B5000FCCF8AE08093C6002C960FB6F894DEBF97
:104B60000FBECDBFDF91CF911F910F91FF900895A0
:104B70001F93CF93DF93182FCDE3D0E1FE018491F3
:104B8000882341F09091C00095FFFCCF8093C60030
:104B90003196F5CFEEE3F7E08491882341F09091D0
:104BA000C00095FFFCCF8093C6003196F5CF809171
:104BB000C00085FFFCCF8AE08093C600FE0184918F
:104BC000EDE3F0E1882349F09091C00095FFFCCF20
:104BD0008093C60031968491F5CF4091AD195091E4
:104BE000AE196091AF197091B01986E397E00E94F9
:104BF000933A4091B1195091B2196091B3197091E3
:104C0000B41983E397E00E94933A4091B51950910B
:104C1000B6196091B7197091B81980E397E00E94B6
:104C2000933A4091B9195091BA196091BB1970919A
:104C3000BC198DE297E00E94933A8091C00085FFF5
:104C4000FCCF8AE08093C600FE018491EDE3F0E1A1
:104C5000882349F09091C00095FFFCCF8093C60057
:104C600031968491F5CFE3E1F7E08491882341F018
:104C70009091C00095FFFCCF8093C6003196F5CF90
:104C80008091C00085FFFCCF8AE08093C600FE01C2
:104C90008491EDE3F0E1882349F09091C00095FF05
:104CA000FCCF8093C60031968491F5CF4091BD1919
:104CB0005091BE196091BF197091C0198AE097E0B8
:104CC0000E94933A4091C1195091C2196091C31941
:104CD0007091C41987E097E00E94933A4091C519FA
:104CE0005091C6196091C7197091C81984E097E076
:104CF0000E94933A4091C9195091CA196091CB19F9
:104D00007091CC1981E097E00E94933A8091C000A5
:104D100085FFFCCF8AE08093C600FE018491EDE31D
:104D2000F0E1882349F09091C00095FFFCCF80937B
:104D3000C60031968491F5CFE3EEF6E084918823A6
:104D400041F09091C00095FFFCCF8093C600319652
:104D5000F5CF8091C00085FFFCCF8AE08093C6002C
:104D6000FE018491EDE3F0E1882349F09091C000C9
:104D700095FFFCCF8093C60031968491F5CF40918A
:104D80009D1950919E1960919F197091A0198AEDFB
:104D900096E00E94A43A4091A1195091A219609105
:104DA000A3197091A41987ED96E00E94A43A40914E
:104DB000A5195091A6196091A7197091A81984EDB1
:104DC00096E00E94A43A4091A9195091AA196091C5
:104DD000AB197091AC1981ED96E00E94A43A8091D4
:104DE000C00085FFFCCF8AE08093C600FE0184915D
:104DF000EDE3F0E1882349F09091C00095FFFCCFEE
:104E00008093C60031968491F5CFECE9F6E0849169
:104E1000882341F09091C00095FFFCCF8093C6009D
:104E20003196F5CF8091C00085FFFCCF8AE080935A
:104E3000C600FE018491EDE3F0E1882349F09091F2
:104E4000C00095FFFCCF8093C60031968491F5CFCA
:104E500040919519509196196091971970919819F0
:104E600083E996E00E94933A4091911950919219EA
:104E7000609193197091941980E996E00E94933A99
:104E80008091C00085FFFCCF8AE08093C600FE01C0
:104E90008491EDE3F0E1882349F09091C00095FF03
:104EA000FCCF8093C60031968491F5CFEDEDF5E00F
:104EB0008491882341F09091C00095FFFCCF8093AE
:104EC000C6003196F5CF8091C00085FFFCCF8AE007
:104ED0008093C600FE018491EDE3F0E1882349F060
:104EE0009091C00095FFFCCF8093C60031968491CD
:104EF000F5CF4091991950919A1960919B19709131
:104F00009C1984ED95E00E94933A40917D1950914F
:104F10007E1960917F197091801981ED95E00E9452
:104F2000933A4091CD195091CE196091CF1970915B
:104F3000D0198EEC95E00E94A43A409181195091CD
:104F4000821960918319709184198BEC95E00E940D
:104F5000933A409185195091861960918719709103
:104F6000881988EC95E00E94933A409189195091F4
:104F70008A1960918B1970918C1985EC95E00E94CB
:104F8000933A40918D1950918E1960918F197091BB
:104F9000901982EC95E00E94933A8091C00085FFC1
:104FA000FCCF8AE08093C600FE018491EDE3F0E13E
:104FB000882349F09091C00095FFFCCF8093C600F4
:104FC00031968491F5CFE0EBF5E08491882341F0B0
:104FD0009091C00095FFFCCF8093C6003196F5CF2D
:104FE0008091C00085FFFCCF8AE08093C600FE015F
:104FF0008491EDE3F0E1882349F09091C00095FFA2
:10500000FCCF8093C60031968491F5CF4091490B37
:1050100050914A0B60914B0B70914C0B87EA95E0D5
:105020000E94933A40914D0B50914E0B60914F0B63
:105030007091500B84EA95E00E94933A4091510B95
:105040005091520B6091530B7091540B81EA95E093
:105050000E94933A8091C00085FFFCCF8AE0809344
:10506000C600FE018491EDE3F0E1882349F09091C0
:10507000C00095FFFCCF8093C60031968491F5CF98
:10508000E3E9F5E08491882341F09091C00095FF19
:10509000FCCF8093C6003196F5CF8091C00085FF8C
:1050A000FCCF8AE08093C600FE018491EDE3F0E13D
:1050B000882349F09091C00095FFFCCF8093C600F3
:1050C00031968491F5CF40919D0250919E0260915E
:1050D0009F027091A00289E895E00E94933A609146
:1050E000990270919A0280919B0290919C020F9478
:1050F0006C3FAB01BC0186E895E00E94933A609159
:1051000095027091960280919702909198020F9467
:10511000783FAB01BC0183E895E00E94933A80910F
:10512000C00085FFFCCF8AE08093C600FE01849119
:10513000EDE3F0E1882349F09091C00095FFFCCFAA
:105140008093C60031968491F5CFEDE6F5E0849129
:10515000882341F09091C00095FFFCCF8093C6005A
:105160003196F5CF8091C00085FFFCCF8AE0809317
:10517000C600FE018491EDE3F0E1882349F09091AF
:10518000C00095FFFCCF8093C60031968491F5CF87
:1051900040918D0250918E0260918F027091900229
:1051A00083E695E00E94933A6091890270918A02A9
:1051B00080918B0290918C020F946C3FAB01BC01EB
:1051C00080E695E00E94933A609185027091860294
:1051D00080918702909188020F94783FAB01BC01C7
:1051E0008DE595E00E94933A8091C00085FFFCCF49
:1051F0008AE08093C600FE018491EDE3F0E188230C
:1052000049F09091C00095FFFCCF8093C600319685
:105210008491F5CFE9E2F5E08491882341F0909103
:10522000C00095FFFCCF8093C6003196F5CF8091EA
:10523000C00085FFFCCF8AE08093C600FE01849108
:10524000EDE3F0E1882349F09091C00095FFFCCF99
:105250008093C60031968491F5CF40911D02509104
:105260001E0260911F02709120028FE195E00E9462
:10527000933A20E030E040E752E4609115027091EB
:10528000160280911702909118020F94A3B2AB01FD
:10529000BC018CE195E00E94933A4091390B50910A
:1052A0003A0B60913B0B70913C0B89E195E00E94B9
:1052B000933A8091C00085FFFCCF8AE08093C600BE
:1052C000FE018491EDE3F0E1882349F09091C00064
:1052D00095FFFCCF8093C60031968491F5CFEDEE1B
:1052E000F4E08491882341F09091C00095FFFCCFB9
:1052F0008093C6003196F5CF8091C00085FFFCCF2A
:105300008AE08093C600FE018491EDE3F0E18823FA
:1053100049F09091C00095FFFCCF8093C600319674
:105320008491F5CF4091350B5091360B6091370B3E
:105330007091380B83EE94E00E94933A20E030E0C5
:1053400040E752E4609111027091120280911302C1
:10535000909114020F94A3B2AB01BC0180EE94E0D3
:105360000E94933A8091C00085FFFCCF8AE0809331
:10537000C600FE018491EDE3F0E1882349F09091AD
:10538000C00095FFFCCF8093C60031968491F5CF85
:10539000E6E8F4E08491882341F09091C00095FF05
:1053A000FCCF8093C6003196F5CF8091C00085FF79
:1053B000FCCF8AE08093C600FE018491EDE3F0E12A
:1053C000882349F09091C00095FFFCCF8093C600E0
:1053D00031968491F5CF40913E0B50E060E070E053
:1053E0008CE794E00E94A43A8091C00085FFFCCF36
:1053F0008AE08093C600FE018491EDE3F0E188230A
:1054000049F09091C00095FFFCCF8093C600319683
:105410008491F5CF8091650B8823A1F1E9E6F4E052
:105420008491882341F09091C00095FFFCCF809338
:10543000C6003196F5CF8091C00085FFFCCF8AE091
:105440008093C600FE018491EDE3F0E1882349F0EA
:105450009091C00095FFFCCF8093C6003196849157
:10546000F5CF40913D0250913E0260913F02709114
:1054700040028FE594E00E94933A8091C00085FF3E
:10548000FCCF11C0E3E4F4E08491882341F09091D3
:10549000C00095FFFCCF8093C6003196F5CF809178
:1054A000C00085FFFCCF8AE08093C6001A3008F464
:1054B0003EC0FE01C491EDE3F0E1CC2349F08091C0
:1054C000C00085FFFCCFC093C6003196C491F5CFD4
:1054D000EAE2F4E08491882341F09091C00095FFC6
:1054E000FCCF8093C6003196F5CF8091C00085FF38
:1054F000FCCF8AE08093C6004091CC135091CD132D
:105500006091CE137091CF1380E294E00E94933AA1
:105510004091C8135091C9136091CA137091CB1375
:1055200086E194E0DF91CF911F910C94933ADF9143
:10553000CF911F910895AF92BF92CF92DF92EF92D9
:10554000FF920F931F93CF93DF93CDB7DEB7E09712
:105550000FB6F894DEBF0FBECDBF80E1E2EDF2E002
:10556000DE01919601900D928A95E1F780E1E2EEDD
:10557000F2E0DE01519601900D928A95E1F780E10B
:10558000E2EFF2E0DE01119601900D928A95E1F7CB
:105590006E0181E2C80ED11C8DEAE82E89E1F82E59
:1055A0008E010F5E1F4F6DEB79E1AE014F5F5F4FD4
:1055B0009DE9A92E99E1B92E20E030E0F601819114
:1055C0009191A191B1916F01F70181939193A19371
:1055D000B1937F01F80181919191A191B1918F01D6
:1055E000FB0181939193A193B193BF01FA01819142
:1055F0009191A191B191AF01F50181939193A19303
:10560000B1935F012F5F3F4F24303105B9F60F94FE
:10561000131C80E090E4ACE9B4E480939519909376
:105620009619A0939719B093981980939119909314
:105630009219A0939319B0939419109299191092FA
:105640009A1910929B1910929C1980E29EE4A0E096
:10565000B0E08093CD199093CE19A093CF19B09359
:10566000D01910927D1910927E1910927F19109204
:10567000801980E090E0A0E7B1E4809381199093D5
:105680008219A0938319B0938419809385199093FC
:105690008619A0938719B09388198DEC9CECACEC1B
:1056A000BEE38093891990938A19A0938B19B093C4
:1056B0008C1980E090E0A0E2B0E480938D19909383
:1056C0008E19A0938F19B09390191092510B1092CC
:1056D000520B1092530B1092540B10924D0B1092D0
:1056E0004E0B10924F0B1092500B1092490B1092D0
:1056F0004A0B10924B0B10924C0B8DE39AE0A1E8F1
:10570000B1E480939D0290939E02A0939F02B09378
:10571000A0026DEC7CEC84E99FE30F94663F6093FC
:10572000990270939A0280939B0290939C0265E881
:105730007BEE80E692E40F94723F60939502709343
:10574000960280939702909398020F94972E80E090
:1057500090E0A0E8BFE38093910290939202A0931F
:105760009302B093940210923E0B80E090E0A0E48C
:10577000B0E480931D0290931E02A0931F02B09389
:10578000200240E050E064E372E44093150250933D
:10579000160260931702709318021092390B109240
:1057A0003A0B10923B0B10923C0B1092350B10925F
:1057B000360B1092370B1092380B40E050E060E04F
:1057C00071E440931102509312026093130270939C
:1057D00014021092650B80933D0290933E02A093B9
:1057E0003F02B09340020E94EE4CEDE3F0E1849161
:1057F000882341F09091C00095FFFCCF8093C600B4
:105800003196F5CFEAEDF3E08491882341F0909151
:10581000C00095FFFCCF8093C6003196F5CF8091F4
:10582000C00085FFFCCF8AE08093C600E0960FB6EB
:10583000F894DEBF0FBECDBFDF91CF911F910F91C6
:10584000FF90EF90DF90CF90BF90AF9008951F939F
:10585000CF93DF93CDB7DEB72C970FB6F894DEBFAA
:105860000FBECDBF162F9C878B8786E591E3A0E006
:10587000B0E089839A83AB83BC8344E0BE016B5F55
:105880007F4FCE010B962ED843E050E0BE016B5FF8
:105890007F4FCE0101960F949FB8892B09F0FFC06E
:1058A00040E16DEA79E1CE010B961CD840E16DEB49
:1058B00079E1CE010B9616D840E16DE979E1CE0190
:1058C0000B9610D80F94131C44E065E979E1CE01E2
:1058D0000B9608D844E061E979E1CE010B9602D835
:1058E00044E069E979E1CE010B960E94722444E01C
:1058F0006DE779E1CE010B960E94722444E06DECD5
:1059000079E1CE010B960E94722444E061E879E1CE
:10591000CE010B960E94722444E065E879E1CE0145
:105920000B960E94722444E069E879E1CE010B965F
:105930000E94722444E06DE879E1CE010B960E944A
:1059400072244CE069E47BE0CE010B960E94722445
:1059500044E062E47BE0CE010B960E94722444E0B6
:105960006DE972E0CE010B960E94722444E069E971
:1059700072E0CE010B960E94722444E065E972E069
:10598000CE010B960E94722444E06DE872E0CE01D5
:105990000B960E94722444E069E872E0CE010B96F7
:1059A0000E94722444E065E872E0CE010B960E94EA
:1059B000722442E0BE01675F7F4FCE010B960E94CA
:1059C000722441E06EE37BE0CE010B960E947224CC
:1059D00044E06DE172E0CE010B960E94722444E037
:1059E00065E172E0CE010B960E94722444E069E307
:1059F0007BE0CE010B960E94722444E065E37BE0DD
:105A0000CE010B960E94722444E061E172E0CE0167
:105A10000B960E94722441E065E67BE0CE010B9676
:105A20000E94722444E06DE372E0CE010B960E9466
:105A300072241A3070F044E06CEC73E1CE010B96E6
:105A40000E94722444E068EC73E1CE010B960E9440
:105A500072240E94EE4C0F94972EEDE3F0E18491B6
:105A6000882341F09091C00095FFFCCF8093C60041
:105A70003196F5CFECEFF3E08491882341F09091DB
:105A8000C00095FFFCCF8093C6003196F5CF809182
:105A9000C00085FFFCCF8AE08093C60001C04BDDCB
:105AA0002C960FB6F894DEBF0FBECDBFDF91CF911D
:105AB0001F910895682F772767FD70958091AD102D
:105AC0009091AE108E549F4E0F9484B89093A41072
:105AD0008093A31021E0892B09F420E0822F089500
:105AE0008091A3109091A41060E070E001960D9455
:105AF0002DB58A3010F0895A01C0805D9091C000A8
:105B000095FFFCCF8093C6000895CF93C82F829550
:105B10008F70EFDF8C2F8F70CF91EBCFCF93C82F8B
:105B2000892FF3DF8C2FCF91F0CFCF93DF93FB0141
:105B300020E030E0DC01ED018D918823A1F14115D9
:105B4000510519F02417350774F58032A1F38A3016
:105B500051F190ED980F9A3020F4682F6295607F94
:105B600008C09FE9980F9630A8F4682F6295607F6F
:105B70006057CE0102967981A0EDA70FAA3018F4E4
:105B8000762F7A2B0CC0AFE9A70FA63018F4775503
:105B9000762B05C088279927821B930B05C071932C
:105BA0002F5F3F4FC7CFC901DF91CF910895E0919B
:105BB000A310F091A4108181882371F06AE573E04D
:105BC0008EE09AE0AED682E475DF882319F00C945B
:105BD00000F008950C9400000895CF93DF9365E6DC
:105BE00073E08EE09AE09DD6F894C0E0D0E060E0EB
:105BF000CE010F9460BB2196C11580E1D807B9F79B
:105C00007894DF91CF910895AF92BF92CF92DF92B7
:105C1000EF92FF920F931F93CF93DF93CDB7DEB731
:105C200060970FB6F894DEBF0FBECDBF67E773E095
:105C30008EE09AE076D681E43DDF8823A9F080915A
:105C4000A3109091A410FC012181283741F440E178
:105C500050E060E070E002960F9495B603C040DF1C
:105C60000F9411B07B0102C0E12CF12C83E422DF00
:105C7000882331F035DF0F9411B0262F872F02C013
:105C800020E080E2FFE1FF22022F182F013020E206
:105C9000120710F000E010E2C8018E0D9F1D813048
:105CA000904220F000E010E20E191F0988E502DFA3
:105CB000882371F18091A3109091A41040E150E0ED
:105CC000BE016F5F7F4F019630DF8C01009701F1BD
:105CD000FE013196CF01800F911FD701E817F90718
:105CE00019F021912D93FACF4AE050E0B8018EE0EF
:105CF0009AE076D66BE873E08EE09AE012D6C701A0
:105D00000DDF8091C00085FFFCCF8AE08093C60044
:105D100080E2B82E9AE0A92E0115110529F1C701DC
:105D2000FDDE8091C00085FFFCCFB092C600670108
:105D3000F0E1CF0ED11CF7012FEFE21AF20A8081B9
:105D40009091C00095FFFCCFB092C600DEDE0150FE
:105D5000110919F0EC14FD0471F78091C00085FF62
:105D6000FCCFA092C600D8CF60960FB6F894DEBFE5
:105D70000FBECDBFDF91CF911F910F91FF90EF909C
:105D8000DF90CF90BF90AF900895AF92BF92CF9227
:105D9000DF92EF92FF920F931F93CF93DF93CDB7D4
:105DA000DEB760970FB6F894DEBF0FBECDBF6CEACA
:105DB00073E08EE09AE0B5D581E47CDE8823A9F01B
:105DC0008091A3109091A410FC012181283741F407
:105DD00040E150E060E070E002960F9495B603C099
:105DE0007FDE0F9411B07B0102C0E12CF12C83E423
:105DF00061DE882331F074DE0F9411B0262F872FD7
:105E000002C020E080E2FFE1FF22022F182F0130C4
:105E100020E2120710F000E010E2C8018E0D9F1D75
:105E20008130904220F000E010E20E191F0988E551
:105E300041DE8823B1F18091A3109091A41040E13C
:105E400050E0BE016F5F7F4F01966FDE8C010097BF
:105E500041F1CE0101965C01C12CD12CC016D106B6
:105E600061F0F50161915F01C6018E0D9F1D0F94D8
:105E700060BBFFEFCF1ADF0AF1CF4AE050E0B80174
:105E80008EE09AE0ADD563EC73E08EE09AE049D500
:105E9000C70144DE8091C00085FFFCCF8AE080937B
:105EA000C60020E2B22E3AE0A32E0115110531F111
:105EB000C70134DE8091C00085FFFCCFB092C600E0
:105EC000670120E1C20ED11CC701EFEFEE1AFE0AF6
:105ED0000F9430BB9091C00095FFFCCFB092C600EC
:105EE00014DE0150110919F0EC14FD0469F78091DA
:105EF000C00085FFFCCFA092C600D7CF60960FB63A
:105F0000F894DEBF0FBECDBFDF91CF911F910F91EF
:105F1000FF90EF90DF90CF90BF90AF900895CF9219
:105F2000DF92EF92FF92CF93DF9367EE73E08EE004
:105F30009AE0F7D480E5BEDD882309F46BC0D0DD9C
:105F40000F9411B06B017C018FEFC816D10411F0D2
:105F500008F060C086E4AEDD882379F0C1DD0F94DF
:105F600011B06115710511F460E004C06130710574
:105F700021F461E08C2D0F94A7A886E59BDD882392
:105F8000B1F0AEDD0F9411B06115710511F460E050
:105F900005C06130710509F03DC061E08C2DDF91D5
:105FA000CF91FF90EF90DF90CF900D94E0A88C2DD3
:105FB0000F9415A9C1E0D0E0892B11F4C0E0D0E026
:105FC000E7EFF3E08191882339F09091C00095FFCD
:105FD000FCCF8093C600F6CF4AE050E0B6018EE0D9
:105FE0009AE0ACD4E6E2F5E08191882339F0909113
:105FF000C00095FFFCCF8093C600F6CF4AE050E08A
:10600000BE018EE09AE0DF91CF91FF90EF90DF909C
:10601000CF909BC4DF91CF91FF90EF90DF90CF9016
:106020000895CF93DF93EC0160E08E810F94E0A898
:1060300081E090E00F9422A761E08E810F94E0A8A8
:1060400081E090E00F9422A760E08E810F94E0A899
:1060500084E690E0DF91CF910D9422A7CF92DF925A
:10606000EF92FF920F931F93CF93DF937C01C0E0D9
:10607000D0E0C62ED12C87010C0F1D1F61E0F80166
:1060800087810F94A7A8B6010C2E02C0759567955D
:106090000A94E2F76170F80187810F94E0A82196D5
:1060A000C430D10541F7C701DF91CF911F910F9106
:1060B000FF90EF90DF90CF90B4CFCF92DF92EF922E
:1060C000FF920F931F93CF93DF937C01C0E0D0E04A
:1060D000C62ED12C87010C0F1D1F61E0F8018781AE
:1060E0000F94A7A8B6010C2E02C0759567950A9467
:1060F000E2F76170F80187810F94E0A82196C8301B
:10610000D10541F7C701DF91CF911F910F91FF900A
:10611000EF90DF90CF9085CF1F93CF93DF93EC016B
:10612000162F642F8C810F94E0A88D818F3F19F07A
:1061300060E00F94E0A88F85612F84FF05C0CE0139
:10614000DF91CF911F91B9CF70E084E0759567958D
:106150008A95E1F7CE0182DF612FCE01DF91CF91E9
:106160001F917CCF40E0D8CF61E0FCDF80E496E077
:106170000D9422A762E0F6DF80E496E00D9422A75A
:10618000CF93DF93CDB7DEB728970FB6F894DEBF75
:106190000FBECDBF28E0E2E0F3E0DE0111960190F2
:1061A0000D922A95E1F7FC012389421710F04FEF79
:1061B000420FFE013196E40FF11DE40FF11D208125
:1061C000260F2068622F28960FB6F894DEBF0FBE08
:1061D000CDBFDF91CF91C6CFFC016089262F24600F
:1061E000208B6C60BFCFCF93DF93EC01423018F06F
:1061F0008F8588608F874B8B1C8A222329F0413042
:1062000019F48F8584608F8780E593EC0F9422A723
:1062100060E08C810F94E0A860E08E810F94E0A88C
:106220008D818F3F19F060E00F94E0A86F8564FDC9
:1062300019C063E0CE0112DF84E991E10F9422A737
:1062400063E0CE010BDF84E991E10F9422A763E0C4
:10625000CE0104DF86E990E00F9422A762E0CE0130
:10626000FDDE13C06062CE017DDF84E991E10F9411
:1062700022A76F856062CE0175DF86E990E00F94FA
:1062800022A76F856062CE016DDF6F856062CE01EF
:1062900069DF8CE390E00F9422A784E0888BCE0125
:1062A0009BDF8CE390E00F9422A7CE015DDF88EBAB
:1062B0009BE00F9422A782E0898B66E0CE0152DF3B
:1062C0008CE390E0DF91CF910D9422A76F927F92A3
:1062D0008F92AF92CF92EF920F931F93CF93DF9352
:1062E000CDB7DEB73C01162F842F5E854F853889E8
:1062F0009989F301848325830683E782C086A1867A
:106300008286538744873587968761E00F94A7A8D4
:10631000F30185818F3F19F061E00F94A7A861E038
:10632000F30186810F94A7A8112319F0F3011786B2
:1063300003C080E1F301878720E041E060E1C30111
:10634000DF91CF911F910F91EF90CF90AF908F90F1
:106350007F906F9048CF8F92AF92CF92EF920F9332
:10636000DC0113961C921E921297EFEFF3E0ED936F
:10637000FC931F921F921F921F928C2CAE2CC02E4A
:10638000E22E042F2FEF462F61E0A0DF0F900F9039
:106390000F900F900F91EF90CF90AF908F90089546
:1063A000CF93DF93EC01423018F08F8588608F87A0
:1063B0004B8B1C8A222329F0413019F48F8584608D
:1063C0008F8780E593EC0F9422A760E08C810F9477
:1063D000E0A860E08E810F94E0A88D818F3F19F0D6
:1063E00060E00F94E0A86F8564FD19C063E0CE0102
:1063F00035DE84E991E10F9422A763E0CE012EDE21
:1064000084E991E10F9422A763E0CE0127DE86E9BB
:1064100090E00F9422A762E0CE0120DE13C06062FC
:10642000CE01A0DE84E991E10F9422A76F8560621E
:10643000CE0198DE86E990E00F9422A76F85606216
:10644000CE0190DE6F856062CE018CDE8CE390E041
:106450000F9422A784E0888BCE01BEDE8CE390E00F
:106460000F9422A7CE0186DE80E496E00F9422A747
:1064700082E0898B66E0CE0175DE8CE390E00F94BC
:1064800022A740E068E0CE017BDE65E879E0CE013E
:106490000F947BA941E068E0CE0172DE65E879E007
:1064A000CE010F947BA942E066E0CE0169DE63E88D
:1064B00079E0CE01DF91CF910D947BA9CF92DF924D
:1064C000EF92FF920F931F93CF93DF931F921F9230
:1064D000CDB7DEB78C01677088E0689FB0011124EA
:1064E0006064C80149835A833DDE4981C42E5A81C4
:1064F000D52EE12CF12CD6016D916D01D801ED91D5
:10650000FC910190F081E02DC8011995BFEFEB1AC5
:10651000FB0AE8E0EE16F10471F70F900F90DF919F
:10652000CF911F910F91FF90EF90DF90CF90089542
:1065300041E0F2DD81E090E008951F920F920FB6E6
:106540000F9211240BB60F922F933F934F935F93AB
:106550006F938F939F93EF93FF93CF93DF931F924C
:10656000CDB7DEB78091C00084FF04C08091C60023
:10657000898319C06091C60020918F0A3091900ADA
:10658000C90101968F7799274091910A5091920AFB
:106590008417950741F0F901E15FF54F608390930F
:1065A000900A80938F0A0F90DF91CF91FF91EF9126
:1065B0009F918F916F915F914F913F912F910F908C
:1065C0000BBE0F900FBE0F901F9018951F920F9249
:1065D0000FB60F9211240BB60F922F933F934F9348
:1065E0005F936F938F939F93EF93FF93CF93DF937B
:1065F0001F92CDB7DEB78091930A9091940A0197CC
:1066000009F58091D00084FF04C08091D600898371
:1066100019C06091D60020918F0A3091900AC9016B
:1066200001968F7799274091910A5091920A841789
:10663000950741F0F901E15FF54F60839093900A6F
:1066400080938F0A0F90DF91CF91FF91EF919F91EF
:106650008F916F915F914F913F912F910F900BBE52
:106660000F900FBE0F901F901895CF92DF92EF9270
:10667000FF926A017B01411581EE580761057105A2
:1066800009F463C082E08093C00060E079E08DE3AC
:1066900090E0A70196010F94B6B421503109410949
:1066A0005109CA01B90122E030E040E050E00F9406
:1066B000B6B491E03093C5002093C4008091C1002E
:1066C00080618093C1008091C10088608093C10087
:1066D0008091C10080688093C100992341F082E0DD
:1066E0008093D00060E079E08DE390E006C01092E6
:1066F000D00060E874E88EE190E0A70196010F9465
:10670000B6B42150310941095109CA01B90122E049
:1067100030E040E050E00F94B6B43093D5002093C1
:10672000D4008091D10080618093D1008091D1000C
:1067300088608093D1008091D10080688093D100DF
:10674000FF90EF90DF90CF9008951092C00090E0FE
:1067500020E130E0AFCF2091910A3091920A8091F0
:106760008F0A9091900A8217930771F0F901E15F07
:10677000F54F80812F5F3F4F2F7733273093920A59
:106780002093910A90E008958FEF9FEF08958091F4
:10679000910A9091920A9093900A80938F0A08959B
:1067A0004F925F926F927F928F929F92AF92BF9221
:1067B000CF92DF92EF92FF920F931F93CF93DF93CD
:1067C000CDB7DEB7A0970FB6F894DEBF0FBECDBF32
:1067D0005C014115510561057105E9F420E030E0E7
:1067E00040E350E060E070E0A0960FB6F894DEBFA2
:1067F0000FBECDBFDF91CF911F910F91FF90EF9012
:10680000DF90CF90BF90AF909F908F907F906F90D0
:106810005F904F905BC08E010F5F1F4FC12CD12C3A
:1068200076014801422E512C612C712C8FEFC81A31
:10683000D80AE80AF80ACB01BA01A30192010F9421
:1068400094B4CA01F80161938F01A901BC014115FB
:1068500051056105710551F7F1E0CF1AD108E10842
:10686000F108F401EC0DFD1D80818A3010F440E345
:1068700001C047E3480F552747FD5095652F752FF9
:1068800020E030E0C50122D081E0C81AD108E1083B
:10689000F108EFEFCE16DE06EE06FE0611F7A09623
:1068A0000FB6F894DEBF0FBECDBFDF91CF911F9121
:1068B0000F91FF90EF90DF90CF90BF90AF909F909F
:1068C0008F907F906F905F904F90089521153105C4
:1068D00039F48091C00085FFFCCF4093C600089535
:1068E0002A30310509F43FC05BCF9A01462F552766
:1068F00047FD5095652F752FE9CFCF93DF93EC01BE
:1069000020E030E04DE050E060E070E0DFDF20E0CC
:1069100030E04AE050E060E070E0CE01DF91CF91DE
:10692000D5CFFB012191BF01222339F03091C00066
:1069300035FFFCCF2093C600F4CFDFCF9A01AB0127
:10694000662757FD6095762FC1CFCF93DF93EC017B
:106950009A01AB01662757FD6095762FB7DFCE0110
:10696000DF91CF91CACFCF92DF92EF92FF92CF9378
:10697000DF93EC016A017B0177FF0FC020E030E07C
:106980004DE250E060E070E0A1DFF094E094D0943C
:10699000C094C11CD11CE11CF11C2AE0B701A60166
:1069A000CE01DF91CF91FF90EF90DF90CF90F8CEA6
:1069B0002115310539F48091C00085FFFCCF40934B
:1069C000C6000895EDCECF93DF93EC019A01462FD8
:1069D00050E060E070E0ECDFCE01DF91CF918DCF31
:1069E0009A01AB0160E070E0E3CFCF93DF93EC015D
:1069F0009A01AB0160E070E0DBDFCE01DF91CF9167
:106A00007CCFCF93DF93EC01D3DFCE01DF91CF9129
:106A100074CF8F929F92AF92BF92CF92DF92EF92FC
:106A2000FF921F93CF93DF93EC016A017B01122F3A
:106A300020E030E0A901C701B6010F94A2AF87FFA3
:106A40000CC020E030E04DE250E060E070E0CE01AC
:106A50003DDFF7FAF094F7F8F094B12C60E070E0C5
:106A600080E09FE3B11641F020E030E040E251E4E5
:106A70000F94A9AFB394F6CF9B01AC01C701B60147
:106A80000F94B2AE6B017C010F9416B04B015C0108
:106A90000F9442B09B01AC01C701B6010F94B1AE97
:106AA0006B017C012AE0B501A401CE0179DE11233E
:106AB00061F0E6E6F6E08191882339F09091C0001C
:106AC00095FFFCCF8093C600F6CF112319F120E08B
:106AD00030E040E251E4C701B6010F94A3B26B016C
:106AE0007C010F9411B04B01AA2497FCA094BA2CFE
:106AF000B501A401CE0137DFC501B4010F9444B044
:106B00009B01AC01C701B6010F94B1AE6B017C01D2
:106B10001150DBCFDF91CF911F91FF90EF90DF906D
:106B2000CF90BF90AF909F908F90089572CFCF93EA
:106B3000DF93EC016EDFCE01DF91CF91DECEFC0161
:106B400065917591859194910895EF92FF920F93BD
:106B50001F93CF93DF93EC01CC0FDD1FCC0FDD1F14
:106B6000CE01875E9F4EEBDF9E012B5A344F790199
:106B70008E01075B144FF8012081318142815381DE
:106B80000F94B2AEF7016083718382839383CE0149
:106B90008F5C9F4ED4DF9E01235D3D4F7901F8014C
:106BA00020813181428153810F94B2AEF70160831D
:106BB000718382839383CE018B5D9F4EC0DFCF5D57
:106BC000DD4FF80120813181428153810F94B2AEB3
:106BD000688379838A839B83DF91CF911F910F9183
:106BE000FF90EF900895CF93C82F40910C025091E1
:106BF0000D0260910E0270910F0240930C0B5093A6
:106C00000D0B60930E0B70930F0B20914702309188
:106C100048023093CB0B2093CA0B24E630E030932C
:106C20004802209347020F94BCA66093070B709311
:106C3000080B8093090B90930A0B8C2FCF910D9426
:106C4000C31D80E00F94C31D80910C0B90910D0B20
:106C5000A0910E0BB0910F0B80930C0290930D023C
:106C6000A0930E02B0930F028091CA0B9091CB0BB0
:106C700090934802809347020F94BCA66093070B41
:106C80007093080B8093090B90930A0B0895682F5B
:106C9000772767FD70958091AD109091AE108E545E
:106CA0009F4E0F9484B89093A4108093A31021E07A
:106CB000892B09F420E0822F08952091AD103091A6
:106CC000AE10BC01C9018E549F4E0F94BCB8909376
:106CD000A4108093A31021E0892B09F420E0822FD7
:106CE00008958091A3109091A4104AE050E060E0D4
:106CF00070E001960D9495B60F931F93CF93DF9399
:106D00000091A3101091A41065E470E0C8010F94E5
:106D100084B8EC01009751F460E070E0C80101967E
:106D2000DF91CF911F910F910D942DB51882809115
:106D3000A3109091A41060E070E001960F942DB51F
:106D400025E42883DF91CF911F910F9108958091C1
:106D5000A3109091A41060E070E001960D942DB501
:106D60002F923F924F925F926F927F928F929F925B
:106D7000AF92BF92CF92DF92EF92FF920F931F9349
:106D8000CF93DF93CDB7DEB760970FB6F894DEBF31
:106D90000FBECDBF1C012A013B014801590120E073
:106DA00030E04CE052E4C301B2010F94B1AE25E5EE
:106DB00035E547E052E40F94A9AF6B017C010F94D5
:106DC0007FB00F9411B08B0177FF12C020E030E04C
:106DD00040E85FE3C701B6010F94D1B118160CF07B
:106DE0005DC0C12CD12CE0E8EE2EEFE3FE2E56C0A4
:106DF00066307105DCF02AEA3AE24CE453E4C30160
:106E0000B2010F94B1AE25E535E547E052E40F94A9
:106E1000A9AF6B017C0120E030E0A9010F94A2AF83
:106E200087FF3FC0C12CD12C76013BC0882777FD5E
:106E30008095982F0F9444B025E535E547E052E45E
:106E40000F94A3B220E030E04CE052E40F94B2AED5
:106E50009B01AC01C301B2010F94B1AE25E535E54C
:106E600047E052E40F94A9AF6B017C0120E030E0D1
:106E7000A9010F94A2AF87FD17C020E030E040E8E1
:106E80005FE3C701B6010F94D1B1181684F4C12C89
:106E9000D12C70E8E72E7FE3F72E09C000E010E068
:106EA00006C005E010E003C0C12CD12C760120E023
:106EB00030E040EC50E4C501B4010F94B1AE2BEAD0
:106EC0003AEA42E052E40F94A9AF2B013C010F943F
:106ED0007FB00F9411B0788B6F8777FF12C020E0DE
:106EE00030E040E85FE3C301B2010F94D1B118165E
:106EF0000CF05FC0412C512C60E8662E6FE3762EBB
:106F000058C0AF85B8891697E4F026E535E549E223
:106F100053E4C501B4010F94B1AE2BEA3AEA42E062
:106F200052E40F94A9AF2B013C0120E030E0A9010D
:106F30000F94A2AF87FD40C0E5E0F0E0F88BEF874B
:106F400046C0882777FD8095982F0F9444B02BEA90
:106F50003AEA42E052E40F94A3B220E030E040EC81
:106F600050E40F94B2AE9B01AC01C501B4010F9483
:106F7000B1AE2BEA3AEA42E052E40F94A9AF2B01FA
:106F80003C0120E030E0A9010F94A2AF87FD1CC0B6
:106F900020E030E040E85FE3C301B2010F94D1B1DB
:106FA0001816ACF4412C512C50E8652E5FE3752E79
:106FB0000EC0188A1F860BC0412C512C320125E0CF
:106FC00030E0388B2F8703C0412C512C3201A701B0
:106FD000960160E070E080E89FE30F94B1AE6983B2
:106FE0007A838B839C83C80101969E838D83AF85B2
:106FF000B8891196BA87A987A301920160E070E071
:1070000080E89FE30F94B1AE6B877C878D879E8766
:1070100047E02F853889429FF001439FF00D1124EE
:10702000F887EF83E00FF11FEE0FFF1FEE0FFF1F3A
:10703000E20DF31D218132814381548169817A817E
:107040008B819C810F94A3B24B015C01EF81F88589
:107050008D819E81E80FF91FEE0FFF1FEE0FFF1FBE
:10706000E20DF31D2181328143815481C701B601B4
:107070000F94A3B29B01AC01C501B4010F94B2AE51
:107080009B01AC016B857C858D859E850F94A3B299
:107090004B015C0127E0E985FA852E9FD0012F9FE7
:1070A000B00D1124B887AF83FD01E00FF11FEE0F83
:1070B000FF1FEE0FFF1FE20DF31D2181328143817F
:1070C000548169817A818B819C810F94A3B26983F9
:1070D0007A838B839C83AF81B8858D819E81A80F35
:1070E000B91FAA0FBB1FAA0FBB1FA20DB31D11967C
:1070F0002D913D914D915C911497C701B6010F946C
:10710000A3B29B01AC0169817A818B819C810F9430
:10711000B2AE9B01AC01C301B2010F94A3B29B01BB
:10712000AC01C501B4010F94B2AE60960FB6F894ED
:10713000DEBF0FBECDBFDF91CF911F910F91FF90AA
:10714000EF90DF90CF90BF90AF909F908F907F9007
:107150006F905F904F903F902F9008954F925F9265
:107160006F927F929F92AF92BF92CF92DF92EF92F7
:10717000FF920F931F93CF93DF937C015B018A01F2
:10718000E9019090E512911014C0FC018081918179
:10719000A281B381FA0180839183A283B383FB012F
:1071A00080819181A281B38188839983AA83BB83E3
:1071B0007FC091FE55C0FC01208131814281538105
:1071C0006091D5127091D6128091D7129091D812F9
:1071D0000F94A3B22B013C01F50120813181428142
:1071E00053816091D9127091DA128091DB129091E3
:1071F000DC120F94A3B29B01AC01C301B2010F9446
:10720000B2AEF8016083718382839383F70120819A
:107210003181428153816091DD127091DE12809143
:10722000DF129091E0120F94A3B26B017C01F50183
:1072300020813181428153816091E1127091E2128B
:107240008091E3129091E4120F94A3B29B01AC01E0
:10725000C701B6010F94B2AE688379838A839B839A
:1072600090FE26C02091BD123091BE124091BF12F7
:107270005091C012F80160817181828193810F94D5
:10728000B2AEF80160837183828393832091C1122F
:107290003091C2124091C3125091C4126881798119
:1072A0008A819B810F94B2AE688379838A839B83A2
:1072B000DF91CF911F910F91FF90EF90DF90CF90D2
:1072C000BF90AF909F907F906F905F904F90089588
:1072D0002F923F924F925F926F927F928F929F92E6
:1072E000AF92BF92CF92DF92EF92FF920F931F93D4
:1072F000CF93DF93CDB7DEB728970FB6F894DEBFF4
:107300000FBECDBF8C011B019E012F5F3F4FAE0111
:107310004B5F5F4F23DF20E030E0A9016D817E816C
:107320008F8198850F94A2AF87FF07C01D821E82B0
:107330001F821886FF24F39401C0F12C20E030E076
:1073400040E451EC69817A818B819C810F94A2AFDA
:1073500087FF0AC080E090E0A0E4B1EC89839A83C3
:10736000AB83BC83FF24F39420E030E04FE753E489
:107370006D817E818F8198850F94D1B1181654F458
:1073800080E090E0AFE7B3E48D839E83AF83B8875E
:10739000FF24F39420E030E042E553E469817A81F0
:1073A0008B819C810F94D1B118164CF480E090E051
:1073B000A2E5B3E489839A83AB83BC8303C0FF2037
:1073C00009F483C0C980DA80EB80FC808D809E80C8
:1073D000AF80B8847090E51271100BC0F801808204
:1073E0009182A282B382F101C082D182E282F382D1
:1073F0006AC070FE1CC02091BD123091BE12409137
:10740000BF125091C012C501B4010F94B1AE4B012F
:107410005C012091C1123091C2124091C31250916F
:10742000C412C701B6010F94B1AE6B017C0171FEAD
:107430004AC02091C5123091C6124091C712509196
:10744000C812C501B4010F94A3B22B013C012091D5
:10745000C9123091CA124091CB125091CC12C7017F
:10746000B6010F94A3B29B01AC01C301B2010F940A
:10747000B2AEF80160837183828393832091CD1231
:107480003091CE124091CF125091D012C501B4016B
:107490000F94A3B24B015C012091D1123091D21212
:1074A0004091D3125091D412C701B6010F94A3B2E8
:1074B0009B01AC01C501B4010F94B2AEF101608330
:1074C000718382839383FF24F3948F2D28960FB6C4
:1074D000F894DEBF0FBECDBFDF91CF911F910F910A
:1074E000FF90EF90DF90CF90BF90AF909F908F90E4
:1074F0007F906F905F904F903F902F900895CF9323
:10750000DF931F92CDB7DEB7BE016F5F7F4F0F9441
:10751000195A0F90DF91CF910895682F87EF9FE060
:107520000D9442BB0895FC012491222341F0309137
:10753000C00035FFFCCF2093C6000196F4CF22E0B7
:1075400030E08EE09AE0F2CAFC012491222341F05F
:107550003091C00035FFFCCF2093C6000196F4CFD8
:107560002AE030E08EE09AE023CACF9363E074E033
:107570008EE09AE0D6D9C1E0C093A1026FEF89E610
:107580009FE00F9442BBC093CE02CF91089563E178
:1075900074E08EE09AE0C5D91092A10260E089E61D
:1075A0009FE00F9442BB1092CE020895EF92FF929B
:1075B0000F931F93CF93DF931F92CDB7DEB78983CD
:1075C0000F94DA558981823009F468C0B4F58823B4
:1075D00009F442C0813009F0F4C09FB7F89480915B
:1075E00002018460809302019FBFEFEFF1EE24E07F
:1075F000E150F0402040E1F700C000009FB7F89450
:10760000809102018B7F809302019FBF40E050E098
:10761000BA018DEE9FE00F9454BB40E050E0BA01F8
:1076200081EF9FE00F9454BB0F90DF91CF911F919A
:107630000F91FF90EF900D94527B833009F45CC062
:10764000843009F0BEC00F90DF91CF911F910F9150
:10765000FF90EF900D94C1839FB7F8948091020141
:107660008460809302019FBF2FEF81EE94E0215050
:1076700080409040E1F700C000009FB7F8948091EF
:1076800002018B7F809302019FBF0F90DF91CF910A
:107690001F910F91FF90EF900D9482560F94825698
:1076A00080EF3BDF1092EC1B1092EB1B6091ED1B07
:1076B00084EC9FE00F9442BB6BEE7BE181EC9FE09A
:1076C0000F9406569FB7F8948091020184608093CE
:1076D00002019FBF8FEF91EEE4E081509040E040C7
:1076E000E1F700C000009FB7F894809102018B7F02
:1076F000809302019FBF65C080EF9FE00F94626B93
:107700004FED5FE062E081E00F94B8879FB7F89497
:10771000809102018460809302019FBFFFEF21EE00
:1077200084E0F15020408040E1F700C000009FB7A6
:10773000F894809102018B7F809302019FBF109289
:10774000F30A1092F20A48ED5FE063E083E00F94E1
:10775000B8874091F20A5091F30A63E083E00F94F6
:10776000E555E12CF12C09E210E06FEFC7010F9411
:1077700060BBC701B8010F9481B4892BD9F4809103
:10778000F20A9091F30A01969093F30A8093F20A19
:1077900041ED5FE063E083E00F94B8874091F20A27
:1077A0005091F30A63E083E00F94E5558FEC9FE07E
:1077B0000F94626B9FEFE91AF90AE114E0E1FE060B
:1077C000A1F60F90DF91CF911F910F91FF90EF9055
:1077D000089580E1E5E5FBE0A0E2BBE001900D92B9
:1077E0008A95E1F708954F925F926F927F928F9200
:1077F0009F92AF92BF92CF92DF92EF92FF92CF9380
:10780000DF9300D01F92CDB7DEB70F9414278BE41F
:107810003EDA882391F070DA6B017C0120E030E0E1
:10782000A9010F94D1B187FD08C0C092CC13D092AA
:10783000CD13E092CE13F092CF1382E528DA88239D
:1078400059F05ADA6B017C0120E030E0A9010F9475
:10785000A2AF87FF83C006C0C12CD12C60E8E62E02
:107860006FEBF62E84E413DA882321F045DA4B011E
:107870005C0106C0812C912C50E8A52E5FEBB52E43
:1078800087E505DA882321F037DA2B013C0106C0B1
:10789000412C512C40E8642E4FEB742E88E4F7D92C
:1078A000882331F029DA69837A838B839C8308C02B
:1078B00080E090E0A0E8BFEB89839A83AB83BC8330
:1078C00020E030E0A901C501B4010F94D1B187FDDA
:1078D00045C020E030E0A901C301B2010F94D1B14D
:1078E00087FD3CC020E030E0A90169817A818B816D
:1078F0009C810F94D1B187FD31C020E030E0A90117
:10790000C501B4010F94A2AF882391F120E030E0CB
:1079100040E05FE3C501B4010F94A3B26B017C01A9
:1079200029813A814B815C81C301B2010F94A3B2DA
:107930004B015C01A7019601C701B6010F94A3B2E8
:107940002BED3FE049E450E40F94A3B29B01AC015E
:10795000C501B4010F94A9AF6B017C0120E030E0B8
:10796000A901C701B6010F94D1B187FF04C00BC0B4
:10797000C12CD12C7601C092C813D092C913E092C9
:10798000CA13F092CB13EDE3F0E18491882341F028
:107990009091C00095FFFCCF8093C6003196F5CF43
:1079A000EEE2FAE08491882341F09091C00095FFC7
:1079B000FCCF8093C6003196F5CF4091CC13509107
:1079C000CD136091CE137091CF1322E030E08EE0A2
:1079D0009AE0ACD88091C00085FFFCCF8AE080930C
:1079E000C600E8E2FAE08491882341F09091C0005B
:1079F00095FFFCCF8093C6003196F5CFC090C81399
:107A0000D090C913E090CA13F090CB1320E030E07F
:107A1000A901C701B6010F94A2AF882361F022E04B
:107A200030E0B701A6018EE09AE080D88091C000D6
:107A300085FFFCCF11C0E3E2FAE08491882341F096
:107A40009091C00095FFFCCF8093C6003196F5CF92
:107A50008091C00085FFFCCF8AE08093C6000F9024
:107A60000F900F900F90DF91CF91FF90EF90DF90EC
:107A7000CF90BF90AF909F908F907F906F905F90CE
:107A80004F9008952F923F924F925F926F927F9204
:107A90008F929F92AF92BF92CF92DF92EF92FF921E
:107AA0000F931F93CF93DF931F92CDB7DEB7E7E01D
:107AB000F8E28591949123DD81E00F94C31D8983C1
:107AC000E0E0F0E1E4918E2F992781950CF49095F8
:107AD0001C0184E00F94A642ADE5BBE01D921D920F
:107AE0001D921C921397E9E5FBE0208131814281D0
:107AF0005381A5E5BBE06D917D918D919C91E1E66F
:107B0000CE2EEBE0DE2EE12CF12C87010F944E1AE5
:107B100060DE85E190E113D82DEC3CEC4CE85FE3AE
:107B20000F94A3B24B015C01B101882777FD8095CA
:107B3000982F0F9444B09B01AC01C501B4010F9480
:107B4000A3B2E8E2FBE020813181428153810F94AE
:107B5000B2AE2B013C01A8E2BBE06D937D938D9307
:107B60009C931397E1E5F2E06081718182819381BA
:107B700060930C0270930D0280930E0290930F029B
:107B800020E030E040E752E40F94A9AF4B015C01E4
:107B9000A4E2BBE02D913D914D915C91E0E2FBE0D0
:107BA0006081718182819381A1E4BBE0BF93AF9337
:107BB000FCE2CF2EFBE0DF2E830172010F94A00DBB
:107BC00082E00F941B400F9414270F94264380E00B
:107BD0000F94C31DADE5BBE01D921D921D921C923A
:107BE0001397E9E5FBE02081318142815381A5E5CE
:107BF000BBE06D917D918D919C91A1E6CA2EABE089
:107C0000DA2EE12CF12C87010F944E1AE2DD2AE0E6
:107C1000229DC001239D900D1124BC01882777FD72
:107C20008095982F0F9444B0E8E2FBE020813181E9
:107C3000428153810F94B2AE2B013C01A8E2BBE01C
:107C40006D937D938D939C93139720E030E040E0FB
:107C50005FE3E1E5F2E060817181828193810F94BD
:107C6000A3B260930C0270930D0280930E02909366
:107C70000F0220E030E040E752E40F94A9AF4B013F
:107C80005C01A4E2BBE02D913D914D915C91E0E25D
:107C9000FBE06081718182819381A1E4BBE0BF93AD
:107CA000AF93BCE2CB2EBBE0DB2E830172010F94BD
:107CB000A00D0F94142789810F94C31D80E090E0DC
:107CC000AFE4B3E4EDE5FBE080839183A283B3836B
:107CD000A9E5BBE02D913D914D915C91E5E5FBE07F
:107CE000608171818281938111E6C12E1BE0D12ECA
:107CF000E12CF12C0FE413E40F944E1A81E00F9065
:107D00000F900F900F900F90DF91CF911F910F91D7
:107D1000FF90EF90DF90CF90BF90AF909F908F90AB
:107D20007F906F905F904F903F902F9008952F928B
:107D30003F924F925F926F927F928F929F92AF92FB
:107D4000BF92CF92DF92EF92FF920F931F93CF9348
:107D5000DF93CDB7DEB729970FB6F894DEBF0FBE1D
:107D6000CDBF3C0181E00F94C31D8F8382E0681674
:107D7000710408F081C2F301E250F04FE491D301A5
:107D8000AA0FBB1FAA0FBB1FBA83A983A75BBD4F56
:107D9000BE83AD838D919D910D90BC91A02D80935C
:107DA0000C0290930D02A0930E02B0930F0281E09B
:107DB000062C01C0880F0A94EAF70F94A642E981C5
:107DC000FA81EB5AF44FF987E88710821182128208
:107DD0001382E0905D0BF0905E0B00915F0B1091B1
:107DE000600B2091590B30915A0B40915B0B5091D5
:107DF0005C0B6091550B7091560B8091570B9091D5
:107E0000580BE1E6CE2EEBE0DE2E0F944E1AE98100
:107E1000FA81E05EF44F2F0180E090E0A0E4B0E44E
:107E200080839183A283B38320E030E040E752E473
:107E300060910C0270910D0280910E0290910F02E0
:107E40000F94A9AF4B015C01E090280BF090290B37
:107E500000912A0B10912B0B2091240B3091250BB4
:107E60004091260B5091270B6091200B7091210BB4
:107E70008091220B9091230BF1E42F2EFBE03F2EFB
:107E80003F922F92ACE2CA2EABE0DA2E0F94A00DF7
:107E90000F9414270F94AB1D80E00F94C31DA88589
:107EA000B9851D921D921D921C921397E0905D0B57
:107EB000F0905E0B00915F0B1091600B2091590BBD
:107EC00030915A0B40915B0B50915C0B6091550BBC
:107ED0007091560B8091570B9091580BB1E6CB2EB9
:107EE000BBE0DB2E0F944E1A80E090E0A0E8BFEBE1
:107EF000F20180839183A283B38320E030E040E7E6
:107F000052E460910C0270910D0280910E029091EA
:107F10000F020F94A9AF4B015C01E090280BF09089
:107F2000290B00912A0B10912B0B2091240B3091DF
:107F3000250B4091260B5091270B6091200B7091DF
:107F4000210B8091220B9091230B3F922F92ECE218
:107F5000CE2EEBE0DE2E0F94A00D0F94142781E0BF
:107F60000F94C31D89819A81835F9F4E0E949F3524
:107F70002DEC3CEC4CE85FEB0F94A3B2D2016D9377
:107F80007D938D939C93139720E030E040E752E47B
:107F900060910C0270910D0280910E0290910F027F
:107FA0000F94A9AF4B015C01E090280BF090290BD6
:107FB00000912A0B10912B0B2091240B3091250B53
:107FC0004091260B5091270B6091200B7091210B53
:107FD0008091220B9091230B3F922F920F94A00D32
:107FE0000F9414270F94AB1D80E00F94C31DE885F8
:107FF000F9851082118212821382E0905D0BF0905D
:108000005E0B00915F0B1091600B2091590B30912A
:108010005A0B40915B0B50915C0B6091550B70912A
:10802000560B8091570B9091580BF1E6CF2EFBE049
:10803000DF2E0F944E1A80E090E0A0E2B1E4F2014E
:1080400080839183A283B38320E030E040E752E451
:1080500060910C0270910D0280910E0290910F02BE
:108060000F94A9AF4B015C01E090280BF090290B15
:1080700000912A0B10912B0B2091240B3091250B92
:108080004091260B5091270B6091200B7091210B92
:108090008091220B9091230B3F922F92ACE2CA2E3B
:1080A000ABE0DA2E0F94A00D0F9414270F94AB1DA4
:1080B00081E00F94C31D80E090E0A0E7B1ECF201F5
:1080C00080839183A283B38320E030E040E05FE3CC
:1080D000AD81BE816D917D918D919C910F94A3B2E4
:1080E00060930C0270930D0280930E0290930F0226
:1080F00020E030E040E752E40F94A9AF4B015C016F
:10810000E090280BF090290B00912A0B10912B0B7B
:108110002091240B3091250B4091260B5091270B79
:108120006091200B7091210B8091220B9091230B79
:108130003F922F920F94A00D0F941427C3010E9419
:10814000A535F301EA5BF44F81E080830F94264369
:108150000F94AB1D80E00F94C31D2AE037ED43E27E
:108160005FE3E885F98560817181828193810F9455
:10817000B1AEA885B9856D937D938D939C9313972C
:10818000E0905D0BF0905E0B00915F0B1091600B27
:108190002091590B30915A0B40915B0B50915C0B25
:1081A0006091550B7091560B8091570B9091580B25
:1081B000B1E6CB2EBBE0DB2E0F944E1A2AE037ED52
:1081C00043E25FE3E885F985608171818281938173
:1081D0000F94B2AEA885B9856D937D938D939C93D2
:1081E0001397F20160837183828393832AE939E9CB
:1081F00049E95EE360910C0270910D0280910E02DC
:1082000090910F020F94A3B220E030E040E752E4D7
:108210000F94A9AF4B015C01E090280BF090290B63
:1082200000912A0B10912B0B2091240B3091250BE0
:108230004091260B5091270B6091200B7091210BE0
:108240008091220B9091230B3F922F92ECE2CE2E45
:10825000EBE0DE2E0F94A00D0F94142710920C0269
:1082600010920D0210920E0210920F020FB6F894A7
:10827000DEBF0FBECDBF62C192E06916710409F086
:108280005DC1E0E0F0E1749010925D0B10925E0B26
:1082900010925F0B1092600B2091590B30915A0B8A
:1082A00040915B0B50915C0B6091550B7091560B9C
:1082B0008091570B9091580BF1E6CF2EFBE0DF2E0B
:1082C000E12CF12C87010F944E1A85E190E10E9478
:1082D0009F354B015C01672D772767FD7095872FD0
:1082E000972F0F9444B02B013C0120E030E040EC8C
:1082F0005FE3C501B4010F94A3B2A30192010F94EF
:10830000A3B269837A838B839C836093280B7093D9
:10831000290B80932A0B90932B0B60915102709143
:108320005202809153029091540260930C02709318
:108330000D0280930E0290930F0220E030E040E7A0
:1083400052E40F94A9AF4B015C012091240B3091B2
:10835000250B4091260B5091270B6091200B7091BB
:10836000210B8091220B9091230BA1E42A2EABE0EC
:108370003A2E3F922F92BCE2CB2EBBE0DB2EE9805F
:10838000FA800B811C810F94A00D0F94142710927A
:108390005D0B10925E0B10925F0B1092600B2091A0
:1083A000590B30915A0B40915B0B50915C0B6091D3
:1083B000550B7091560B8091570B9091580B11E60D
:1083C000C12E1BE0D12EE12CF12C87010F944E1A07
:1083D00089E090E10E949F359058A30192010F948B
:1083E000A3B269837A838B839C836093280B7093F9
:1083F000290B80932A0B90932B0B20E030E040E771
:1084000052E460910C0270910D0280910E029091E5
:108410000F020F94A9AF4B015C012091240B309106
:10842000250B4091260B5091270B6091200B7091EA
:10843000210B8091220B9091230B3F922F920CE203
:10844000C02E0BE0D02EE980FA800B811C810F94A6
:10845000A00D0F94142789E090E10E949F359B01A5
:10846000AC010F94B2AEA30192010F94A3B22B0101
:108470003C016093280B7093290B80932A0B9093F7
:108480002B0B20E030E040E05FE3609151027091FF
:10849000520280915302909154020F94A3B26093C0
:1084A0000C0270930D0280930E0290930F0220E055
:1084B00030E040E752E40F94A9AF4B015C012091FA
:1084C000240B3091250B4091260B5091270B609186
:1084D000200B7091210B8091220B9091230B3F92E6
:1084E0002F92830172010F94A00D0F94142782E044
:1084F00090E00E94A53580915D0B90915E0BA0915C
:108500005F0BB091600B8093280B9093290BA09385
:108510002A0BB0932B0B10920C0210920D021092AA
:108520000E0210920F020F94AB1D81E08093480B56
:108530000F900F900F900F900F900F908F812996B2
:108540000FB6F894DEBF0FBECDBFDF91CF911F9164
:108550000F91FF90EF90DF90CF90BF90AF909F90E2
:108560008F907F906F905F904F903F902F900D94E1
:10857000C31DCF92DF92EF92FF920F931F9329D9E1
:1085800080E090E0D4DB81E090E0D1DBE0905D0B17
:10859000F0905E0B00915F0B1091600B2091590BD6
:1085A00030915A0B40915B0B50915C0B6091550BD5
:1085B0007091560B8091570B9091580BF1E6CF2E8E
:1085C000FBE0DF2E0F944E1A1F910F91FF90EF905A
:1085D000DF90CF900D94AB1D0F94BCA66093070B5A
:1085E0007093080B8093090B90930A0B089520E079
:1085F00030E0A90168EB71E084E50F940AAB69E112
:1086000070E080E090E00F94EBA684E50F9430AE2C
:1086100064E170E080E090E00D94EBA67F928F9291
:108620009F92AF92BF92CF92DF92EF92FF920F9301
:108630001F93CF93DF9300D01F92CDB7DEB7109278
:10864000E31A1092E21A1092E11A1092E01A0F94B3
:10865000DA5586ED9EE00F94626B8E010F5F1F4F1F
:108660007E0125E0E20EF11C8EE09AE00E94AB3321
:108670008F3FEFEF9E07C1F3F80181938F01EE1555
:10868000FF0591F789809A80AB80BC808091C00003
:1086900085FFFCCF8BE28093C600C12CD12C7601E4
:1086A000ABE27A2E8091910B882309F450C001EB44
:1086B0001AE0C814D904EA04FB04A1F08EE09AE0A1
:1086C0000E94AB338F3FFFEF9F07C1F32FEFC21A1A
:1086D000D20AE20AF20AF80181938F01FAE0013F1F
:1086E0001F0739F761EB7AE084ED9BE00E94DDAA79
:1086F0008091C00085FFFCCF7092C6000F94AA380D
:10870000C814D904EA04FB0469F671DF60E084ED63
:108710009BE00E9410AC1092910BE3ECF7E2859184
:108720009491FC012491222341F03091C00035FF47
:10873000FCCF2093C6000196F4CF8091C00085FF46
:10874000FCCF8AE08093C60080E090E000C00F90EC
:108750000F900F900F90DF91CF911F910F91FF908D
:10876000EF90DF90CF90BF90AF909F908F907F90D1
:1087700008950F94BCA66093070B7093080B809329
:10878000090B90930A0BE091AD10F091AE10E155FA
:10879000FF4E80818130B9F4E7E5F7E2859194914D
:1087A000FC012491222341F03091C00035FFFCCF21
:1087B0002093C6000196F4CF8091C00085FFFCCFC6
:1087C0008AE08093C60008958EE09AE00E94C73345
:1087D000EDE2F7E285919491FC012491222341F08E
:1087E0003091C00035FFFCCF2093C6000196F4CF36
:1087F0004091931050919410609195107091961043
:108800004F5F5F4F6F4F7F4F2AE030E08EE09AE07E
:108810000E9466348091C00085FFFCCF8AE080937F
:10882000C600A7CF8F929F92AF92BF92CF92DF9256
:10883000EF92FF920F931F93CF93DF93B2E1EB2E52
:10884000B6E0FB2E05E51BE0C0E2DBE08CECC82EB9
:108850008BE0D82EF70181917F010E944736882353
:1088600019F10E94A7364B015C01F601808181114C
:1088700003C060910B0B01C061E070E080E090E00C
:108880000F9444B0F80120813181428153810F94CB
:10889000A3B29B01AC01C501B4010F94B2AE6883D1
:1088A00079838A839B8309C0F80180819181A281A9
:1088B000B38188839983AA83BB830C5F1F4F24965F
:1088C000FFEFCF1ADF0A86E1E81686E0F80611F618
:1088D00086E40E9447368823D9F00E94A7366B01B0
:1088E0007C016093100B7093110B8093120B90938B
:1088F000130B20E030E0A9010F94D1B1181644F415
:10890000C0920C02D0920D02E0920E02F0920F0281
:10891000DF91CF911F910F91FF90EF90DF90CF905B
:10892000BF90AF909F908F9008957CDF89E40E9464
:108930004736882359F00E94A7366093140B709332
:10894000150B8093160B9093170B08C01092140B05
:108950001092150B1092160B1092170B8AE40E94BE
:108960004736882359F00E94A7366093180B7093FE
:10897000190B80931A0B90931B0B08951092180BF0
:108980001092190B10921A0B10921B0B0895CF9294
:10899000DF92EF92FF92CF93DF93EC01BC016C5F0B
:1089A0007F4F0E94683920E030E0A90160913502D4
:1089B0007091360280913702909138020F94B2AED6
:1089C0006B017C019B01AC01688579858A859B855B
:1089D0000F94A2AF87FF04C0C886D986EA86FB86BB
:1089E000C0902902D0902A02E0902B02F0902C0235
:1089F000A7019601688579858A859B850F94D1B1F9
:108A0000181624F4C886D986EA86FB86DF91CF91B2
:108A1000FF90EF90DF90CF9008952F923F924F926A
:108A20005F926F927F928F929F92AF92BF92CF92FE
:108A3000DF92EF92FF920F931F93CF93DF93CDB707
:108A4000DEB7AB970FB6F894DEBF0FBECDBF9F87E2
:108A50008E87798B688B5B8B4A8B3D8B2C8B1F8B26
:108A60000E8BED82DC018D909D90AD90BC9040907E
:108A7000550B5090560B6090570B7090580BDB01C4
:108A80008D919D910D90BC91A02D88879987AA8783
:108A9000BB87C090590BD0905A0BE0905B0BF090C5
:108AA0005C0B20915D0B30915E0B40915F0B509100
:108AB000600BEA89FB8960817181828193810F94C7
:108AC000B1AE688F798F8A8F9B8F8091E61281116A
:108AD00073C0AE89BF898D909D90AD90BC90EA899E
:108AE000FB89E080F18002811381A889B9892D91E9
:108AF0003D914D915C91EE85FF8560817181828110
:108B00009381FE013596FF93EF93CC88DD880F9417
:108B1000A00DEE85FF8580819181A281B381809334
:108B2000550B9093560BA093570BB093580BE889B5
:108B3000F98980819181A281B3818093590B9093AF
:108B40005A0BA0935B0BB0935C0BEA89FB89808185
:108B50009181A281B38180935D0B90935E0BA09372
:108B60005F0BB093600BEC89FD8980819181A281BC
:108B7000B3818093610B9093620BA093630BB093CE
:108B8000640B0F900F90AB960FB6F894DEBF0FBE3C
:108B9000CDBFDF91CF911F910F91FF90EF90DF90AC
:108BA000CF90BF90AF909F908F907F906F905F908D
:108BB0004F903F902F900895A3019201C501B401F9
:108BC0000F94B1AE2B013C0120E030E0A9010F94DD
:108BD000D1B153014201181624F0B7FAB094B7F896
:108BE000B094A7019601688579858A859B850F9445
:108BF000B1AE688779878A879B8720E030E0A9013A
:108C00000F94D1B1288539854A855B8518160CF0FB
:108C10005058C501B4010F94B2AE6B017C0120E045
:108C200030E0A9010F94D1B118160CF052CF20E01A
:108C300030E040EF51E4C701B6010F94A9AF0F94A3
:108C40008FAF0F9411B07D876C87623071050CF483
:108C500040CF2091610B3091620B4091630B50919A
:108C6000640BAC89BD896D917D918D919C910F9420
:108C7000B1AE6C8F7D8F8E8F9F8F22242394312CE9
:108C80008C859D85AA2797FDA095BA2F88A799A7BF
:108C9000AAA7BBA7DE011596BF83AE83B1018827C3
:108CA00077FD8095982F0F9444B06B017C0168A5E7
:108CB00079A58AA59BA50F9444B09B01AC01C7017F
:108CC000B6010F94A9AF6B017C01EE89FF8980800A
:108CD0009180A280B3802C8D3D8D4E8D5F8D0F9441
:108CE000A3B29B01AC016091610B7091620B80910A
:108CF000630B9091640B0F94B2AE69837A838B837C
:108D00009C83288D398D4A8D5B8DC701B6010F94E8
:108D1000A3B220915D0B30915E0B40915F0B50919F
:108D2000600B0F94B2AE68A379A38AA39BA3288596
:108D300039854A855B85C701B6010F94A3B220919E
:108D4000590B30915A0B40915B0B50915C0B0F9477
:108D5000B2AE6CA37DA38EA39FA3A3019201C70112
:108D6000B6010F94A3B22091550B3091560B409150
:108D7000570B5091580B0F94B2AEFF81FF932E8189
:108D80002F93DE0111966D01E8A0F9A00AA11BA1A5
:108D90002CA13DA14EA15FA10F94A00DBFEF2B1AF6
:108DA0003B0A0F900F90EC85FD852E163F0609F0CB
:108DB00075CF8FCE4F925F926F927F928F929F92DC
:108DC000AF92BF92CF92DF92EF92FF920F931F93D9
:108DD000CF93DF93CDB7DEB728970FB6F894DEBFF9
:108DE0000FBECDBF80E29BE0D2DD0F94BCA66093A6
:108DF000070B7093080B8093090B90930A0B8091DB
:108E0000200B9091210BA091220BB091230B8D830D
:108E10009E83AF83B8879C01AD016091550B709123
:108E2000560B8091570B9091580B0F94A2AF811164
:108E300097C04090240B5090250B6090260B7090AB
:108E4000270BA30192016091590B70915A0B8091ED
:108E50005B0B90915C0B0F94A2AF811181C020E05D
:108E600030E040E752E460910C0270910D02809175
:108E70000E0290910F020F94A9AF4B015C01E0909C
:108E8000280BF090290B00912A0B10912B0B81E4F9
:108E90009BE09F938F932CE2C22E2BE0D22EA30156
:108EA00092016D817E818F8198850F94A00D0F9026
:108EB0000F908091200B9091210BA091220BB091EB
:108EC000230B8093550B9093560BA093570BB093A5
:108ED000580B8091240B9091250BA091260BB091FB
:108EE000270B8093590B90935A0BA0935B0BB09375
:108EF0005C0B8091280B9091290BA0912A0BB091CB
:108F00002B0B80935D0B90935E0BA0935F0BB09344
:108F1000600B80912C0B90912D0BA0912E0BB0919A
:108F20002F0B8093610B9093620BA093630BB09314
:108F3000640B28960FB6F894DEBF0FBECDBFDF914D
:108F4000CF911F910F91FF90EF90DF90CF90BF9046
:108F5000AF909F908F907F906F905F904F9008950B
:108F6000E090410B6091470270914802882777FD9D
:108F70008095982F0F9444B020910C0230910D02EF
:108F800040910E0250910F020F94A3B22EE333ECE6
:108F90004EE259E30F94A3B269837A838B839C8357
:108FA0008E010F5F1F4F2CE23BE048E25BE064E282
:108FB0007BE080E29BE031DD7CCF4F925F926F924D
:108FC0007F928F929F92AF92BF92CF92DF92EF9259
:108FD000FF920F931F93CF93C62FE091410BF0E0C8
:108FE000882309F4D9C0DF01A35CB44F8C918111AF
:108FF000AFC18091550B9091560BA091570BB0913A
:10900000580B8093200B9093210BA093220BB093CD
:10901000230B8091590B90915A0BA0915B0BB0914F
:109020005C0B8093240B9093250BA093260BB0939D
:10903000270B80915D0B90915E0BA0915F0BB0911F
:10904000600B8093280B9093290BA0932A0BB0936D
:109050002B0BC090610BD090620BE090630BF090F3
:10906000640BC0922C0BD0922D0BE0922E0BF09241
:109070002F0BEE0FFF1FEE0FFF1FE75CFD4F208150
:10908000318142815381662349F0609119027091C8
:109090001A0280911B0290911C0208C060911D026F
:1090A00070911E0280911F02909120020F94A9AF2F
:1090B0009B01AC01C701B6010F94B2AE6093610B86
:1090C0007093620B8093630B9093640B81E69BE03B
:1090D0000F94ED1B80900C0290900D02A0900E0258
:1090E000B0900F0220E030E040E752E460911502BA
:1090F0007091160280911702909118020F94A3B2FA
:1091000060930C0270930D0280930E0290930F02F5
:10911000E091410BF0E0E35CF44F81E080834ADEB4
:109120002091390B30913A0B40913B0B50913C0B05
:1091300060915D0B70915E0B80915F0B9091600B65
:109140000F94B1AE7B018C0160935D0B70935E0B4D
:1091500080935F0B9093600B2091590B30915A0BC9
:1091600040915B0B50915C0B6091550B7091560BCD
:109170008091570B9091580BE1E6CE2EEBE0DE2E5E
:109180000F944E1A17DE80920C0290920D02A0925C
:109190000E02B0920F02DCC0E35CF44F80818823A2
:1091A00009F4D6C08090550B9090560BA090570BA9
:1091B000B090580B8092200B9092210BA092220B22
:1091C000B092230B4090590B50905A0B60905B0B60
:1091D00070905C0B4092240B5092250B6092260BF2
:1091E0007092270B60915D0B70915E0B80915F0B0D
:1091F0009091600B6093280B7093290B80932A0B3E
:1092000090932B0B0091610B1091620B2091630BDB
:109210003091640B00932C0B10932D0B20932E0B8D
:1092200030932F0B2091390B30913A0B40913B0B2F
:1092300050913C0B0F94B2AE7B018C0160935D0B9F
:1092400070935E0B80935F0B9093600B31E6C32E9F
:109250003BE0D32EA3019201C501B4010F944E1A35
:109260001091410BCC2389F02091310B3091320BBE
:109270004091330B5091340B6091190270911A0296
:1092800080911B0290911C0210C02091350B3091EF
:10929000360B4091370B5091380B60911D02709145
:1092A0001E0280911F02909120020F94B2AE24E022
:1092B000129FF0011124E75CFD4F20813181428132
:1092C00053810F94A9AF9B01AC016091610B709128
:1092D000620B8091630B9091640B0F94B1AE60931D
:1092E000610B7093620B8093630B9093640B81E628
:1092F0009BE00F94ED1BC0900C02D0900D02E0900B
:109300000E02F0900F0220E030E040E752E460915E
:1093100011027091120280911302909114020F9425
:10932000A3B260930C0270930D0280930E0290938F
:109330000F02E091410BF0E0E35CF44F10823ADD64
:10934000C0920C02D0920D02E0920E02F0920F0237
:10935000CF911F910F91FF90EF90DF90CF90BF9032
:10936000AF909F908F907F906F905F904F900895F7
:10937000AF92BF92CF92DF92EF92FF920F931F9323
:10938000CF93DF93D82F2091180B3091190B409178
:109390001A0B50911B0B6091140B7091150B80915F
:1093A000160B9091170B0F94DEB1C62F172F082FB5
:1093B000F92E6091470270914802882777FD8095C9
:1093C000982F0F9444B020910C0230910D024091DF
:1093D0000E0250910F020F94A3B220E030E040E75C
:1093E00052E40F94A9AF20E030E048EC52E40F942F
:1093F000A9AF2091410B2F93DF93FF920F931F93FF
:10940000CF935B016C01B2E0EB2E01E020E044E180
:109410005BE060E27BE085E59BE00F945204809185
:10942000200B9091210BA091220BB091230B8093E4
:10943000550B9093560BA093570BB093580B8091FC
:10944000240B9091250BA091260BB091270B8093B4
:10945000590B90935A0BA0935B0BB0935C0B8091CC
:10946000280B9091290BA0912A0BB0912B0B809384
:109470005D0B90935E0BA0935F0BB093600B80919C
:109480002C0B90912D0BA0912E0BB0912F0B809354
:10949000610B9093620BA093630BB093640B0F94DA
:1094A000BCA66093070B7093080B8093090B9093F5
:1094B0000A0B0F900F900F900F900F900F90DF916D
:1094C000CF911F910F91FF90EF90DF90CF90BF90C1
:1094D000AF900895EC01ECE1FAE08491882341F02B
:1094E0009091C00095FFFCCF8093C6003196F5CFD8
:1094F00070E04AE050E08EE09AE00E94A534F894D3
:109500000F944431179A1092460B169A1092470BFB
:10951000149AE3E4F0E18491882341F09091C00033
:1095200095FFFCCF8093C6003196F5CFEDEDF7E2C5
:1095300085919491FC012491222341F03091C00047
:1095400035FFFCCF2093C6000196F4CF8091C00078
:1095500085FFFCCF8AE08093C6002097C9F0FE010A
:109560008491FE01882349F09091C00095FFFCCFC3
:109570008093C60031968491F5CF8091C00085FF1D
:10958000FCCF8AE08093C600CE010E947F3A06C0DD
:10959000E9E9F7E2859194910F9417577894C6E022
:1095A000D0E0219751F068EC70E080E090E00F94FB
:1095B000EBA680E00F947058F4CFF894FFCFCF92D1
:1095C000DF92EF92FF920F931F93CF93C82F80915A
:1095D000A9109091AA10039714F40E9461B40F94FB
:1095E000BCA60091030B1091040B2091050B309148
:1095F000060BC090070BD090080BE090090BF09081
:109600000A0B6C197D098E099F0906171707280791
:10961000390740F4012B022B032B21F064E082EC8C
:1096200098E058DF409108025091090260910A02C7
:1096300070910B02452B462B472B19F10F94BCA6BA
:109640000091070B1091080B2091090B30910A0B28
:10965000601B710B820B930B0091080210910902A1
:1096600020910A0230910B020617170728073907C5
:1096700040F49091D1138091D013981302C0CC2361
:1096800049F0CF911F910F91FF90EF90DF90CF9015
:109690000D94CE0B179A1092460B169A1092470B08
:1096A000149AEFCF0F9444318091F50A81113DC097
:1096B00081E08093F50A8091931090919410A0918D
:1096C0009510B091961080938F1090939010A09366
:1096D0009110B0939210E3E4F0E18491882341F07B
:1096E0009091C00095FFFCCF8093C6003196F5CFD6
:1096F000E3EDF7E285919491FC012491222341F05E
:109700003091C00035FFFCCF2093C6000196F4CF06
:109710008091C00085FFFCCF8AE08093C600E9EB12
:10972000F6E2859194910D94F15608958091F50A91
:109730000895CF93DF93EC018091410B8093F60A5B
:1097400084E50E944736811102C080E084C00E94F7
:10975000A7360F9416B06093F60A6623B1F3EDE3D3
:10976000F0E18491882341F09091C00095FFFCCFF7
:109770008093C6003196F5CFCD36D10509F435C0BA
:1097800064F4C836D105B1F0C936D10509F052C02C
:10979000EBE8F7E2A591B49124C0CA3DD10509F4E4
:1097A00032C0CD3DD10509F045C0EFE7F7E2A59104
:1097B000B4913DC0EDE8F7E285919491FC012491CC
:1097C000222309F437C03091C00035FFFCCF20932D
:1097D000C6000196F3CF9091C00095FFFCCF809317
:1097E000C6008D918111F7CF25C0E9E8F7E2A59178
:1097F000B4918D918823F1F09091C00095FFFCCF3A
:109800008093C600F6CFE1E8F7E2A591B4918D917F
:10981000882381F09091C00095FFFCCF8093C60013
:10982000F6CF9091C00095FFFCCF8093C6008D913C
:109830008111F7CF6091F60A70E04AE050E08EE0C7
:109840009AE00E949E348091C00085FFFCCF8AE0A0
:109850008093C60081E0DF91CF9108954F925F928F
:109860006F927F928F929F92AF92BF92CF92DF9230
:10987000EF92FF92CF93DF9300D01F92CDB7DEB768
:109880002B013C0129833A834B835C838DEE9FE05F
:109890000F9430BB8F3F01F58EEE9FE00F9430BBED
:1098A0008F3FD1F48FEE9FE00F9430BB8F3FA1F438
:1098B00080EF9FE00F9430BB8F3F71F440E050E0A9
:1098C000BA018DEE9FE00F9454BB40E050E0BA0126
:1098D00081EF9FE00F9454BB81EF9FE00F9438BB62
:1098E0004B015C018DEE9FE00F9438BB6B017C0156
:1098F00069817A818B819C812CE330E040E050E0EB
:109900000F9494B4C20ED31EE41EF51EB701A60137
:109910008DEE9FE00F9454BBC301B20128EE33E0FB
:1099200040E050E00F9494B4BA01A901480D591DCC
:109930006A1D7B1D81EF9FE00F9454BB10928B0B2F
:1099400010928C0B10928D0B10928E0B0F900F902B
:109950000F900F90DF91CF91FF90EF90DF90CF901D
:10996000BF90AF909F908F907F906F905F904F903F
:109970000895CF92DF92EF92FF922091650B222300
:10998000F1F020E030E040E05FE30F94A3B26B0120
:109990007C0120E030E0A9010F94A2AF882379F088
:1099A000A7019601C701B6010F94A3B22BED3FE0CA
:1099B00049E450E40F94A3B29B01AC0104C020E041
:1099C00030E040E85FE360E070E080E89FE30F9400
:1099D000A9AFFF90EF90DF90CF90089560913D0286
:1099E00070913E0280913F0290914002C2DF6093ED
:1099F000390270933A0280933B0290933C0208959F
:109A0000CF93DF93EC010F94AA3881E0D8DD80E09A
:109A10000F947058209799F0C233D10540F062E35B
:109A200070E080E090E00F94EBA6E297ECCFBE01EF
:109A300080E090E00F94EBA6C0E0D0E0E4CFDF91AF
:109A4000CF9108952F923F924F925F926F927F92A3
:109A50008F929F92AF92BF92CF92DF92EF92FF923E
:109A60001F93CF93DF934B015C01CC24CA94DC2C71
:109A7000760151E1252E5AE0352E68EE462E63E040
:109A8000562E612C712C1AE08091300B811126C169
:109A90002FEFC216D206E206F20651F0F7FC1EC105
:109AA0000F94BCA66C197D09683B7B4008F016C179
:109AB0000F94BCA6681979098A099B09693E73400D
:109AC0008105910508F47FC08091ED1B811177C05D
:109AD000E9E1FAE08491882341F09091C00095FF7C
:109AE000FCCF8093C6003196F5CFE091F60A24E0D2
:109AF000E29FF0011124E652F54E408151816281CE
:109B0000738121E030E08EE09AE00E949635E5E135
:109B1000FAE08491882341F09091C00095FFFCCF3A
:109B20008093C6003196F5CF6091F60A70E04AE066
:109B300050E08EE09AE00E949E34F1018491E1E1D0
:109B4000FAE0882349F09091C00095FFFCCF809304
:109B5000C60031968491F5CFF7FE03C0E3E9F9E042
:109B600025C00F94BCA64B015C01C701B601685427
:109B7000744F8F4F9F4F681979098A099B09A30178
:109B800092010F9494B4BA01A9012AE030E08EE06A
:109B90009AE00E9466348091C00085FFFCCF0DC022
:109BA0009091C00095FFFCCF8093C60081918111F8
:109BB000F7CF8091C00085FFFCCF1093C6000F94B3
:109BC000BCA64B015C010F94AA3880E0F8DC80E071
:109BD0000F947058FFEFCF16DF06EF06FF0609F06F
:109BE00046C08091F40AE091F60AF0E0EF01CC0F54
:109BF000DD1FCC0FDD1FC652D54EEE0FFF1FEE51FD
:109C0000F54E8823D1F080819181BC01882777FDB2
:109C10008095982F0F9444B020E030E040E85FE357
:109C20000F94B1AE9B01AC01688179818A819B81DF
:109C30000F94D1B187FF4DC027CF80819181BC01A6
:109C4000882777FD8095982F0F9444B020E030E06E
:109C500040E85FE30F94B2AE9B01AC01688179816B
:109C60008A819B810F94A2AF18169CF50DCFF7FC4B
:109C70000BCFE091F60AF0E0EF01CC0FDD1FCC0F27
:109C8000DD1FC652D54EEE0FFF1FEE51F54E8081FF
:109C90009181BC01882777FD8095982F0F9444B05F
:109CA0009B01AC01688179818A819B810F94B1AE5F
:109CB0000F9411B097FF07C09095809570956195AE
:109CC0007F4F8F4F9F4F66307105810591050CF4D2
:109CD000DBCE0F94BCA66B017C01D6CEDF91CF9179
:109CE0001F91FF90EF90DF90CF90BF90AF909F902B
:109CF0008F907F906F905F904F903F902F9008953E
:109D0000CF93DF931F921F92CDB7DEB7BE016F5F77
:109D10007F4F88EF9FE00F94175689819A81815673
:109D2000904F803A9F4020F11A821982E8EEF9E0C4
:109D30008491882341F09091C00095FFFCCF8093DF
:109D4000C6003196F5CF8091C00085FFFCCF8AE038
:109D50008093C600BE016F5F7F4F88EF9FE00F9436
:109D600006568BEA99E00F94E55B81E00F94DD598C
:109D70000F900F90DF91CF9108952F923F924F92C5
:109D80005F926F927F928F929F92AF92BF92CF928B
:109D9000DF92EF92FF920F931F93CF93DF93CDB794
:109DA000DEB7CA58D2400FB6F894DEBF0FBECDBFA3
:109DB000C958DD4F688379838A839B83C757D24014
:109DC000FE01E75FFD4F88E2DF011D928A95E9F70A
:109DD000E850F24080E991E0DF019C011D922150A2
:109DE0003040E1F7C75ADD4F19821882C955D24079
:109DF000CE01875A9D4F5C014E019FE6891A9EEF66
:109E0000990ADE01AF51BE4F3D0190EBC92E9FE094
:109E1000D92E23E2E22EF12C00E010E0C359DD4FF1
:109E20008882CD56D240CD58DD4F9882C357D2405C
:109E3000B701882777FD8095982F0F9444B0D30100
:109E40006D937D938D939D933D01F501619171918A
:109E50005F01882777FD8095982F0F9444B0D40137
:109E60006D937D938D939D934D010F5F1F4F063032
:109E7000110559F0B501C6010F941756B5E0EB0E68
:109E8000F11CE2E0CE0ED11CD3CFCF51DE4F2881A2
:109E900039814A815B81C15ED140C958DD4F6881FB
:109EA00079818A819B81C757D2400F94A2AF87FDE9
:109EB0002BC3FE01EF51FE4F7F016E01FFE2CF1A6F
:109EC000FEEFDF0A3E012BEB621A2DEF720AC35937
:109ED000DD4F0881CD56D240CD58DD4F1881C35794
:109EE000D24085E090E0CF58DD4F99838883C157F9
:109EF000D240CF58DD4FA881B981C157D2401197C8
:109F0000CF58DD4FB983A883C157D240F7012089CC
:109F100031894289538964897589868997890F9423
:109F2000B1AE4B015C01D80150962D913D914D9100
:109F30005C91539754966D917D918D919C9157971B
:109F40000F94B1AEA50194010F94A9AFF6019293BD
:109F50008293729362936F01D301BE92AE929E92EE
:109F60008E923D0104501109B4E0EB1AF108CF586C
:109F7000DD4FE881F981C157D240EF2B09F0B9CF0D
:109F80006E01FFECCF1AFDEFDF0A3E0127E4621AF3
:109F90002EEF720A2E013DE3430E511CCE010196B5
:109FA0007C0101E010E0D6018D909D90AD90BC90B9
:109FB000139714962D913D914D915C911797C50182
:109FC000B4010F94B2AE9B01AC010F94B2AEF70195
:109FD00064A775A786A797A70130110541F080A651
:109FE00091A6A2A6B3A684829582A682B7820F5FAD
:109FF0001F4FD30114962D913D914D915C91179770
:10A0000018966D917D918D919C911B970F94B1AE97
:10A0100020E030E040EC50E40F94A3B2F201608302
:10A02000718382839383F4E0CF0ED11C2CE2E20E85
:10A03000F11C34E0630E711C88E2480E511C05309F
:10A04000110509F0B0CF8E010B5A1F4F6E0191E53B
:10A05000C90ED11C22242394312C2C0E3D1EA8EDB8
:10A060002A0E311CF801B897208131814281538139
:10A07000F80160817181828193810F94A9AF4B01B6
:10A080005C01E12CF12C3601F8E26F1A710826010F
:10A090004E0C5F1CF301EE0DFF1D248135814681BE
:10A0A0005781C501B4010F94A3B29B01AC01D20149
:10A0B00014966D917D918D919C9117970F94B1AEEF
:10A0C000F2016483758386839783F4E0EF0EF11CBD
:10A0D00024E1E216F104D9F6045D1F4F38E2C30E05
:10A0E000D11C0215130509F0BDCF1E0185EB280E0A
:10A0F000311C6E0191EBC90ED11C3E01A7EE6A1A0C
:10A10000ADEF7A0A14E0E12EF12C270100E010E017
:10A11000812C912CA12CB12CF601E00FF11FD30161
:10A12000A00FB11F2D913D914D915C916081718186
:10A13000828193810F94A3B29B01AC01B401C5014C
:10A140000F94B2AE4B015C01BFEF4B1A5B0A0C5F80
:10A150001F4FE5E04E165104F9F69B01AC01D10109
:10A160006D917D918D919C910F94B1AEF6012081FE
:10A170003181428153810F94A9AFD3016D937D93B7
:10A180008D939C931397B1E0EB1AF108E8E22E1A35
:10A190003108FCE2CF1AD10824E0621A7108E114F8
:10A1A000F10409F0B2CFCB50DE4F88819981AA81AA
:10A1B000BB81C55FD140C957DD4F88839983AA838E
:10A1C000BB83C758D2408E01075F1D4FDE01AF5CD5
:10A1D000BD4FC558DD4FB983A883CB57D240C35973
:10A1E000DD4F2880CD56D240CD58DD4F3880C35743
:10A1F000D240FE01EF51FE4FC358DD4FF983E88393
:10A20000CD57D240C358DD4FA881B981CD57D24038
:10A21000CD90DD90ED90FD90C358DD4FB983A883BC
:10A22000CD57D240C958DD4F288139814A815B81A1
:10A23000C757D240C701B6010F94A2AF1816B4F0A9
:10A24000C358DD4FE881F981CD57D240208131815B
:10A2500042815381C958DD4F688179818A819B8110
:10A26000C757D2400F94A2AF1816FCF4CF58DD4F59
:10A2700028813981C157D2402430310509F01FC1EE
:10A28000C957DD4F288139814A815B81C758D24047
:10A29000C958DD4F688179818A819B81C757D24037
:10A2A0000F94D1B118160CF00AC1D80114968D91F3
:10A2B0009D910D90BC91A02DC158DD4F888399834D
:10A2C000AA83BB83CF57D240F8014080518062807F
:10A2D0007380C558DD4FA881B981CB57D2408D918D
:10A2E0009D910D90BC91A02DC359DD4F888399831A
:10A2F000AA83BB83CD56D240D1018D919D910D9003
:10A30000BC91A02DCD57DD4F88839983AA83BB8351
:10A31000C358D240A7019601C958DD4F68817981A1
:10A320008A819B81C757D2400F94B1AECD58DD4F83
:10A33000688379838A839B83C357D24020E030E0CF
:10A3400040E450E40F9406B36B017C01A301920139
:10A35000C158DD4F688179818A819B81CF57D24076
:10A360000F94B1AE4B015C0120E030E040EC50E4D2
:10A37000C359DD4F688179818A819B81CD56D24056
:10A380000F94A3B29B01AC01C501B4010F94A9AF16
:10A39000A70196010F94A3B26B017C0120E030E08D
:10A3A00040E05FE3C301B2010F94A3B24B015C0133
:10A3B000CD58DD4F288139814A815B81C357D24016
:10A3C000CA01B9010F94A3B29B01AC01C501B4014C
:10A3D0000F94A3B29B01AC01C701B6010F94B2AEBA
:10A3E0006B017C01CD57DD4F288139814A815B812A
:10A3F000C358D240F10164817581868197810F94A1
:10A40000B1AEC359DD4F288139814A815B81CD5678
:10A41000D2400F94A9AF4B015C01C359DD4F288195
:10A4200039814A815B81CD56D240CA01B9010F946E
:10A43000B2AEA30192010F94A3B22B013C01C35908
:10A44000DD4F288139814A815B81CD56D240C15888
:10A45000DD4F688179818A819B81CF57D2400F94EB
:10A46000A3B29B01AC01C301B2010F94B2AE20E0D4
:10A4700030E040EC50E40F94A9AF9B01AC01C50162
:10A48000B4010F94B1AECD58DD4F288139814A8196
:10A490005B81C357D2400F94A3B29B01AC01C701AB
:10A4A000B6010F94B2AECD57DD4F288139814A8174
:10A4B0005B81C358D2400F94B2AE4B015C01CF58C0
:10A4C000DD4F28813981C157D2402F5F3F4FCF5890
:10A4D000DD4F39832883C157D2400C5F1F4FC558C9
:10A4E000DD4F88819981CB57D2400496C558DD4F06
:10A4F00099838883CB57D24094E0290E311C2530B4
:10A50000310509F07FCE04C0812C912CA12CB12CF7
:10A51000B401C501C657DD4F0FB6F894DEBF0FBEBC
:10A52000CDBFDF91CF911F910F91FF90EF90DF9002
:10A53000CF90BF90AF909F908F907F906F905F90E3
:10A540004F903F902F9008958091BF0B8823C9F0C2
:10A5500086EA9FE00F9430BB882399F06091D41A6B
:10A560007091D51A8091D61A9091D71A06DC209155
:10A57000B5193091B6194091B7195091B8190D9489
:10A58000A9AF60E070E0CB0108954F925F926F92A7
:10A590007F928F929F92AF92BF92CF92DF92EF9273
:10A5A000FF920F931F93CF93DF93CDB7DEB728971A
:10A5B0000FB6F894DEBF0FBECDBF0F941427809165
:10A5C0004702909148029093CB0B8093CA0BE09185
:10A5D000410BF0E0EE0FFF1FEE51F54E60817181EF
:10A5E000882777FD8095982F0F9444B06093B30B24
:10A5F0007093B40B8093B50B9093B60B80913F0B87
:10A600009091400B9093B20B8093B10B0F94BCA62A
:10A610006093990B70939A0B80939B0B90939C0B78
:10A620008091550B9091560BA091570BB091580B00
:10A6300089839A83AB83BC838093A10B9093A20BF5
:10A64000A093A30BB093A40B4090590B50905A0BBE
:10A6500060905B0B70905C0B4092A50B5092A60B28
:10A660006092A70B7092A80B80915D0B90915E0B8E
:10A67000A0915F0BB091600B8D839E83AF83B887F1
:10A680008093A90B9093AA0BA093AB0BB093AC0B48
:10A690006091610B7091620B8091630B9091640BE0
:10A6A0006093AD0B7093AE0B8093AF0B9093B00B98
:10A6B00020E030E040E85FE30F94B1AE6093610BBF
:10A6C0007093620B8093630B9093640B81E49BE027
:10A6D0009F938F93812C912CB8ECAB2EB3E4BB2EBF
:10A6E00011E6C12E1BE0D12EED80FE800F81188572
:10A6F000A301920169817A818B819C810F94A00DC5
:10A7000020E030E040EA51E460915D0B70915E0B17
:10A7100080915F0B9091600B0F94B2AE2B013C01C6
:10A720000F900F9020E030E042E553E40F94D1B158
:10A7300018164CF040925D0B50925E0B60925F0BCE
:10A740007092600B0CC080E090E0A2E5B3E48093CF
:10A750005D0B90935E0BA0935F0BB093600BE0904A
:10A760005D0BF0905E0B00915F0B1091600B2091E0
:10A77000590B30915A0B40915B0B50915C0B6091DF
:10A78000550B7091560B8091570B9091580BA1E48B
:10A790006A2EABE07A2E7F926F92812C912CB0E7DB
:10A7A000AB2EB1E4BB2EE1E6CE2EEBE0DE2E0F9415
:10A7B000A00D1092E31A1092E21A1092E51A10926C
:10A7C000E41A1092E71A1092E61A80E090E0A8E4EA
:10A7D000B2E48093550B9093560BA093570BB09314
:10A7E000580B80E090E0AEE3B3E48093590B909374
:10A7F0005A0BA0935B0BB0935C0BE0905D0BF09059
:10A800005E0B00915F0B1091600B7F926F92812C19
:10A81000912CF8E4AF2EF2E4BF2E9C01AD01C501EE
:10A82000B4010F94A00D1092400B10923F0B0F90AB
:10A830000F900F900F9028960FB6F894DEBF0FBEC2
:10A84000CDBFDF91CF911F910F91FF90EF90DF90DF
:10A85000CF90BF90AF909F908F907F906F905F90C0
:10A860004F900D941427E091410B84E0E89FF00194
:10A870001124E652F54E4081518162817381E8EAEC
:10A88000F9E08491882341F09091C00095FFFCCFBE
:10A890008093C6003196F5CF22E030E08EE09AE05A
:10A8A0000E949635E4EAF9E08491882341F0909182
:10A8B000C00095FFFCCF8093C6003196F5CF609124
:10A8C000410B70E04AE050E08EE09AE00E949E3436
:10A8D000E0EAF9E08491882341F09091C00095FF6F
:10A8E000FCCF8093C6003196F5CF4091C81A5091A5
:10A8F000C91A6091CA1A7091CB1A21E030E08EE03B
:10A900009AE00E9496358091C00085FFFCCF8AE0D6
:10A910008093C6000895CF93DF9300D000D0CDB7C9
:10A92000DEB7179A1092460B169A1092470BEBE976
:10A93000F9E08491882341F09091C00095FFFCCF0D
:10A940008093C6003196F5CF8091C00085FFFCCF83
:10A950008AE08093C60083E40F94C2463C012090B5
:10A960008B1030908C1040908D1050908E100F9462
:10A970007B1C281A390A410851080E949EB9281ADE
:10A98000390A4108510857FE03C0212C312C2101FE
:10A990009091D1138091D013981799F0E091D01332
:10A9A00027E5E29FF0011124EE52FC4E20E030E05A
:10A9B00040E752E462A173A184A195A10F94A3B2D0
:10A9C00008C060910C0270910D0280910E0290916E
:10A9D0000F020F9411B07E836D830F94250C0E949B
:10A9E00048B21092D60B789420E030E040E85FE364
:10A9F0006091610B7091620B8091630B9091640B7D
:10AA00000F94B1AE69837A838B839C83E0905D0B56
:10AA1000F0905E0B00915F0B1091600B2091590B31
:10AA200030915A0B40915B0B50915C0B6091550B30
:10AA30007091560B8091570B9091580BA1E4BBE09D
:10AA4000BF93AF93812C912CE8ECAE2EE3E4BE2EA5
:10AA5000DE0111966D010F94A00D20E030E040E87A
:10AA60005FE36091610B7091620B8091630B909139
:10AA7000640B0F94B1AE69837A838B839C832FE838
:10AA800032EC45EF5FE360915D0B70915E0B80915E
:10AA90005F0B9091600B0F94B2AE6B017C0167E08D
:10AAA00074E066197709F4E076956795FA95E1F711
:10AAB00080E090E00F9442B02091B5193091B61922
:10AAC0004091B7195091B8190F94A9AF9B01AC01EF
:10AAD000C701B6010F94B2AE7B018C012091590BD6
:10AAE00030915A0B40915B0B50915C0B6091550B70
:10AAF0007091560B8091570B9091580BA1E4BBE0DD
:10AB0000BF93AF93812C912CA0E2AA2EA2E4BA2E7F
:10AB1000DE0111966D010F94A00DB201A10181E932
:10AB20009FE00F9454BB0F900F900F900F9005E78C
:10AB30001FE0F12CB3E0EB2E8091E612882341F167
:10AB40008F2D6E2D0F9460B4B5E18B02F0011124AE
:10AB500023E09202E00DF11D1124EE0FFF1FEE0F16
:10AB6000FF1FEA51FD4E20E030E04AE754E46181E6
:10AB70007281838194810F94A3B220E030E040E0A1
:10AB80005FE30F94B2AE0F947FB00F9411B002C088
:10AB900060E070E0C8010F945CBBF3940E5F1F4F40
:10ABA00089E0F812C9CFB30183E79FE00F945CBB43
:10ABB0004091550B5091560B6091570B7091580B6B
:10ABC0008DE99FE00F9454BB4091590B50915A0B63
:10ABD00060915B0B70915C0B81EA9FE00F9454BB1A
:10ABE00040915D0B50915E0B60915F0B7091600B1B
:10ABF0008DE89FE00F9454BBBE016B5F7F4F89E8E7
:10AC00009FE00F940656E091410BF0E0EE0FFF1F1E
:10AC1000EE51F54E60818CE89FE00F9442BB60914D
:10AC2000E01A8BE89FE00F9442BB60913F0B88E8ED
:10AC30009FE00F9442BB61E085EA9FE00F9442BB26
:10AC40000F941427E6E9F9E08491882341F090916C
:10AC5000C00095FFFCCF8093C6003196F5CF83E40A
:10AC60000F94C2464AE050E0BC018EE09AE00E9498
:10AC7000F53484E69FE00F9430BB61E0680F84E612
:10AC80009FE00F9442BBEBE8F9E08491882341F008
:10AC90009091C00095FFFCCF8093C6003196F5CF10
:10ACA0008091C00085FFFCCF8AE08093C600F894B5
:10ACB000FFCF6C987498EAE6F0E080818160808331
:10ACC00080818D7F8083EC9A08951F920F920FB63A
:10ACD0000F9211240BB60F922F933F934F935F93D4
:10ACE0006F937F938F939F93AF93BF93EF93FF9354
:10ACF000EC98E6E8F9E08491882341F09091C00057
:10AD000095FFFCCF8093C6003196F5CF8091C000AF
:10AD100085FFFCCF8AE08093C6008091D60B81111D
:10AD2000FADDFF91EF91BF91AF919F918F917F914C
:10AD30006F915F914F913F912F910F900BBE0F90AC
:10AD40000FBE0F901F901895BF92CF92DF92EF9297
:10AD5000FF920F931F93CF93DF93CDB7DEB7E197A9
:10AD60000FB6F894DEBF0FBECDBF88E89FE00F940A
:10AD700030BBB82EBE01605D7F4F89E89FE00F9425
:10AD80001756EFE2F8E08491882341F09091C000DB
:10AD900095FFFCCF8093C6003196F5CF68A979A9BD
:10ADA0004AE050E08EE09AE00E94A5348E01015EF8
:10ADB0001F4F85E9E82E8FE0F82ED02EC12EC70157
:10ADC0000F9430BBF80181938F01FFEFEF1AFF0A58
:10ADD0008DE9E8168FE0F80691F71FA2ED2DFC2D06
:10ADE0008191882339F09091C00095FFFCCF80932A
:10ADF000C600F6CF6AE278E08D2D9C2D0F94DFB768
:10AE0000CF92DF9283E298E09F938F938E010F5F42
:10AE10001F4F1F930F930F9404B90F900F900F9033
:10AE20000F900F900F907E0195E0E90EF11CF70155
:10AE30008081882349F0992787FD90950F94CEB79C
:10AE4000F70181937F01F3CF60E0C8010E94BEB299
:10AE500081E99FE00F9438BBF62EE72ED82EC92E3D
:10AE6000E8E0F8E08491882341F09091C00095FFDC
:10AE7000FCCF8093C6003196F5CF2AE030E04F2D0D
:10AE80005E2D6D2D7C2D8EE09AE00E94013561E0F3
:10AE900084E098E00E94BEB26FEF77E0C8010F94A3
:10AEA000EAB78DE99FE00F9438BB6CA77DA78EA70A
:10AEB0009FA7CE018C960F94665EBC01C8010F94CB
:10AEC00079B86CEF77E0C8010F94DFB781EA9FE0B3
:10AED0000F9438BB6CA77DA78EA79FA7CE018C9639
:10AEE0000F94665EBC01C8010F9479B865EF77E0F6
:10AEF000C8010F94DFB760E0C8010E94BEB260EFE6
:10AF000077E0C8010F94EAB78DE89FE00F9438BB53
:10AF10006CA77DA78EA79FA7CE018C960F94665E27
:10AF2000BC01C8010F9479B860E0C8010E94BEB2AC
:10AF300061E085EE97E00E94BEB289A98F9388A94F
:10AF40008F938EED97E09F938F931F930F930F94A2
:10AF500004B960E0C8010E94BEB267ED77E0C801A5
:10AF60000F94EAB78B2D90E09DA78CA7CE018C960D
:10AF70000F94C860BC01C8010F9479B860E0C801A3
:10AF80000E94BEB2CF92DF92EF92FF928EEC97E0DA
:10AF90009F938F931F930F930F9404B960E0C801A0
:10AFA0000E94BEB261E08AEC97E00E94BEB20FB68A
:10AFB000F894DEBF0FBECDBFE1960FB6F894DEBFAA
:10AFC0000FBECDBFDF91CF911F910F91FF90EF90FA
:10AFD000DF90CF90BF9008954F925F926F927F92D3
:10AFE000AF92BF92CF92DF92EF92FF920F931F9397
:10AFF000CF93DF93CDB7DEB7E0970FB6F894DEBFFF
:10B000000FBECDBF2B013C0169017A018091B00ACE
:10B010008111E5C0F8940F945B1C80918B10909186
:10B020008C10A0918D10B0918E108093AC0A9093EB
:10B03000AD0AA093AE0AB093AF0A0F947B1C409167
:10B04000AC0A5091AD0A6091AE0A7091AF0A481BEC
:10B05000590B610971094093AC0A5093AD0A609392
:10B06000AE0A7093AF0A0E949EB94091AC0A50910B
:10B07000AD0A6091AE0A7091AF0A481B590B610985
:10B0800071094093AC0A5093AD0A6093AE0A709375
:10B09000AF0A9091D1138091D013981799F0E09155
:10B0A000D01387E5E89FF0011124EE52FC4E20E01A
:10B0B00030E040E752E462A173A184A195A10F940E
:10B0C000A3B208C060910C0270910D0280910E0233
:10B0D00090910F026093980A7093990A80939A0A4C
:10B0E00090939B0A0F94250C80E1E5E5FBE0ACE929
:10B0F000BAE001900D928A95E1F78091410B80931F
:10B10000970A809107028093960A0E9448B2109293
:10B11000D60B81E08093B00A789420E030E0A9015A
:10B12000C301B2010F94A2AF81110AC020E030E048
:10B13000A901C701B6010F94A2AF882309F44FC03B
:10B1400065EC77E0FE0131965F01CF010F94EAB71D
:10B15000F50101900020E9F78F01015011092091BC
:10B16000A40A3091A50A4091A60A5091A70AC301EA
:10B17000B2010F94B2AE23E048E00F940DB562EC3B
:10B1800077E0C5010F94DFB7F50101900020E9F7E2
:10B190008F010150110923E046E0C701B6010F9469
:10B1A0000DB56FEB77E0C5010F94DFB7F5010190A6
:10B1B0000020E9F78F01015011096091510270914F
:10B1C0005202809153029091540223E048E00F9480
:10B1D0000DB560E0C5010E94BEB20E9454B4E09675
:10B1E0000FB6F894DEBF0FBECDBFDF91CF911F9198
:10B1F0000F91FF90EF90DF90CF90BF90AF907F9036
:10B200006F905F904F90089520E030E0A90160E0DA
:10B2100070E080E291E4E0CE8F929F92AF92BF9275
:10B22000CF92DF92EF92FF920F931F93CF93DF9312
:10B2300000D01F92CDB7DEB79B01AC018091B00A60
:10B24000882309F497C08091970A8093410B8091DD
:10B25000980A9091990AA0919A0AB0919B0A8093BA
:10B260000C0290930D02A0930E02B0930F02609116
:10B27000A80A7091A90A8091AA0A9091AB0A0F942A
:10B28000B1AE69837A838B839C83CE0101960F9440
:10B29000ED1B20E030E040E551E4609151027091F7
:10B2A000520280915302909154020F94A9AF4B0126
:10B2B0005C01E090A40AF090A50A0091A60A109102
:10B2C000A70A2091A00A3091A10A4091A20A5091A8
:10B2D000A30A60919C0A70919D0A80919E0A9091A8
:10B2E0009F0AE1E4FBE0FF93EF93E8EACE2EEAE069
:10B2F000DE2E0F94A00D0F94142780E1ECE9FAE004
:10B30000A5E5BBE001900D928A95E1F780E1E5E5C6
:10B31000FBE0A0E2BBE001900D928A95E1F740913D
:10B32000AC0A5091AD0A6091AE0A7091AF0A409399
:10B33000720E5093730E6093740E7093750E8DEBB6
:10B340009DE00E94329A8091AC0A9091AD0AA09142
:10B35000AE0AB091AF0A80938B1090938C10A0939B
:10B360008D10B0938E1081E08093D60B1092B00AAE
:10B370000F900F900F900F900F900F90DF91CF9143
:10B380001F910F91FF90EF90DF90CF90BF90AF9003
:10B390009F908F90089560E070E0CB013DCFEAEA86
:10B3A000F7E08491882341F09091C00095FFFCCF95
:10B3B0008093C6003196F5CF4091550B5091560BB6
:10B3C0006091570B7091580B23E030E08EE09AE0CB
:10B3D0000E949635E7EAF7E08491882341F0909146
:10B3E000C00095FFFCCF8093C6003196F5CF409109
:10B3F000590B50915A0B60915B0B70915C0B23E0E1
:10B4000030E08EE09AE00E949635E4EAF7E084911D
:10B41000882341F09091C00095FFFCCF8093C60037
:10B420003196F5CF40915D0B50915E0B60915F0BB3
:10B430007091600B23E030E08EE09AE00E94963538
:10B44000E2EAF7E08491882341F09091C00095FFF3
:10B45000FCCF8093C6003196F5CF8091C00085FF68
:10B46000FCCF8AE08093C6000895EAE8F7E0849173
:10B47000882341F09091C00095FFFCCF8093C600D7
:10B480003196F5CF0F948327AB01BC0123E030E068
:10B490008EE09AE00E949635E7E8F7E084918823F1
:10B4A00041F09091C00095FFFCCF8093C60031968B
:10B4B000F5CF81E00F948327AB01BC0123E030E09E
:10B4C0008EE09AE00E949635E4E8F7E084918823C4
:10B4D00041F09091C00095FFFCCF8093C60031965B
:10B4E000F5CF82E00F948327AB01BC0123E030E06D
:10B4F0008EE09AE00E949635E2E8F7E08491882396
:10B5000041F09091C00095FFFCCF8093C60031962A
:10B51000F5CF8091C00085FFFCCF8AE08093C60004
:10B520000895EF92FF920F931F93CF93DF93EEE670
:10B53000F7E08491882341F09091C00095FFFCCF03
:10B540008093C6003196F5CF06EE12E1FCE6EF2EB1
:10B55000F7E0FF2EC0E0D0E0F801EC0FFD1F4181C5
:10B5600052816381748123E030E08EE09AE00E9492
:10B570009635F7018491ECE6F7E0882349F0909145
:10B58000C00095FFFCCF8093C60031968491F5CF23
:10B590002496CC31D10501F7045E1F4FF3E10A3A3E
:10B5A0001F07C1F6EBE6F7E08491882341F0909104
:10B5B000C00095FFFCCF8093C6003196F5CF8091F7
:10B5C000C00085FFFCCF8AE08093C600DF91CF9159
:10B5D0001F910F91FF90EF9008952F923F924F92FD
:10B5E0005F926F927F928F929F92AF92BF92CF9213
:10B5F000DF92EF92FF920F931F93CF93DF93CDB71C
:10B60000DEB7C955D1090FB6F894DEBF0FBECDBF66
:10B6100084E294E00E945D368823B1F08091A3100B
:10B620009091A4106AE270E005960F9484B8009798
:10B6300011F0DC011C928091A3109091A41005964A
:10B640000F94E4560C94898A89E294E00E945D3656
:10B65000882309F481C18FE294E00E945D3688233B
:10B6600091F08091ED1B882311F40C94898A0F943A
:10B67000BCA66093D00B7093D10B8093D20B9093A8
:10B68000D30B0C94898A84E394E00E945D3688236E
:10B6900061F060918F0B7091900B4AE050E08EE06A
:10B6A0009AE00E94F5340C94898A88E394E00E9421
:10B6B0005D368823C1F08091ED1B882361F0609195
:10B6C000EB1B7091EC1B4AE050E08EE09AE00E9488
:10B6D000A5340C94898A6BE374E08EE09AE00E94B2
:10B6E00091340C94898A8DE494E00E945D3688231D
:10B6F00079F16091A3107091A4106D5F7F4F21E0EC
:10B7000041E084ED9BE00E9480AC8091C50D90915A
:10B71000C60DA091C70DB091C80D8093720E909385
:10B72000730EA093740EB093750E8DEB9DE00E9486
:10B7300069992091C00025FFFCCF8093C6000A972D
:10B7400021F760E084ED9BE00E9410AC0C94898AA4
:10B7500080E594E00E945D36882399F00E94F742CC
:10B7600081E08093910B6091A3107091A4106C5FA5
:10B770007F4F21E040E084ED9BE00E9480AC0C9480
:10B78000898A84E594E00E945D36882309F44FC0DD
:10B790008091ED1B882309F49ECF1092940A109299
:10B7A000930AE7E5F4E08191882339F09091C00095
:10B7B00095FFFCCF8093C600F6CF00E010E0EE24AA
:10B7C000E394F12C80918F0A9091900A2091910A34
:10B7D0003091920A821B930B8F779927892BA9F0BE
:10B7E0008EE09AE00E94AB33F092940AE092930AC2
:10B7F0009091C00095FFFCCF8093C6000F5F1F4F54
:10B800001092940A1092930ADDCF03311105D4F2FD
:10B8100081E090E09093940A8093930A8091C00015
:10B8200085FFFCCF8AE08093C6000C94898A8AE564
:10B8300094E00E945D368823A9F0EEE5F4E0819162
:10B84000882339F09091C00095FFFCCF8093C6000B
:10B85000F6CF8091C00085FFFCCF8AE08093C600C0
:10B860000C94898A89E694E00E945D368823A9F0C9
:10B87000EDE6F4E08191882339F09091C00095FFC6
:10B88000FCCF8093C600F6CF8091C00085FFFCCF2F
:10B890008AE08093C6000C94898A8BE894E00E9429
:10B8A0005D36882321F00F9482560C94898A80E9B2
:10B8B00094E00E945D36882341F060E070E088EFFC
:10B8C0009FE00F9406560C94898A83E994E00E94C5
:10B8D0005D36882359F063E974E08EE09AE00E94B7
:10B8E000913440E052EC61E070E010C08EE994E0E9
:10B8F0000E945D36882381F06EE974E08EE09AE064
:10B900000E94913440E054E961E170E08EE09AE0F9
:10B910000E9435330C94FE8B8AEA94E00E945D36D7
:10B92000882361F00F94BCA66093BB0B7093BC0B93
:10B930008093BD0B9093BE0B0C94898A8FEA94E0A0
:10B940000E945D36882311F40C94898A61E080E0BE
:10B950000E94D63A0C94898A8EE50E94473681115E
:10B960000C94898A87E40E944736882311F40C944A
:10B97000126E0E94A7360F9411B06C34710509F451
:10B9800034C47CF56430710509F409C154F46230A3
:10B99000710509F4ECC00CF0F6C077FF78C00C9488
:10B9A000898A6C31710509F451C17CF46A307105E2
:10B9B00009F446C16B30710511F00C94898A60E07E
:10B9C00080E00E94DD470C94898A6E31710509F48C
:10B9D00051C36B34710511F00C94898A08E210E0B0
:10B9E000FAC36735710511F40C94926D14F5603546
:10B9F000710511F40C94C9656CF46F34710511F084
:10BA00000C94898A0FEF10E0A1E9CA2EADE0DA2E7E
:10BA10000C94B8656135710511F40C94D96C6635D8
:10BA2000710511F00C94898A86EE0E948D3A0C946F
:10BA3000898A6C35710511F40C949B6D7CF46A3520
:10BA4000710511F40C94976D6B35710511F00C9420
:10BA5000898A81E080930B0B0C94898A6236710588
:10BA600011F40C94FD6D6336710511F00C94898A04
:10BA70001092ED1B0F9487566091ED1B84EC9FE0B4
:10BA80000F9442BB82E00F9470580C94898A809185
:10BA9000F50A81110C94898A0E94124460918B0BE3
:10BAA00070918C0B80918D0B90918E0B0F9442B006
:10BAB0004B015C01C090610BD090620BE090630B76
:10BAC000F090640B40902C0B50902D0B60902E0B3F
:10BAD00070902F0BA3019201C701B6010F94B1AE74
:10BAE00020E030E048EC52E40F94A3B29B01AC019B
:10BAF000C501B4010F94D1B11816E4F4A701960161
:10BB0000C301B2010F94B1AE20E030E048EC52E442
:10BB10000F94A3B29B01AC01C501B4010F94B2AE66
:10BB20000F9416B060938B0B70938C0B80938D0BDE
:10BB300090938E0B80913E0B8823A9F088E50E949C
:10BB40004736811110C089E50E94473681110BC02C
:10BB50008AE50E944736811106C085E40E94473677
:10BB600081110C948C8A0E94DA460C94898A809107
:10BB7000F50A81110C94898A0E94954481E00E9403
:10BB8000B8490C94898A8091F50A81110C94898AAC
:10BB90000E94954480E00E94B8490C94898A80E50F
:10BBA0000E944736882339F00E94A7360F9416B0BA
:10BBB0004B015C0103C0812C912C540183E50E9450
:10BBC0004736882361F00E94A73620E030E04AE73C
:10BBD00054E40F94A3B20F9416B04B015C0181148E
:10BBE0009104A104B10431F0EDEEF7E28591949156
:10BBF0000F94F1560F9414270F94BCA62B013C010F
:10BC0000480C591C6A1C7B1C0F94BCA66093070B44
:10BC10007093080B8093090B90930A0B0F94BCA6AA
:10BC2000641575058605970510F00C94898A0F94A4
:10BC3000AA3880E00E94DF4A80E00F947058EECF6F
:10BC400060E081E00E94DD470C94898A0F941427FC
:10BC5000EFEBFEE08491882341F09091C00095FFC6
:10BC6000FCCF8093C6003196F5CF99DBE1EBFEE087
:10BC70008491882341F09091C00095FFFCCF809380
:10BC8000C6003196F5CFF1DB81E08093C00B88E5EB
:10BC90000E944736182F89E50E944736082F8AE50B
:10BCA0000E944736782E101308C0181305C0772459
:10BCB000739401E011E001C0012F0E94BED8609092
:10BCC000E6121092E61282E00F94832760935D0BD8
:10BCD00070935E0B80935F0B9093600B71100F94C9
:10BCE000A00140910C0250910D0260910E027091E2
:10BCF0000F0240930C0B50930D0B60930E0B70933F
:10BD00000F0B80914702909148029093CB0B809348
:10BD1000CA0B84E690E090934802809347020F9408
:10BD2000BCA66093070B7093080B8093090B90934C
:10BD30000A0B81E00F94C31D80E1E5E5FBE0A0E282
:10BD4000BBE001900D928A95E1F710920C021092DF
:10BD50000D0210920E0210920F02112321F080E0CA
:10BD600090E00E94973E002321F081E090E00E9445
:10BD7000973E88E50E944736882341F00E9471363D
:10BD8000672B682B692B11F00C94BB8A89E50E9404
:10BD90004736882341F00E947136672B682B692B48
:10BDA00011F00C94D18A772009F4F1C08091460BF0
:10BDB000882321F08091470B811108C080E090E03A
:10BDC0000E94973E81E090E00E94973E0E9413D926
:10BDD000E6E4F3E385919591A591B49189839A83E3
:10BDE000AB83BC83E2E4F3E385919591A591B49193
:10BDF0008F8F98A3A9A3BAA324E23BE040E25BE0C3
:10BE0000BE016F5F7F4FCE014F960E94AE380E94F9
:10BE100085D820E030E040E451EC6091240B709133
:10BE2000250B8091260B9091270B0F94A2AF87FFD3
:10BE30000CC080E090E0A0E4B1EC8093240B9093E0
:10BE4000250BA093260BB093270B80E090E0A0EA8F
:10BE5000B0E48093280B9093290BA0932A0BB09306
:10BE60002B0B20E030E040E251E4609151027091F0
:10BE7000520280915302909154020F94A9AF6093A3
:10BE80000C0270930D0280930E0290930F02109299
:10BE90005D0B10925E0B10925F0B1092600B80E0B6
:10BEA0000F94C31DE0905D0BF0905E0B00915F0B53
:10BEB0001091600B2091590B30915A0B40915B0B04
:10BEC00050915C0B6091550B7091560B8091570B04
:10BED0009091580BF1E6CF2EFBE0DF2E0F944E1A17
:10BEE00080900C0290900D02A0900E02B0900F0274
:10BEF000E090280BF090290B00912A0B10912B0B4E
:10BF00002091240B3091250B4091260B5091270B4B
:10BF10006091200B7091210B8091220B9091230B4B
:10BF2000E1E4FBE0FF93EF93ACE2CA2EABE0DA2E44
:10BF30000F94A00D0F9414278091200B9091210B4A
:10BF4000A091220BB091230B8093550B9093560B2D
:10BF5000A093570BB093580B8091240B9091250B15
:10BF6000A091260BB091270B8093590B90935A0BFD
:10BF7000A0935B0BB0935C0B81E00F94C31D0F94F7
:10BF8000AB1D82E090E00E94973E0F900F908AE5F3
:10BF90000E944736882341F00E947136672B682B38
:10BFA000692B11F00C94E78AE0905D0BF0905E0B2A
:10BFB00000915F0B1091600B2091590B30915A0B3F
:10BFC00040915B0B50915C0B6091550B7091560B3F
:10BFD0008091570B9091580BE1E6CE2EEBE0DE2ED0
:10BFE0000F944E1A80E00F94C31D80910C0B90911A
:10BFF0000D0BA0910E0BB0910F0B80930C02909340
:10C000000D02A0930E02B0930F028091CA0B909183
:10C01000CB0B90934802809347020F94BCA6609389
:10C02000070B7093080B8093090B90930A0B0F94E6
:10C03000AB1D0E9413D90E942FDB88E50E94473672
:10C0400081110C94FD8A89E50E94473681110C9478
:10C05000FD8A87E50E94473681110C94FD8A8AE5A6
:10C060000E94473681110C94FD8A0F941427109278
:10C07000C00B8FC50F94142781E00E94F335809187
:10C08000510290915202A0915302B09154028093B8
:10C090000C0290930D02A0930E02B0930F0220E0C9
:10C0A00030E043E060E070E080E291EC0E94BEDBB3
:10C0B000EBE3F8E285919491FC012491222341F075
:10C0C0003091C00035FFFCCF2093C6000196F4CF1D
:10C0D000E8E8FEE08491882341F09091C00095FF4C
:10C0E000FCCF8093C6003196F5CF4091550B50910F
:10C0F000560B6091570B7091580B25E030E08EE0A5
:10C100009AE00E949635E3E8FEE08491882341F0AE
:10C110009091C00095FFFCCF8093C6003196F5CF7B
:10C120004091590B50915A0B60915B0B70915C0BD5
:10C1300025E030E08EE09AE00E949635EEE7FEE0E2
:10C140008491882341F09091C00095FFFCCF8093AB
:10C15000C6003196F5CF40915D0B50915E0B60911A
:10C160005F0B7091600B25E030E08EE09AE00E945A
:10C170009635ECE7FEE08491882341F09091C00071
:10C1800095FFFCCF8093C6003196F5CF0E942136F3
:10C190000C94898A9091C00095FFFCCF8093C600D3
:10C1A00081918111F7CFB801882777FD8095982F6D
:10C1B0000F9444B00E94BD4EAB01BC0122E030E0C0
:10C1C0008EE09AE00E9497350F5F1F4F0F361105E2
:10C1D00011F40C94898A4AE050E0B8018EE09AE0AC
:10C1E0000E949E34E7E8F9E0DBCF8091460B88237C
:10C1F00041F08091470B882321F08091480B8111F9
:10C2000009C00E9454B461E085E79EE00E949CB39F
:10C210000C94898AE7E5FEE08491882341F09091AF
:10C22000C00095FFFCCF8093C6003196F5CF80917A
:10C23000C00085FFFCCF8AE08093C6001A82198275
:10C240008090D41A9090D51AA090D61AB090D71A90
:10C2500020E030E040EA50E4C501B4010F94A9AFFA
:10C260000F9411B045E0469F9001479F300D112477
:10C27000B901882777FD8095982F0F9444B02B0142
:10C280003C0120E030E04CE052E40F94A2AF87FF85
:10C2900006C0412C512C9CE0692E92E4792EA50118
:10C2A0009401C301B2010F94A2AF87FF0AC020E03E
:10C2B00030E040EA50E4C301B2010F94B2AE2B016A
:10C2C0003C01E3E4FEE08491882341F09091C000BA
:10C2D00095FFFCCF8093C6003196F5CF22E030E089
:10C2E000B301A2018EE09AE00E94973520E030E091
:10C2F00040EF51E4C301B2010F94B1AE20E030E051
:10C3000040E251E40F94A3B220E030E040EA50E470
:10C310000F94A9AF20E030E048E452E40F94B2AEAD
:10C320000F9411B07093E11A6093E01A84E090E0EA
:10C330009093840B8093830B81E090E09093820B29
:10C340008093810BE1EBF6E28591949121E0892BBA
:10C3500009F420E02093860B80E090E0ACE8B2E4A2
:10C360008093550B9093560BA093570BB093580B9B
:10C3700080E090E0A0E4B0EC8093590B90935A0BCE
:10C38000A0935B0BB0935C0B80E090E0A0E8BFE370
:10C3900080935D0B90935E0BA0935F0BB093600B4B
:10C3A00081E49BE09F938F93812C912C18E4A12E24
:10C3B00012E4B12E01E6C02E0BE0D02EE12CF12CC0
:10C3C00000E81FE320E030E040E450EC60E070E083
:10C3D0008CE892E40F94A00D0F9414270F900F9007
:10C3E000A30192016091D41A7091D51A8091D61A46
:10C3F0009091D71A0F94A2AF87FF07C088EE93E001
:10C400000E94004D0E943354EBCF60E086EA9FE02B
:10C410000F9442BB80E090E0A0EAB0E480935D0B13
:10C4200090935E0BA0935F0BB093600B2091590B20
:10C4300030915A0B40915B0B50915C0B6091550B06
:10C440007091560B8091570B9091580BE1E4FBE0F3
:10C45000FF93EF93812C912CE8E4AE2EE2E4BE2E04
:10C46000F1E6CF2EFBE0DF2EE12CF12C00EA10E408
:10C470000F94A00DE2E4F3E385919591A591B49119
:10C480008093550B9093560BA093570BB093580B7A
:10C49000E6E4F3E325913591459154912093590BAE
:10C4A00030935A0B40935B0B50935C0BE0905D0B09
:10C4B000F0905E0B00915F0B1091600B6091550B3B
:10C4C0007091560B8091570B9091580BE1E4FBE073
:10C4D000FF93EF93812C912CB8E4AB2EB2E4BB2EEA
:10C4E0000F94A00D0F94142720E030E043E060E0AB
:10C4F00070E080E89FEB0E94BEDB80915D0B909125
:10C500005E0BA0915F0BB091600B24968CAF9DAF3A
:10C51000AEAFBFAF2497E2E4FEE084910F900F909E
:10C520000F900F9040915D0B50915E0B60915F0BEF
:10C530007091600B882349F09091C00095FFFCCF6B
:10C540008093C60031968491F5CF8091C00085FF1D
:10C55000FCCF8AE08093C600EBE3FEE08491882361
:10C5600041F09091C00095FFFCCF8093C6003196BA
:10C57000F5CF22E030E08EE09AE00E949635EAE3C3
:10C58000FEE08491882341F09091C00095FFFCCF9C
:10C590008093C6003196F5CF8091C00085FFFCCF17
:10C5A0008AE08093C6002EEAA22E2FE0B22E33E25C
:10C5B000E32EF12C0FEF1FEF4AE0D42E53E0252E8F
:10C5C0005EE0352E62E0862E6EE0962EB70188275B
:10C5D00077FD8095982F0F9444B068AF79AF8AAFFC
:10C5E0009BAFE3E3FEE08491882341F09091C0008B
:10C5F00095FFFCCF8093C6003196F5CF4AE050E01E
:10C60000B8016E5F7F4F8EE09AE00E949E34E6E2B2
:10C61000FEE08491882341F09091C00095FFFCCF0B
:10C620008093C6003196F5CF8091C00085FFFCCF86
:10C63000D092C600E2E1FEE08491882341F090911F
:10C64000C00095FFFCCF8093C6003196F5CF4AE03D
:10C6500050E0B7018EE09AE00E949E34F10184918F
:10C66000E3E0FEE0882349F09091C00095FFFCCF05
:10C670008093C60031968491F5CF4AE050E060E0A7
:10C6800070E08EE09AE00E949E34F4018491E2E032
:10C69000FEE0882349F09091C00095FFFCCF809385
:10C6A000C60031968491F5CF8091C00085FFFCCF04
:10C6B000D092C6000F3FFFEF1F0731F0BE016F5F42
:10C6C0007F4FC5010F94065628AD39AD4AAD5BAD1D
:10C6D000C301B2010F94A2AF181664F40F5F1F4F8D
:10C6E00025E0E20EF11C32E0A30EB11C053011056D
:10C6F00009F06CCF280187E2481A88EF580A440CE9
:10C70000551C380193E0690E711C85E0809F100173
:10C71000819F300C112419AE18AEADE22A0E311CE7
:10C72000C301029705970CF0C7C168AD79AD620DE2
:10C73000731D882777FD8095982F0F9444B06CAFB8
:10C740007DAF8EAF9FAFEBEFFDE08491882341F08A
:10C750009091C00095FFFCCF8093C6003196F5CF35
:10C760004AE050E0B3018EE09AE00E949E34E8EF88
:10C77000FDE08491882341F09091C00095FFFCCFAB
:10C780008093C6003196F5CF8091C00085FFFCCF25
:10C79000FAE0F093C6007092820B6092810B20E069
:10C7A00030E040EF51E46CAD7DAD8EAD9FAD0F94A8
:10C7B000B1AE20E030E040E251E40F94A3B220E0BB
:10C7C00030E040EA50E40F94A9AF20E030E048E4C4
:10C7D00052E40F94B2AE0F9411B07093E11A6093CB
:10C7E000E01A80E090E0ACE8B2E48093550B9093BF
:10C7F000560BA093570BB093580B80E090E0A0E449
:10C80000B0EC8093590B90935A0BA0935B0BB093B1
:10C810005C0B80E090E0A0E8BFE380935D0B909319
:10C820005E0BA0935F0BB093600BA1E4BBE0BF93E2
:10C83000AF93812C912CA8E4AA2EA2E4BA2EB1E6E3
:10C84000CB2EBBE0DB2EE12CF12C00E81FE320E037
:10C8500030E040E450EC60E070E08CE892E40F944B
:10C86000A00D0F9414270F900F902CAD3DAD4EAD41
:10C870005FAD6091D41A7091D51A8091D61A9091BB
:10C88000D71A0F94A2AF87FF07C088EE93E00E94EB
:10C89000004D0E943354E9CF80E090E0A0EAB0E47C
:10C8A00080935D0B90935E0BA0935F0BB093600B36
:10C8B0002091590B30915A0B40915B0B50915C0BBE
:10C8C0006091550B7091560B8091570B9091580BBE
:10C8D000A1E4BBE0BF93AF93812C912CB8E4AB2EC5
:10C8E000B2E4BB2E11E6C12E1BE0D12EE12CF12CBF
:10C8F00000EA10E40F94A00DE2E4F3E38591959132
:10C90000A591B4918093550B9093560BA093570B20
:10C91000B093580BE6E4F3E325913591459154919A
:10C920002093590B30935A0B40935B0B50935C0B45
:10C93000E0905D0BF0905E0B00915F0B1091600B2F
:10C940006091550B7091560B8091570B9091580B3D
:10C95000A1E4BBE0BF93AF93812C912CF8E4AF2E00
:10C96000F2E4BF2E0F94A00D0F94142720E030E0C6
:10C9700043E060E070E080E89FEB0E94BEDB24961D
:10C980002CAD3DAD4EAD5FAD249760915D0B7091C8
:10C990005E0B80915F0B9091600B0F94B1AE209174
:10C9A000B5193091B6194091B7195091B8190F9433
:10C9B000A3B20F9411B07A836983E7EFFDE084910D
:10C9C0000F900F900F900F90882349F09091C00026
:10C9D00095FFFCCF8093C60031968491F5CF80916E
:10C9E000C00085FFFCCFFAE0F093C600E3EEFDE067
:10C9F0008491882341F09091C00095FFFCCF8093F3
:10CA0000C6003196F5CF4091D41A5091D51A609155
:10CA1000D61A7091D71A22E030E08EE09AE00E9498
:10CA20009635E4EDFDE08491882341F09091C000BB
:10CA300095FFFCCF8093C6003196F5CF24962CADA0
:10CA40003DAD4EAD5FAD249760915D0B70915E0B77
:10CA500080915F0B9091600B0F94B1AEAB01BC0164
:10CA600022E030E08EE09AE00E949635E3EDFDE0B2
:10CA70008491882341F09091C00095FFFCCF809372
:10CA8000C6003196F5CF8091C00085FFFCCFFAE05B
:10CA9000F093C600BE016F5F7F4FC2010F94065630
:10CAA00022E0420E511C3FEF631A730A88AD99AD24
:10CAB000059699AF88AF34CE1092840B1092830BF9
:10CAC0001092860B61E086EA9FE00F9442BBE4E996
:10CAD000FDE08491882341F09091C00095FFFCCF48
:10CAE0008093C6003196F5CF8091C00085FFFCCFC2
:10CAF0008AE08093C600179A1092460B169A1092FD
:10CB0000470B149AEFEAF6E2859194910F94E55B56
:10CB100081E00F94DD5982E00F9470581092E11A71
:10CB20001092E01A0C94898A84E690E00E94004DED
:10CB300091E0E91AF108C1F74AE050E0B8018EE04F
:10CB40009AE00E949E34F6012491E1E9FDE0211172
:10CB500017C06091680B7091690B4AE050E08EE05D
:10CB60009AE00E94A5340550110911F40C94898AA9
:10CB70001093400B00933F0BF4E6EF2EF12CD4CF33
:10CB80003091C00035FFFCCF2093C6003196249130
:10CB9000DECF81E08093940B86E50E9447368823A0
:10CBA000A1F08091A3109091A410DC0111962C911A
:10CBB000293069F02F7D71F04AE050E060E070E0CC
:10CBC00001960F9495B668AF07C018AE05C0B1E0E6
:10CBD000B8AF02C0E1E0E8AF2091460B8091F11BB5
:10CBE0009091F21B222341F02091470B222321F048
:10CBF0002091480B21110FC0029749F00E9454B4B4
:10CC000061E08AE89DE00E949CB30C94898A1092AE
:10CC1000940B0C94898A1092950A029721F4109231
:10CC2000940B0C94898AF091860B2E96FFAF2E9769
:10CC30002091830B3091840B60963FAF2EAF6097AD
:10CC40008091810B9091820B62969FAF8EAF62971D
:10CC500081E08093860B81E090E09093840B809339
:10CC6000830B83E190E09093820B8093810B81E0B2
:10CC70000F94705886EE92E10F946D020F94A0010C
:10CC800080E090E0A0EAB0E480935D0B90935E0BAF
:10CC9000A0935F0BB093600B20E030E040E752E4DC
:10CCA000609151027091520280915302909154020E
:10CCB0000F94A9AF4B015C012091590B30915A0B95
:10CCC00040915B0B50915C0B6091550B7091560B32
:10CCD0008091570B9091580BE1E4FBE0FF93EF93A9
:10CCE00011E6C12E1BE0D12EE12CF12C00EA10E45C
:10CCF0000F94A00DE2E4F3E385919591A591B49191
:10CD00008093550B9093560BA093570BB093580BF1
:10CD1000E6E4F3E385919591A591B4918093590B45
:10CD200090935A0BA0935B0BB0935C0B69E57BE08F
:10CD300085E59BE00E94683929968FAF29970F906F
:10CD40000F9098AD19160CF45FC020E030E040EF72
:10CD500051E46091490270914A0280914B02909196
:10CD60004C020F94A9AF4B015C01E0905D0BF09079
:10CD70005E0B00915F0B1091600B2091590B30916D
:10CD80005A0B40915B0B50915C0B6091550B70916D
:10CD9000560B8091570B9091580BE1E4FBE0FF9309
:10CDA000EF93B1E6CB2EBBE0DB2E0F94A00D0F94DA
:10CDB000142720E030E040EA51E46091490270918C
:10CDC0004A0280914B0290914C020F94A9AF0F94AC
:10CDD00011B08B0120E030E040E252E4609151025A
:10CDE0007091520280915302909154020F94A9AF16
:10CDF0000F9411B07B010E9471D88CAF0F900F90EF
:10CE0000A8AD1A1614F129C02996BFAD2997BB23E6
:10CE100071F0E8E6FDE08491882309F496CF9091C3
:10CE2000C00095FFFCCF8093C6003196F4CFEEE3AF
:10CE3000FDE08491882309F488CF9091C00095FF8C
:10CE4000FCCF8093C6003196F4CF9CAD992379F145
:10CE5000ECE1FDE08491811122C080E00E94F33575
:10CE6000E2E4F3E32696FFAFEEAF2697212C312CB8
:10CE7000C701AA2797FDA095BA2F66968CAF9DAFE4
:10CE8000AEAFBFAF6697C801AA2797FDA095BA2F8E
:10CE90006A968CAF9DAFAEAFBFAF6A9715C0909149
:10CEA000C00095FFFCCF8093C6003196D3CFE6EF4C
:10CEB000FCE08491882389F29091C00095FFFCCF1B
:10CEC0008093C6003196F5CFA8AD1A16A4F4E5EF0D
:10CED000FCE08491882341F09091C00095FFFCCF45
:10CEE0008093C6003196F5CF8091C00085FFFCCFBE
:10CEF0008AE08093C600C10163E070E00F9481B4C2
:10CF000028967FAF6EAF289722969FAF8EAF22975D
:10CF10002796FFAD2797F0FF08C022E030E0281BDE
:10CF2000390B22963FAF2EAF22973CAD332309F445
:10CF300077C02114310409F473C028968EAD9FADDB
:10CF40002897880F991F2896AEADBFAD28978A0FF6
:10CF50009B1F2296EEADFFAD22978E0F9F1F880F6D
:10CF6000991F8D53904F0F943DBBBC01882777FDCF
:10CF70008095982F0F9444B02AE037ED43E25CE3AC
:10CF80000F94A3B22091E7123091E8124091E91278
:10CF90005091EA120F94B2AE2B013C01F8AD1F166E
:10CFA0000CF041C0EFEDFCE08491882341F09091BA
:10CFB000C00095FFFCCF8093C6003196F5CF4AE0C4
:10CFC00050E0B1018EE09AE00E949E34EDECFCE06E
:10CFD0008491882341F09091C00095FFFCCF80930D
:10CFE000C6003196F5CF25E030E0B301A2018EE016
:10CFF0009AE00E949635ECECFCE08491882341F0A5
:10D000009091C00095FFFCCF8093C6003196F5CF7C
:10D010008091C00085FFFCCF8AE08093C60003C0EA
:10D02000412C512C320180E090E0A0EAB0E48093E2
:10D030005D0B90935E0BA0935F0BB093600B6696B5
:10D040006CAD7DAD8EAD9FAD66970F9444B02D96BF
:10D050006CAF7DAF8EAF9FAF2D972091590B309164
:10D060005A0B40915B0B50915C0B6091550B70918A
:10D07000560B8091570B9091580BA1E4BBE0BF93E6
:10D08000AF932D968CAC9DACAEACBFAC2D97B1E6FA
:10D09000CB2EBBE0DB2EE12CF12C00EA10E40F9448
:10D0A000A00D0F9414272696EEADFFAD269785911F
:10D0B0009591A591B4918093550B9093560BA093A5
:10D0C000570BB093580B2696EEADFFAD26973496CE
:10D0D00085919591A591B4918093590B90935A0B9A
:10D0E000A0935B0BB0935C0B69E57BE085E59BE06F
:10D0F0000E9468390F900F90F8AD1F16A4F16A9640
:10D100006CAD7DAD8EAD9FAD6A970F9444B04B0171
:10D110005C01E0905D0BF0905E0B00915F0B109155
:10D12000600B2091590B30915A0B40915B0B509141
:10D130005C0B6091550B7091560B8091570B909141
:10D14000580BA1E4BBE0BF93AF93A1E6CA2EABE0BE
:10D15000DA2E0F94A00D0F9414270F900F90FCADB2
:10D16000F11129C034C04AE050E0B1018EE09AE0EC
:10D170000E949E3429962FAD2997222371F0EDEB62
:10D18000FCE08491882309F4BACF9091C00095FF08
:10D19000FCCF8093C6003196F4CFEBEAFCE084919B
:10D1A000882309F4ACCF9091C00095FFFCCF809309
:10D1B000C6003196F4CF2114310449F020E030E06C
:10D1C00040E85FE3C301B2010F94B1AE04C060E078
:10D1D00070E080E291EC20E030E043E00E94BEDBB2
:10D1E000811103C0E7E2F8E21AC080905D0B9090D5
:10D1F0005E0BA0905F0BB090600BA501940160E006
:10D2000070E080EA90E40F94B1AE2DEC3CEC4CEC75
:10D210005DE30F94A2AF87FF05C0E5E2F8E26590F9
:10D22000749004C1FCADFF2391F0A5019401C301EA
:10D23000B2010F94B1AE9F7720E030E040E85FE3A9
:10D240000F94D1B118161CF4E9E2F8E2E8CF28AD4A
:10D250002A305CF40E94A4524B015C0138AD1316D5
:10D260000CF09CC0ECE8FCE05FC0E7EAFCE08491D5
:10D27000882341F09091C00095FFFCCF8093C600B9
:10D280003196F5CF4091550B5091560B6091570B4D
:10D290007091580B25E030E08EE09AE00E949635C0
:10D2A000E6EAFCE08491882341F09091C00095FF6C
:10D2B000FCCF8093C6003196F5CF8091C00085FFEA
:10D2C000FCCF8AE08093C600E2EAFCE084918823E8
:10D2D00041F09091C00095FFFCCF8093C60031963D
:10D2E000F5CF4091590B50915A0B60915B0B7091A7
:10D2F0005C0B25E030E08EE09AE00E949635E0EA93
:10D30000FCE08491882309F4A5CF9091C00095FF9B
:10D31000FCCF8093C6003196F4CF9091C00095FF6A
:10D32000FCCF8093C600319684918111F6CF409155
:10D330005D0B50915E0B60915F0B7091600B25E06F
:10D3400030E08EE09AE00E949635E2E8FCE08491BD
:10D35000882341F09091C00095FFFCCF8093C600D8
:10D360003196F5CF25E030E0B501A4018EE09AE0DA
:10D370000E949635E1E8FCE08491882341F0909189
:10D38000C00095FFFCCF8093C6003196F5CF809109
:10D39000C00085FFFCCF8AE08093C60087E0289616
:10D3A000AEADBFAD28978A9F80018B9F100D1124D1
:10D3B0002296EEADFFAD22970E0F1F1F000F111F1B
:10D3C000000F111F0A511D4EA501940160915D0BC4
:10D3D00070915E0B80915F0B9091600B0F94B1AEDA
:10D3E000D80111966D937D938D939C9314978091A2
:10D3F000810B9091820B01979093820B8093810B0C
:10D40000BFEF2B1A3B0A81E00F9470582696EEADC1
:10D41000FFAD269738962696FFAFEEAF2697F9E038
:10D420002F16310409F050CD612C712C28AD243118
:10D43000A4F0EAE5FCE08491882341F09091C000DB
:10D4400095FFFCCF8093C6003196F5CF8091C00048
:10D4500085FFFCCF8AE08093C60080E090E0A0EAE0
:10D46000B0E480935D0B90935E0BA0935F0BB09341
:10D47000600B38AD343114F1E5E4FCE0849188238D
:10D4800041F09091C00095FFFCCF8093C60031968B
:10D49000F5CF8091C00085FFFCCF8AE08093C60065
:10D4A00040915D0B50915E0B60915F0B7091600B32
:10D4B00025E030E08EE09AE00E949635E0905D0B2A
:10D4C000F0905E0B00915F0B1091600B2091590B57
:10D4D00030915A0B40915B0B50915C0B6091550B56
:10D4E0007091560B8091570B9091580BE1E4FBE043
:10D4F000FF93EF932D968CAC9DACAEACBFAC2D974B
:10D50000E1E6CE2EEBE0DE2E0F94A00D0F94142753
:10D510000F900F9089E02816310421F060E0C301DC
:10D520000C9417750E942136E2E3FCE08491882375
:10D5300041F09091C00095FFFCCF8093C6003196DA
:10D54000F5CF8091C00085FFFCCF8AE08093C600B4
:10D550000F948801E1E2FCE08491882341F09091EE
:10D56000C00095FFFCCF8093C6003196F5CF809127
:10D57000C00085FFFCCF8AE08093C60080EC9FE06E
:10D580000F9430BBEE24E394813009F0E12C98AD88
:10D5900019164CF0DE0111966D01F12C2CE4622E6F
:10D5A00036E4732E1CC0EE2069F0E6E0FCE08491C6
:10D5B000882381F39091C00095FFFCCF8093C60033
:10D5C0003196F5CFE7EEFBE08491882319F3909133
:10D5D000C00095FFFCCF8093C6003196F5CF6982DD
:10D5E000B2E5BA837B8282E48C83F60181916F017C
:10D5F0000E944736882319F00E9471361EC0EE2023
:10D6000009F436C1F1E0FF1528F0F11009C08FEBE5
:10D610009FE00BC022E0F21206C08DEB9FE005C038
:10D620008EEB9FE002C08CEB9FE00F9430BB682F25
:10D63000772767FD7095872F972F611571058105F5
:10D64000910509F415C10F9444B02FE632E143E887
:10D650005AE30F94A3B24B015C019F7727E139EDA8
:10D660004EEC5DE30F94D1B118160CF037C0E3E433
:10D67000F0E18491882341F09091C00095FFFCCFA8
:10D680008093C6003196F5CFE3ECFBE084918823CC
:10D6900041F09091C00095FFFCCF8093C600319679
:10D6A000F5CF22E030E0B501A4018EE09AE00E94BF
:10D6B0009635EAEBFBE08491882341F09091C0001D
:10D6C00095FFFCCF8093C6003196F5CF8091C000C6
:10D6D00085FFFCCF8AE08093C600CAC0F2E0FF1647
:10D6E00009F469C023E0F21609F494C031E0F3169E
:10D6F00089F120E030E040E05FE3C501B4010F9420
:10D70000A3B21B012C0107EE12E1A2019101D80185
:10D7100014966D917D918D919C9117970F94B2AE57
:10D72000F8016483758386839783A50194016081E2
:10D730007181828193810F94B2AED8016D937D93F4
:10D740008D939C931397045E1F4FB3E10B331B071C
:10D75000E1F68EC020E030E040E05FE3C501B401B7
:10D760000F94A3B21B012C010BEE12E1A201910157
:10D77000F80160817181828193810F94B2AED801EA
:10D780006D937D938D939C931397A50194011496AB
:10D790006D917D918D919C9117970F94B2AEF80188
:10D7A0006483758386839783045E1F4FF3E10F3391
:10D7B0001F07E1F65DC020E030E040E05FE3C50117
:10D7C000B4010F94A3B21B012C0107EE12E1A201D8
:10D7D0009101D8015C966D917D918D919C915F979F
:10D7E0000F94B2AEF801648F758F868F978FA50165
:10D7F000940160817181828193810F94B2AED801CE
:10D800006D937D938D939D938D01B2E1033F1B0733
:10D81000F1F62EC020E030E040E05FE3C501B40146
:10D820000F94A3B21B012C0103E013E1A2019101AB
:10D83000F80160817181828193810F94B2AED80129
:10D840006D937D938D939D938D01A50194015896C1
:10D850006D917D918D919C915B970F94B2AEF80183
:10D86000608F718F828F938FF3E10F301F07F1F676
:10D87000F39424E0F212B3CEE9E9FBE0849188232B
:10D8800041F09091C00095FFFCCF8093C600319687
:10D89000F5CF8091C00085FFFCCF8AE08093C60061
:10D8A00086EE92E10F948802E7E8FBE084918823FA
:10D8B00041F09091C00095FFFCCF8093C600319657
:10D8C000F5CF8091C00085FFFCCF8AE08093C60031
:10D8D00081E08093E612EBE6FBE08491882341F03F
:10D8E0009091C00095FFFCCF8093C6003196F5CF94
:10D8F0008091C00085FFFCCF8AE08093C6000E9423
:10D9000075F7EAE5FBE08491882341F09091C0002F
:10D9100095FFFCCF8093C6003196F5CF8091C00073
:10D9200085FFFCCF8AE08093C600E091410B34E094
:10D93000E39FF0011124E652F54E20E030E042E092
:10D9400053E460817181828193810F94D1B1181663
:10D9500094F48091BF0B882371F086EA9FE00F94C6
:10D9600030BB882341F08091E01A9091E11AC29770
:10D9700014F00C945F8B2E968FAD2E978093860BB0
:10D980006096AEADBFAD6097B093840BA093830B50
:10D990006296EEADFFAD6297F093820BE093810B40
:10D9A0001092940B1092930B82E00F9470580C9489
:10D9B000898A8091E612882309F49EC0E0E5FBE0A5
:10D9C0008491882341F09091C00095FFFCCF809313
:10D9D000C6003196F5CF4AE050E067E070E08EE097
:10D9E0009AE00E949E34EEE4FBE08491882341F0AB
:10D9F0009091C00095FFFCCF8093C6003196F5CF83
:10DA00004AE050E067E070E08EE09AE00E949E34C9
:10DA1000EBE3FBE08491882341F09091C00095FFF7
:10DA2000FCCF8093C6003196F5CF4AE050E065E028
:10DA300070E08EE09AE00E949E34E9E2FBE084917F
:10DA4000882341F09091C00095FFFCCF8093C600E1
:10DA50003196F5CF8091C00085FFFCCF8AE080939E
:10DA6000C60000E010E086E2A82E8BE0B82E94E21B
:10DA7000892E9BE0992EE12CF12C980122573C4EE7
:10DA80006901F5018491E6E2FBE0882349F0909179
:10DA9000C00095FFFCCF8093C60031968491F5CFEE
:10DAA000F601EE0DFF1D418152816381748125E0F5
:10DAB00030E08EE09AE00E949635F4E0EF0EF11C23
:10DAC0002CE1E216F104E9F6F4018491E4E2FBE0D2
:10DAD000882349F09091C00095FFFCCF8093C60049
:10DAE00031968491F5CF0C5111090C33FFEF1F07CC
:10DAF00009F0C1CF0C94898AE6E0FBE08491882389
:10DB000041F09091C00095FFFCCF8093C600319604
:10DB1000F5CF8091C00085FFFCCF8AE08093C600DE
:10DB20000C94898A81E00E948D3A0C94898A109223
:10DB30000B0B0C94898A85E40E944736811102C040
:10DB40000F941427B2E16B2EB6E07B2E19E4812EE0
:10DB50001BE0912E05E5A02E0BE0B02E512CD30139
:10DB60008D913D010E9447368823D9F1B3E05B12C5
:10DB70000CC00E94A736F501608371838283938372
:10DB800081E69BE00F94ED1B2CC00E94A736D401C8
:10DB90002D913D914D915C910F94B2AEF501608352
:10DBA000718382839383E0905D0BF0905E0B009114
:10DBB0005F0B1091600B2091590B30915A0B4091E3
:10DBC0005B0B50915C0B6091550B7091560B8091E3
:10DBD000570B9091580BA1E6CA2EABE0DA2E0F94AA
:10DBE0004E1A5394F4E08F0E911C24E0A20EB11C47
:10DBF00034E05312B4CF0C94898A81E08093ED1BFA
:10DC00000F94BCA66093D00B7093D10B8093D20B72
:10DC10009093D30B6091ED1B84EC9FE00F9442BB7B
:10DC20000C94898A8DE40E944736882311F40C9461
:10DC30007088E091A310F091A41031968191803208
:10DC4000E9F38930D9F380538A30B0F0E7EFFAE096
:10DC50008491882341F09091C00095FFFCCF809380
:10DC6000C6003196F5CF8091C00085FFFCCF8AE0D9
:10DC70008093C6000C94898A0E94A7360F9411B035
:10DC80006B3C710511F40C948D7C0CF021C16F324A
:10DC9000710509F4AAC60CF06AC06931710509F46E
:10DCA00051C3B4F56431710509F4F1C294F46131E2
:10DCB000710509F4E0C234F46230710508F434C22D
:10DCC0000C945B886231710511F40C9464780C94A7
:10DCD0005B886631710509F414C30CF40CC3673119
:10DCE000710509F414C36831710511F00C945B8857
:10DCF00084ED9BE00E94D8A70F94BCA66093FF0A16
:10DD00007093000B8093010B9093020B0C94898A03
:10DD10006E31710509F45FC38CF46B31710509F440
:10DD200025C30CF415C36C31710509F425C36D319D
:10DD3000710511F40C94898A0C945B886A32710520
:10DD400009F477C454F46F31710509F412C46032D8
:10DD5000710509F478C30C945B886C32710509F481
:10DD6000AFC46D32710509F4BAC40C945B886D368A
:10DD7000710509F4B2C70CF064C06535710511F482
:10DD80000C949D780CF03DC06235710511F40C9433
:10DD90005B785CF56135710511F00C945B880F942C
:10DDA00044310F941427149A0F9496271092400B25
:10DDB00010923F0B68EE73E080E090E00F94EBA6CA
:10DDC00010921002E9E5F7E24591549122EB3AE016
:10DDD00060EB7AE082EB94E00E94B6BC0F94F156BF
:10DDE00080E00F9470580C94898A6335710511F4A2
:10DDF0000C945F786435710511F40C9464780C947C
:10DE00005B886936710509F425C65CF46C357105CB
:10DE100011F40C94B8786836710509F4EAC50C94CD
:10DE20005B886A36710511F40C942B786B3671059A
:10DE300011F00C945B881092400B10923F0B0C94E5
:10DE4000898A6837710511F40C94837AFCF462377F
:10DE5000710511F40C947B794CF46037710511F065
:10DE60000C945B8863E082EC98E0E1C56337710550
:10DE700011F40C943B796737710511F00C945B88B1
:10DE8000E5E8F7E2859194910C94947A6E3B7105E4
:10DE900009F4B9C75CF46937710511F40C94887AF8
:10DEA0006C38710509F4C5C50C945B88683C710534
:10DEB00011F40C94FB7B693C710511F00C945B88A8
:10DEC00002E116E06DE9E62E69E1F62E0C94727C13
:10DED000673F81E0780711F40C94B8800CF07EC0A5
:10DEE0006C32A1E07A0711F40C94BD7EC4F5603D5C
:10DEF000710511F40C94977DA4F46D3C710511F437
:10DF00000C94CC7C14F40C94AA7C6E3C710511F436
:10DF10000C94437D6F3C710511F40C94607D0C945E
:10DF20005B886D3D710511F40C94317E64F4613DA4
:10DF3000710511F40C94BF7D6C3D710511F40C94C6
:10DF4000207E0C945B88623E710511F40C945B7E1C
:10DF5000603F710511F40C94898A0C945B886036DB
:10DF6000E1E07E07E4F46E35F1E07F0714F00C94F5
:10DF7000898A6E3221E0720711F40C94628014F4E5
:10DF80000C94F57E6F3281E0780711F40C94718067
:10DF90006033714011F40C94C07F0C945B88643F33
:10DFA000A1E07A0711F40C94AA804CF46039714016
:10DFB00011F00C945B880F9414270C94898A653FA8
:10DFC000F1E07F0711F40C94B180663F714011F0CD
:10DFD0000C945B880E949B2A0C94898A6E3833E0EB
:10DFE000730711F40C949C850CF047C06D3B92E0D4
:10DFF000790711F40C94ED86FCF46835B2E07B07E8
:10E0000011F40C94CC815CF46D3F714011F00C94D0
:10E010005B880F948256EDE3F0E10C94C48069357F
:10E0200022E0720711F40C9457856A35724011F49E
:10E030000C9465850C945B88643883E0780711F450
:10E040000C9473856CF46E3BA2E07A0711F40C9487
:10E05000FD876335734011F40C94D6800C945B8873
:10E060006B38E3E07E0711F40C9476856C387340CE
:10E0700011F40C94898A0C945B88633923E072074D
:10E0800011F40C940686D4F4603983E0780711F417
:10E090000C94D18514F40C949F856139A3E07A0720
:10E0A00011F40C9403866239734011F00C945B8870
:10E0B00010924D1B0F9427440C94898A6639E3E033
:10E0C0007E0711F40C94BB866CF4643923E072076C
:10E0D00011F40C940C866539734011F40C94898604
:10E0E0000C945B88603A83E0780709F415C2673EB8
:10E0F000734011F00C945B881092F50A0F941D5731
:10E1000080918F1090919010A0919110B0919210E9
:10E110008093931090939410A0939510B0939610C1
:10E120000E94E4430C94898A0091A3101091A410DA
:10E130000E5F1F4F80E50E944736882379F00E94CA
:10E14000A7360F9416B04B015C01FF24F3946115C0
:10E1500071058105910531F4F12C04C0F12C812C5D
:10E16000912C540183E50E944736882399F00E9440
:10E17000A73620E030E04AE754E40F94A3B20F94AE
:10E1800016B04B015C01EE24E39461157105810525
:10E19000910509F4E12C6AE270E0C8010F9484B89B
:10E1A000009711F0DC011C92F801CF01219120327F
:10E1B000E1F3F11007C0E11005C0222319F00F941C
:10E1C000E45606C0EBE9F6E2859194910F94F1567E
:10E1D00081E00F94C4560F9414270F94BCA660934B
:10E1E000070B7093080B8093090B90930A0B811413
:10E1F0009104A104B104A9F00F94BCA62B013C0129
:10E20000480C591C6A1C7B1C0F94BCA66415750530
:10E2100086059705C8F40F94F85A811115C00C941F
:10E22000A18B0F94F65A882311F40C94898A0F94C9
:10E23000F85A81110CC00F94AA3881E00E94DF4A7D
:10E2400080E00F947058F3CF80E00F94C456809113
:10E25000D60B882341F0E9E2F7E2859194910F947F
:10E26000F1560C94898AE3E8F6E2859194910F9433
:10E27000F1560C94898AEBE5F7E2859194910F941D
:10E28000F15617981698159814980C94898AE1E11C
:10E29000F8E285919491FC012491222341F0309180
:10E2A000C00035FFFCCF2093C6000196F4CF8091CB
:10E2B000C00085FFFCCF8AE08093C60084ED9BE020
:10E2C0000E94A9A6E5EEF7E285919491FC012491C4
:10E2D000222341F03091C00035FFFCCF2093C600CF
:10E2E0000196F4CF8091C00085FFFCCF8AE0809337
:10E2F000C6000C94898A84ED9BE00E94FFA60C94D2
:10E30000898A84ED9BE00E94D4A70C94898A80912D
:10E31000A3109091A4106AE270E004960F9484B860
:10E32000009711F0DC011C926091A3107091A41071
:10E330006C5F7F4F21E041E084ED9BE00E9480AC68
:10E340000C94898A84ED9BE00E94DFA70C94898A53
:10E350008091D70B882311F40C94898A83E50E945D
:10E36000473681110C94AB8B0C94898A84ED9BE029
:10E370000E9484A90C94898A8091A3109091A41082
:10E380006AE270E004960F9484B88C010097A9F0BB
:10E390008091AD109091AE106EE470E08E549F4E5F
:10E3A0000F9484B860E270E00F9484B80196909363
:10E3B000A4108093A310F80110826091A3107091B3
:10E3C000A4106C5F7F4F21E040E084ED9BE00E9451
:10E3D00080AC0C94898A8091D70B882311F40C941B
:10E3E000898A60E084ED9BE00E9410AC8091A310CC
:10E3F0009091A4106AE270E004960F9484B88C01A6
:10E400000097A9F08091AD109091AE106EE470E08D
:10E410008E549F4E0F9484B860E270E00F9484B8DD
:10E4200001969093A4108093A310D8011C92609140
:10E43000A3107091A4106C5F7F4F84ED9BE00E944D
:10E4400043A80C94898A8091D60B81110F941427CC
:10E450000091A3101091A4100C5F1F4F6AE270E0AE
:10E46000C8010F9484B87C0161E270E0C8010F9488
:10E4700084B8009719F08C010F5F1F4FE114F1046D
:10E4800011F0F701108280E50E944736F82E2091A6
:10E49000A3103091A4100217130708F4F12C8091F7
:10E4A000D70B882311F40C94898A21E02F2541E0B1
:10E4B000B80184ED9BE00E9480AC83E50E94473662
:10E4C0008823B9F02091A3103091A41020173107B0
:10E4D00080F40E947136AB01BC014093720E5093E0
:10E4E000730E6093740E7093750E8DEB9DE00E9419
:10E4F000329A84ED9BE00E94D8A7F1100C94898A8F
:10E500000F94BCA66093FF0A7093000B8093010BDD
:10E510009093020B0C94898A8091A3109091A4107F
:10E520006AE270E005960F9484B88C010097A9F018
:10E530008091AD109091AE106EE470E08E549F4EBD
:10E540000F9484B860E270E00F9484B801969093C1
:10E55000A4108093A310D8011C926091A310709115
:10E56000A4106B5F7F4F84ED9BE00E94BEAF0C94C4
:10E57000898A0F94BCA66093FB0A7093FC0A80936F
:10E58000FD0A9093FE0A0091FF0A1091000B209162
:10E59000010B3091020B601B710B820B930B28EE69
:10E5A00033E040E050E00F9494B4CA01B9012CE389
:10E5B00030E040E050E00F9494B47F936F933F932A
:10E5C0002F9388EE9AE09F938F93CE0101969F93AD
:10E5D0008F930F9404B9EDE3F0E184910FB6F894B2
:10E5E000DEBF0FBECDBFEDE3F0E1882349F090918F
:10E5F000C00095FFFCCF8093C60031968491F5CF83
:10E60000FE0131968191882339F09091C00095FFE9
:10E61000FCCF8093C600F6CF8091C00085FFFCCF71
:10E620008AE08093C600CE0101960F94E4560C94C4
:10E63000898A83E50E944736882311F40C94898ADD
:10E640000E94A7360F9411B0F62EE72E862F9E2D2E
:10E650008C0180E50E944736882331F00F3F110579
:10E6600009F010F40C94BC8B0DE010E0EAEDF5E03D
:10E67000819191918017910711F40C94898A26E079
:10E68000E231F207A9F70630110539F48F2D9E2DDE
:10E690009093400B80933F0B04C017FF02C00C9473
:10E6A000898A61E0802F0F94A7A86F2D802F0F9487
:10E6B000E0A86F2D7E2D802F0F948FA70C94898A50
:10E6C0008FEF0E948D3A60E070E088EF9FE00F943A
:10E6D0005CBB0E942BD80E94BED80C94898A8AE524
:10E6E0000E944736382E811112C01092E11A109202
:10E6F000E01A1092E31A1092E21A1092E51A1092A0
:10E70000E41A1092E71A1092E61A0F942D5680E040
:10E710000F94DD5986EE92E10F946D020E94BED8EF
:10E720000F94BB011092460B1092470B1092480BAE
:10E7300081E00E94F335E3E4F8E2859194910E9430
:10E740007F3A0E94B9420E94423D882309F448C1A1
:10E750000E94EC4220E030E048E452E46091DA1A92
:10E760007091DB1A8091DC1A9091DD1A0F94D1B16F
:10E77000181684F020E030E048E452E46091C81AB2
:10E780007091C91A8091CA1A9091CB1A0F94D1B185
:10E79000181624F4332011F40C94C38B80E090E01D
:10E7A000A0EAB0E480935D0B90935E0BA0935F0BA7
:10E7B000B093600B20E030E040E252E460915102FF
:10E7C0007091520280915302909154020F94A9AF1C
:10E7D0004B015C012091590B30915A0B40915B0B1E
:10E7E00050915C0B6091550B7091560B8091570BBB
:10E7F0009091580BE1E4FBE0FF93EF93E1E6CE2E1E
:10E80000EBE0DE2EE12CF12C00EA10E40F94A00DD9
:10E810000F94142786E50E9447360F900F908823A7
:10E82000A1F08091A3109091A410DC0111962C917D
:10E83000293069F02F7D71F04AE050E060E070E02F
:10E8400001960F9495B668AF07C018AE05C0B1E049
:10E85000B8AF02C0E1E0E8AF3320B1F00E9421364A
:10E860000E9413D90E942FDB0E94DBF7882309F452
:10E87000B5C087EF9FE00F9430BB803F09F0AEC07A
:10E8800081E00E948D3AAAC08FEF0E948D3A60E02D
:10E8900070E088EF9FE00F945CBB1982BE016F5F50
:10E8A0007F4F88AD0E9432F03C010E942136212C1E
:10E8B000312C10EA412E10E4512E20925D0B309243
:10E8C0005E0B40925F0B5092600B20E030E040E224
:10E8D00052E46091510270915202809153029091E2
:10E8E00054020F94A9AF4B015C012091590B309158
:10E8F0005A0B40915B0B50915C0B6091550B7091E2
:10E90000560B8091570B9091580BA1E4BBE0BF933D
:10E91000AF9301E6C02E0BE0D02E820171010F945F
:10E92000A00D0F9414270F900F9077FC48C0198208
:10E9300086EE92E10F946D020E9485D881E00E94DC
:10E94000F3350E94B942AE014F5F5F4F68AD81E081
:10E950000E94F3F93C010E94213620925D0B309217
:10E960005E0B40925F0B5092600B20E030E040E283
:10E9700052E4609151027091520280915302909141
:10E9800054020F94A9AF4B015C012091590B3091B7
:10E990005A0B40915B0B50915C0B6091550B709141
:10E9A000560B8091570B9091580BA1E4BBE0BF939D
:10E9B000AF930F94A00D0F9414270F900F906981BF
:10E9C000C3010F941E5C77FC09C086EE0E948D3A4D
:10E9D000EDE3F8E2859194910F94E55B0F94264363
:10E9E00081E00F94DD590C94898A0F949F6F0C94E9
:10E9F000898A88E690E00E94994B81110C94898A5B
:10EA000083E50E944736882371F00091F60A0E9440
:10EA1000A73610E0000F111F0E51154E0F9411B0C4
:10EA2000D8016D937C930F9443310C94898A0E9492
:10EA30006A4A83E50E944736882311F40C94898A38
:10EA40000E94A7360F9411B07093E11A6093E01AF8
:10EA50000C94898A89E690E00E94994B81110C946C
:10EA6000898AE2EEFAE08491882341F09091C00017
:10EA700095FFFCCF8093C6003196F5CFE091F60A62
:10EA8000B4E0EB9FF0011124E652F54E4081518134
:10EA90006281738121E030E08EE09AE00E94963539
:10EAA000EFEDFAE08491882341F09091C00095FF4A
:10EAB000FCCF8093C6003196F5CFE091F60AF0E0E6
:10EAC000EE0FFF1FEE51F54E60817181882777FDB3
:10EAD0008095982F0F9444B0AB01BC0121E030E049
:10EAE0008EE09AE00E949635EBEDFAE0849188235F
:10EAF00041F09091C00095FFFCCF8093C600319605
:10EB0000F5CF4091C81A5091C91A6091CA1A7091F4
:10EB1000CB1A21E030E08EE09AE00E949635E8EDD5
:10EB2000FAE08491882341F09091C00095FFFCCFDA
:10EB30008093C6003196F5CF6091E01A7091E11A8A
:10EB4000882777FD8095982F0F9444B0AB01BC01C6
:10EB500021E030E08EE09AE00E949635E5EDFAE0A3
:10EB60008491882341F09091C00095FFFCCF809361
:10EB7000C6003196F5CF4AE050E060E070E08EE0EC
:10EB80009AE00E949E34E3EDFAE08491882341F0FC
:10EB90009091C00095FFFCCF8093C6003196F5CFD1
:10EBA0004091DA1A5091DB1A6091DC1A7091DD1AEB
:10EBB00021E030E08EE09AE00E949635E0EDFAE048
:10EBC0008491882341F09091C00095FFFCCF809301
:10EBD000C6003196F5CF6091E21A7091E31A88274A
:10EBE00077FD8095982F0F9444B0AB01BC0121E0D4
:10EBF00030E08EE09AE00E949635ECECFAE08491E9
:10EC0000882341F09091C00095FFFCCF8093C6000F
:10EC10003196F5CF8091F60A90E00F94C42E4AE029
:10EC200050E0BC018EE09AE00E949E34E7ECFAE0EE
:10EC30008491882341F09091C00095FFFCCF809390
:10EC4000C6003196F5CF8FEF9FEF0F94C42E4AE0A8
:10EC500050E0BC018EE09AE00E949E34E3ECFAE0C2
:10EC60008491882341F09091C00095FFFCCF809360
:10EC7000C6003196F5CF4091D41A5091D51A6091C3
:10EC8000D61A7091D71A21E030E08EE09AE00E9407
:10EC90009635EFEBFAE08491882341F09091C00023
:10ECA00095FFFCCF8093C6003196F5CF4091CE1AE8
:10ECB0005091CF1A6091D01A7091D11A21E030E0B2
:10ECC0008EE09AE00E9496358091C00085FFFCCFCF
:10ECD0008AE08093C6000C94FE8B8DE690E00E9443
:10ECE000994B81110C94898AE1EBF7E2859194911B
:10ECF0000F94F15681E090E090938A0B8093890BFA
:10ED00008091ED1B882321F081E090E00F945F5605
:10ED100083E50E944736882391F00091F60A0E940D
:10ED2000A73610E0000F111F0E51154E0F9411B0B1
:10ED3000F8017183608381E08093060215C082E54B
:10ED40000E944736882381F00091F60A0E94A73678
:10ED500010E0000F111F0E51154E0F9411B0D80185
:10ED60006D937C93109206020F9443310F94BCA6CE
:10ED70006B017C010091F60A10E0F801EE0FFF1F15
:10ED8000EE51F54E60817181882777FD8095982F2F
:10ED90000F9444B0F801EE0FFF1FEE0FFF1FE65275
:10EDA000F54E11E020813181428153810F94D1B120
:10EDB00018160CF010E01093F40A1092300BC701F3
:10EDC000B6010E94224DEFEAF7E2859194910F94EB
:10EDD000F15682E090E090938A0B8093890B8091AA
:10EDE000ED1B882321F082E090E00F945F560F9492
:10EDF000BCA66093070B7093080B8093090B90934C
:10EE00000A0B0C94898AEBE2F8E2859194910F94B5
:10EE1000F15683E090E090938A0B8093890B809168
:10EE2000ED1B882321F081E090E00F945F5683E58D
:10EE30000E944736882361F00E94A7360F9411B0D4
:10EE40007093E11A6093E01A81E0809306020FC08C
:10EE500082E50E944736882351F00E94A7360F941E
:10EE600011B07093E11A6093E01A109206020F94A9
:10EE7000BCA62B013C011092300B6091E01A7091FE
:10EE8000E11A882777FD8095982F0F9444B011E000
:10EE90002091C81A3091C91A4091CA1A5091CB1AC0
:10EEA0000F94D1B118160CF010E01093F40A0CEB8B
:10EEB0001AE098EBE92E9AE0F92E24EBA22E2AE034
:10EEC000B22E3AE0D32E8091F40A6091E01A70914C
:10EED000E11A882309F490C08091300B81118CC015
:10EEE000882777FD8095982F0F9444B02091C81AF9
:10EEF0003091C91A4091CA1A5091CB1A0F94D1B1CE
:10EF000018160CF090C00F94BCA6641975098609F8
:10EF10009709693E73408105910508F464C08091AA
:10EF2000ED1B81115CC0E091410B24E0E29FF001F8
:10EF30001124E652F54E4081518162817381F801BE
:10EF40008491ECEBFAE0882349F09091C00095FFA2
:10EF5000FCCF8093C60031968491F5CF22E030E05B
:10EF60008EE09AE00E949635F7018491E8EBFAE092
:10EF7000882349F09091C00095FFFCCF8093C60094
:10EF800031968491F5CF6091410B70E04AE050E0FA
:10EF90008EE09AE00E949E34F5018491E4EBFAE061
:10EFA000882349F09091C00095FFFCCF8093C60064
:10EFB00031968491F5CF4091C81A5091C91A609149
:10EFC000CA1A7091CB1A21E030E08EE09AE00E94DC
:10EFD00096358091C00085FFFCCFD092C6000F947B
:10EFE000BCA62B013C010F94AA3880E00E94DF4AA6
:10EFF00080E00F94705867CF882777FD8095982F11
:10F000000F9444B02091C81A3091C91A4091CA1A7D
:10F010005091CB1A0F94A2AF87FF05C080910602D2
:10F02000882309F470CFEDE2F8E2859194910F9472
:10F03000F15684E090E090938A0B8093890B0F94B3
:10F04000BCA66093070B7093080B8093090B9093F9
:10F050000A0B0C94898A83E50E944736882319F1AC
:10F060000E94A73620E030E0A9010F94A2AF87FDEF
:10F070000FC00E94A73620E030E04FE753E40F9422
:10F08000D1B1181644F00E94A7360F9411B005C0F4
:10F0900060E070E002C06FEF70E07093400B60932F
:10F0A0003F0B0C94898A8FEF90E09093400B8093F4
:10F0B0003F0B0C94898A1092CF0B0C94898A81E0C3
:10F0C0008093CF0B0C94898A83E50E94473688236E
:10F0D00099F00E94A73620E030E04AE754E40F940C
:10F0E000A3B20F9416B06093080270930902809344
:10F0F0000A0290930B021DC088E50E9447368111D9
:10F100000C94DF8B89E50E94473681110C94DF8BCC
:10F110008AE50E94473681110C94DF8B85E40E94BA
:10F12000473681110C94DF8B0F941427149A0F9497
:10F1300096271092800B0C94898A83E50E944736AB
:10F14000882311F40C94898A0E94A73620E030E0CD
:10F150004AE754E40F94A3B20F9416B06093030BE4
:10F160007093040B8093050B9093060B0C94898A83
:10F1700022E136E039AF28AF0DEA19E1BDEBEB2E05
:10F18000B9E1FB2E8DE6282E89E1382ED12CA8ADD1
:10F19000B9AD8D91B9AFA8AF0E944736882309F465
:10F1A0005CC0B3E0DB1252C00E94A7362B013C01C9
:10F1B00020E030E040EA51E40F94A2AF87FF3FC067
:10F1C000A3019201F80160817181828193810F9482
:10F1D000A9AF4B015C019B01AC0160918D1970914D
:10F1E0008E1980918F19909190190F94A3B260930A
:10F1F0008D1970938E1980938F1990939019A50192
:10F200009401D7016D917D918D919C910F94A3B242
:10F21000F7016083718382839383D1016D917D9126
:10F220008D919C910F9442B0A50194010F94A3B2CB
:10F230000F9416B0F1016083718382839383D801A8
:10F240004D925D926D927C92139707C00E94A736F3
:10F25000F8016083718382839383D3940C5F1F4F83
:10F26000F4E0EF0EF11C24E0220E311C34E0D31246
:10F270008ECF0C94898A86E50E9447368823B9F0A0
:10F280000F9409A3FC012491222341F03091C00086
:10F2900035FFFCCF2093C6000196F4CF8091C000CB
:10F2A00085FFFCCF8AE08093C6000C94898A85E5AF
:10F2B0000E944736882369F08091A3109091A41092
:10F2C00001969093A4108093A3100F947AA50C94A8
:10F2D000898AE7E8F7E285919491FC012491222341
:10F2E00011F40C94898A3091C00035FFFCCF209333
:10F2F000C6000196F2CFEDEAFAE08491882341F04E
:10F300009091C00095FFFCCF8093C6003196F5CF59
:10F310004091550B5091560B6091570B7091580BC3
:10F3200022E030E08EE09AE00E949635E9EAFAE0C9
:10F330008491882341F09091C00095FFFCCF809389
:10F34000C6003196F5CF4091590B50915A0B609100
:10F350005B0B70915C0B22E030E08EE09AE00E9443
:10F360009635E5EAFAE08491882341F09091C00057
:10F3700095FFFCCF8093C6003196F5CF40915D0B91
:10F3800050915E0B60915F0B7091600B22E030E05A
:10F390008EE09AE00E949635E1EAFAE084918823B3
:10F3A00041F09091C00095FFFCCF8093C60031964C
:10F3B000F5CF4091610B5091620B6091630B70919E
:10F3C000640B22E030E08EE09AE00E949635E7EF91
:10F3D000F7E285919491FC012491222341F0309130
:10F3E000C00035FFFCCF2093C6000196F4CF80E02B
:10F3F0000F9475270F9444B02091AD193091AE1938
:10F400004091AF195091B0190F94A9AFAB01BC0155
:10F4100022E030E08EE09AE00E949635EDE9FAE0D5
:10F420008491882341F09091C00095FFFCCF809398
:10F43000C6003196F5CF81E00F9475270F9444B044
:10F440002091B1193091B2194091B3195091B4196A
:10F450000F94A9AFAB01BC0122E030E08EE09AE04E
:10F460000E949635E9E9FAE08491882341F0909171
:10F47000C00095FFFCCF8093C6003196F5CF82E0A7
:10F480000F9475270F9444B02091B5193091B61997
:10F490004091B7195091B8190F94A9AFAB01BC01B5
:10F4A00022E030E08EE09AE00E949635E5E9FAE04D
:10F4B0008491882341F09091C00095FFFCCF809308
:10F4C000C6003196F5CF83E00F9475270F9444B0B2
:10F4D0002091B9193091BA194091BB195091BC19BA
:10F4E0000F94A9AFAB01BC0122E030E08EE09AE0BE
:10F4F0000E9496358091C00085FFFCCF8AE0809302
:10F50000C6000C94898A80E00F94C31D0C94898AEC
:10F5100081E00F94C31D0C94898A3091C00035FF9F
:10F52000FCCF2093C6000196FC0124912111F5CF58
:10F530008091C00085FFFCCF8AE08093C600E1E99E
:10F54000F6E285919491FC012491222341F03091BF
:10F55000C00035FFFCCF2093C6000196F4CF1E9B60
:10F5600010C0E9EEF7E285919491FC0124912223E9
:10F57000C1F03091C00035FFFCCF2093C60001964A
:10F58000F4CFE7EEF7E285919491FC0124912223D8
:10F5900041F03091C00035FFFCCF2093C6000196AA
:10F5A000F4CF8091C00085FFFCCF8AE08093C60035
:10F5B000E3E9F6E285919491FC012491222341F044
:10F5C0003091C00035FFFCCF2093C6000196F4CFE8
:10F5D0008091060182FF10C0E9EEF7E285919491D7
:10F5E000FC0124912223C1F03091C00035FFFCCFF3
:10F5F0002093C6000196F4CFE7EEF7E2859194914F
:10F60000FC012491222341F03091C00035FFFCCF52
:10F610002093C6000196F4CF8091C00085FFFCCFF7
:10F620008AE08093C600EBE8F6E285919491FC01B4
:10F630002491222341F03091C00035FFFCCF20936C
:10F64000C6000196F4CF1D9B10C0E9EEF7E285914C
:10F650009491FC0124912223C1F03091C00035FF28
:10F66000FCCF2093C6000196F4CFE7EEF7E2859138
:10F670009491FC012491222341F03091C00035FF88
:10F68000FCCF2093C6000196F4CF8091C00085FF87
:10F69000FCCF8AE08093C600EDE8F6E28591949174
:10F6A000FC012491222341F03091C00035FFFCCFB2
:10F6B0002093C6000196F4CF8091060187FF10C009
:10F6C000E9EEF7E285919491FC0124912223C1F0A7
:10F6D0003091C00035FFFCCF2093C6000196F4CFD7
:10F6E000E7EEF7E285919491FC012491222341F009
:10F6F0003091C00035FFFCCF2093C6000196F4CFB7
:10F700008091C00085FFFCCF8AE08093C600E5E8C9
:10F71000F6E285919491FC012491222341F03091ED
:10F72000C00035FFFCCF2093C6000196F4CF1C9B90
:10F7300010C0E9EEF7E285919491FC012491222317
:10F74000C1F03091C00035FFFCCF2093C600019678
:10F75000F4CFE7EEF7E285919491FC012491222306
:10F7600041F03091C00035FFFCCF2093C6000196D8
:10F77000F4CF8091C00085FFFCCF8AE08093C60063
:10F78000E7E8F6E285919491FC012491222341F06F
:10F790003091C00035FFFCCF2093C6000196F4CF16
:10F7A000019910C0E9EEF7E285919491FC01249152
:10F7B0002223C1F03091C00035FFFCCF2093C6005A
:10F7C0000196F4CFE7EEF7E285919491FC01249144
:10F7D000222341F03091C00035FFFCCF2093C600BA
:10F7E0000196F4CF8091C00085FFFCCF8AE0809322
:10F7F000C6000C94898A8091410B8093F60A84E5B7
:10F800000E944736882329F10E94A7360F9416B02C
:10F810006093F60A6623E9F0EDE3F0E18491882332
:10F8200041F09091C00095FFFCCF8093C6003196C7
:10F83000F5CFE3E8F7E2A591B4918D91882311F417
:10F840000C94898A9091C00095FFFCCF8093C600EC
:10F85000F4CF84E40E944736882311F40C94898AFB
:10F860000E94A73620E030E0A9010F94A2AF8111D9
:10F8700003C01092650B32C00091F60A10E00E949E
:10F88000A736F801EE0FFF1FEE0FFF1FE35CFD4FE1
:10F890006083718382839383E0903D02F0903E0207
:10F8A00000913F021091400220E030E0A901B70131
:10F8B000C8010F94A2AF811104C0E12CF12C00E427
:10F8C00010E4C701D80180933D0290933E02A093BB
:10F8D0003F02B093400281E08093650B0E94EE4CA2
:10F8E0000C94898AD8018D918D010E944736882316
:10F8F00049F00E94A7360F9416B0F7016083718318
:10F9000082839383F4E0EF0EF11C26E006311207A8
:10F9100049F70F94131C0C94898A02E116E05DEB01
:10F92000E52E59E1F52ED8018D918D010E944736C3
:10F93000882339F00E94A736F701608371838283A0
:10F940009383F4E0EF0EF11C26E00631120759F71D
:10F950000C94898A83E50E944736882351F00E94DF
:10F96000A736609395197093961980939719909381
:10F97000981984E50E944736882311F40C94898AEB
:10F980000E94A736609391197093921980939319EE
:10F99000909394190C94898A83E50E9447368823B2
:10F9A00051F00E94A7366093991970939A19809329
:10F9B0009B1990939C1984E50E944736882351F047
:10F9C0000E94A73660937D1970937E1980937F19EA
:10F9D0009093801982E40E944736882361F00E9448
:10F9E000A7360F9416B06093CD197093CE198093FB
:10F9F000CF199093D01988E50E944736882391F05B
:10FA00000E94A73660938519709386198093871991
:10FA10009093881960938119709382198093831948
:10FA20009093841989E50E944736882351F00E94FB
:10FA3000A7366093851970938619809387199093E0
:10FA400088198AE50E944736882351F00E94A7361C
:10FA50006093891970938A1980938B1990938C19EC
:10FA600085E40E944736882311F40C94898A0E9409
:10FA7000A73660938D1970938E1980938F19909388
:10FA800090190C94898A02E116E049E4E42E4BE0D7
:10FA9000F42ED8018D918D010E944736882339F0CC
:10FAA0000E94A736F7016083718382839383F4E019
:10FAB000EF0EF11C26E00531120759F70C94898AE4
:10FAC00083E50E944736882351F00E94A736609351
:10FAD0001D0270931E0280931F029093200286E401
:10FAE0000E944736882381F00E94A73620E030E04C
:10FAF00040E752E40F94A9AF609315027093160289
:10FB000080931702909318028AE50E944736882353
:10FB100011F40C94898A0E94A7366093390B709374
:10FB20003A0B80933B0B90933C0B0C94898A83E5B2
:10FB30000E944736882351F00E94A7366093350B08
:10FB40007093360B8093370B9093380B86E40E94AA
:10FB50004736882311F40C94898A0E94A73620E046
:10FB600030E040E752E40F94A9AF60931102709324
:10FB7000120280931302909314020C94898A83E5F5
:10FB80000E944736882311F40C94898A0E94A73674
:10FB90000F9411B06115710551F06130710569F470
:10FBA00081E080933E0B10923D0B0C94898A109259
:10FBB0003E0B10923D0B0C94898AEDE3F0E18491A9
:10FBC000882341F09091C00095FFFCCF8093C60040
:10FBD0003196F5CFE3EAF6E285919491FC01249108
:10FBE000222341F03091C00035FFFCCF2093C600A6
:10FBF0000196F4CFE091AD10F091AE10EE54FF4EAF
:10FC00008191882339F09091C00095FFFCCF8093BB
:10FC1000C600F6CFE0E9FAE08491882341F09091A4
:10FC2000C00095FFFCCF8093C6003196F5CF809140
:10FC3000C00085FFFCCF8AE08093C6000C94898ABF
:10FC400083E50E944736882311F40C94898A0E9428
:10FC5000A7360F9411B070934802609347020C943A
:10FC6000898A83E50E944736882311F40C94898A97
:10FC70000E94A7360F9411B06B017C0184E50E94AD
:10FC80004736882391F08DED90E00E94994B8111C9
:10FC90000C94898AE091F60AF0E0EE0FFF1FED5B0D
:10FCA000FD4FD182C0820C94898AD0924602C092C4
:10FCB00045020C94898A80E50E944736882311F416
:10FCC0000C94898A0E94A7360F9411B0D62E062F65
:10FCD000172F83E50E944736882331F00E94A7360C
:10FCE0000F9411B07B0103C0EE24EA94FE2CC701EF
:10FCF0000196039710F00C94898AEAEDF5E0819162
:10FD000091918017910711F40C94898A26E0E231D1
:10FD1000F207A9F717FF02C00C94898A0F941427E1
:10FD2000CD2C60E08D2D0F94A7A83FEFE316F306CE
:10FD300031F0EA94EF2871F000E010E00DC08D2D55
:10FD40000F9415A931E020E0892B09F030E0032F52
:10FD5000122F02C001E010E08C2D0F9415A980171E
:10FD6000910711F40C94898A0F94AA3880E00E94BC
:10FD7000DF4A80E00F947058EFCF83E50E9447364A
:10FD8000882331F00E94A7360F9411B08B0102C076
:10FD90000EE610E080E50E944736882331F00E948D
:10FDA000A7360F9411B0CB0102C088EE93E06C012E
:10FDB000EE24D7FCE094FE2C1016110684F420E00B
:10FDC00030E0A901B80184E50F940AABC701B60180
:10FDD0000F94EBA684E50F9430AE0C94898AC7018A
:10FDE000B6010F94EBA60C94898A80E50E944736F1
:10FDF000882351F00E94A73660939D0270939E0263
:10FE000080939F029093A00289E40E944736882342
:10FE100061F00E94A7360F94663F60939902709339
:10FE20009A0280939B0290939C0284E40E9447363E
:10FE3000882361F00E94A7360F94723F6093950269
:10FE400070939602809397029093980283E40E94A5
:10FE50004736882351F00E94A73660939102709331
:10FE6000920280939302909394020F94972EE7E569
:10FE7000F7E285919491FC012491222341F0309185
:10FE8000C00035FFFCCF2093C6000196F4CFEFEB06
:10FE9000F4E08191882339F09091C00095FFFCCF68
:10FEA0008093C600F6CF40919D0250919E026091D2
:10FEB0009F027091A00222E030E08EE09AE00E9462
:10FEC0009635E3ECF4E08191882339F09091C000FD
:10FED00095FFFCCF8093C600F6CF60919902709198
:10FEE0009A0280919B0290919C020F946C3FAB010F
:10FEF000BC0122E030E08EE09AE00E949635E7EC0B
:10FF0000F4E08191882339F09091C00095FFFCCFF7
:10FF10008093C600F6CF6091950270919602809111
:10FF20009702909198020F94783FAB01BC0122E0B8
:10FF300030E08EE09AE00E949635EBECF4E081919F
:10FF4000882339F09091C00095FFFCCF8093C600C4
:10FF5000F6CF40919102509192026091930270917C
:10FF6000940222E030E08EE09AE00E949635809183
:10FF7000C00085FFFCCF8AE08093C6000C94898A7C
:10FF800080E50E944736882351F00E94A73660938F
:10FF90008D0270938E0280938F029093900289E479
:10FFA0000E944736882361F00E94A7360F94663F6F
:10FFB0006093890270938A0280938B0290938C02E3
:10FFC00084E40E944736882361F00E94A7360F948C
:10FFD000723F6093850270938602809387029093AC
:10FFE00088020F94972EE7E5F7E285919491FC0142
:10FFF0002491222341F03091C00035FFFCCF2093A3
:020000021000EC
:10000000C6000196F4CFEFEBF4E08191882339F03C
:100010009091C00095FFFCCF8093C600F6CF409131
:100020008D0250918E0260918F027091900222E0B9
:1000300030E08EE09AE00E949635E3ECF4E08191A6
:10004000882339F09091C00095FFFCCF8093C600C3
:10005000F6CF6091890270918A0280918B02909113
:100060008C020F946C3FAB01BC0122E030E08EE0CB
:100070009AE00E949635E7ECF4E08191882339F00C
:100080009091C00095FFFCCF8093C600F6CF6091A1
:1000900085027091860280918702909188020F9468
:1000A000783FAB01BC0122E030E08EE09AE00E9494
:1000B00096358091C00085FFFCCF8AE08093C60012
:1000C0000C94898A83E50E944736882319F00E94A0
:1000D000A73603C060E070E0CB010F940A1C0C94BB
:1000E000898A85E40E944736882341F00E94A7361A
:1000F0000F9411B08B0177FF03C009C000E010E03E
:10010000812C912C96E1A92E93E4B92E06C0812C66
:10011000912C8CE8A82E82E4B82E83E50E94473605
:10012000882321F00E94A7364B015C0183E40E94E2
:100130004736882331F00E94A7360F9411B09B01F7
:1001400002C025E030E0A801C501B4010F94573189
:100150000C94898A60E084E190E00E9498240C94D9
:10016000898A60E084E190E00E94272C0C94898ABF
:1001700080E00E94B8250C94898A9091C00095FF78
:10018000FCCF8093C600319684918111F6CFE0E8D0
:10019000FAE08491882311F40C94898A9091C0002C
:1001A00095FFFCCF8093C6003196F3CF8AE50E947D
:1001B0004736882309F4B0C00E94A7364B015C0182
:1001C00020E030E040E751EC0F94D1B187FD4EC004
:1001D00020E030E040EA50ECC501B4010F94A2AF3A
:1001E00018160CF443C0B7FAB094B7F8B0948092E4
:1001F000420B9092430BA092440BB092450BEDE35F
:10020000F0E18491882341F09091C00095FFFCCFEC
:100210008093C6003196F5CFE7E5F7E2459154911A
:10022000E9E8F6E2859194912FE73AE068E879E011
:100230000E94B6BCFC012491222341F03091C00001
:1002400035FFFCCF2093C6000196F4CF8091C0000B
:1002500085FFFCCF8AE08093C6008091C00085FFB7
:10026000FCCF8AE08093C6000C94898AEDE3F0E12C
:100270008491882341F09091C00095FFFCCF80933A
:10028000C6003196F5CFE9E8F6E285919491FC013C
:100290002491222341F03091C00035FFFCCF209300
:1002A000C6000196F4CFE5E8F6E285919491FC0151
:1002B0002491222341F03091C00035FFFCCF2093E0
:1002C000C6000196F4CF4AE050E061EF7FEF8EE088
:1002D0009AE00E949E34E7E8F6E285919491FC0151
:1002E0002491222341F03091C00035FFFCCF2093B0
:1002F000C6000196F4CF4AE050E06BEF7FEF8EE04E
:100300009AE00E949E348091C00085FFFCCF8AE075
:100310008093C6000C94898AEDE3F0E184918823F0
:1003200041F09091C00095FFFCCF8093C6003196BC
:10033000F5CFE9E8F6E2859194916BE77AE00E94C7
:1003400095BCFC012491222341F03091C00035FF7F
:10035000FCCF2093C6000196F4CF8091C00085FFAA
:10036000FCCF8AE08093C6004091420B5091430B32
:100370006091440B7091450B705822E030E08EE0A4
:100380009AE00E9496358091C00085FFFCCF8AE0FC
:100390008093C6000C94898A6FEC74E08EE09AE03A
:1003A0000E9491340F9414278091ED1B882321F033
:1003B00086E190E00F945F56809147029091480249
:1003C0009093420280934102C090550BD090560BFF
:1003D000E090570BF090580BCF8ED8A2E9A2FAA26A
:1003E0000091590B10915A0B20915B0B30915C0BD3
:1003F0000BA31CA32DA33EA340915D0B50915E0B5C
:1004000060915F0B7091600B4FA358A769A77AA703
:100410008091610B9091620BA091630BB091640B82
:100420008BA79CA7ADA7BEA7C982DA82EB82FC820C
:100430000D831E832F83388749875A876B877C8774
:100440008D879E87AF87B88B85E40E9447368823C7
:1004500059F00E94A7369B01AC016BA57CA58DA528
:100460009EA50F94B2AE0AC020E030E040E050E418
:100470006BA57CA58DA59EA50F94B1AE6BA77CA79F
:100480008DA79EA7EFA0F8A409A51AA52BA13CA1B2
:100490004DA15EA16F8D78A189A19AA1E1E4FBE055
:1004A000FF93EF93812C912CB8ECAB2EB3E4BB2ED1
:1004B000DE019B966D010F94A00D8AE50E944736E0
:1004C0000F900F90882349F00E94A7369B01AC0142
:1004D0006FA178A589A59AA51EC020E030E040E074
:1004E00050E46FA178A589A59AA50F94B2AE4B01EF
:1004F0005C016FA378A789A79AA720E030E040E2CB
:1005000051E40F94A2AF87FF0CC020E030E040E23E
:1005100051E4C501B4010F94B2AE6FA378A789A7C7
:100520009AA7EFA0F8A409A51AA52BA13CA14DA15B
:100530005EA16F8D78A189A19AA1E1E4FBE0FF9310
:10054000EF93812C912CA0E7AA2EA1E4BA2EFE01F4
:10055000BB966F010F94A00D88E50E9447360F905F
:100560000F90882379F00E94A7369B01AC016F8D14
:1005700078A189A19AA10F94B2AE6F8F78A389A3B5
:100580009AA308C080E090E0A3E5B3E48F8F98A31E
:10059000A9A3BAA389E50E944736882339F00E94AF
:1005A000A7366BA37CA38DA39EA304C01BA21CA291
:1005B0001DA21EA2EFA0F8A409A51AA52BA13CA17B
:1005C0004DA15EA16F8D78A189A19AA1E1E4FBE024
:1005D000FF93EF93812C912CF8E4AF2EF2E4BF2E21
:1005E000DE019B966D010F94A00D0F94142781E0FE
:1005F0008093860BE1EAF6E2859194910F94F1568F
:100600008CE40E9447360F900F90882359F00E9487
:10061000A7369B01AC016BA57CA58DA59EA50F946B
:10062000B2AE0AC020E030E040EA52E46BA57CA5FF
:100630008DA59EA50F94B1AE6BA77CA78DA79EA795
:10064000EFA0F8A409A51AA52BA13CA14DA15EA17C
:100650006F8D78A189A19AA1E1E4FBE0FF93EF936C
:10066000812C912CE8ECAE2EE3E4BE2EFE01BB966D
:100670006F010F94A00D0F941427149A64E670E094
:1006800080E090E00F94EBA60F9403740F94BCA647
:100690006093950B7093960B8093970B9093980BA8
:1006A0000F900F9000E010E0F12C0F94F85A811198
:1006B0002AC0F3940F94AA3881E00E94DF4AF11017
:1006C000F4CF043FF1E01F0711F400E010E0809147
:1006D00001018460809301010115110531F49FB778
:1006E000F89480910201846008C00431110541F43E
:1006F0009FB7F894809102018B7F809302019FBF86
:100700000F5F1F4FD2CF9FB7F894809102018B7F6C
:10071000809302019FBF20E030E04CE852E46BA5DB
:100720007CA58DA59EA50F94B2AE6BA77CA78DA7C7
:100730009EA7EFA0F8A409A51AA52BA13CA14DA145
:100740005EA16F8D78A189A19AA1F1E46F2EFBE0E3
:100750007F2E7F926F92812C912CA0EAAA2EA1E489
:10076000BA2EDE019B966D010F94A00D20E030E0C3
:1007700048E452E46BA57CA58DA59EA50F94B2AE6E
:100780006BA77CA78DA79EA7EFA0F8A409A51AA523
:100790002BA13CA14DA15EA16F8D78A189A19AA149
:1007A0007F926F92812C912CA12CB0E4BB2E0F94E0
:1007B000A00D1092B80B1092B70B0F946B740F90A2
:1007C0000F900F900F908091B70B9091B80B0197FD
:1007D00009F48CC01092B80B1092B70B0F94AB7445
:1007E0008091B70B9091B80B8230910571F103970E
:1007F00009F076C020E030E048E452E46BA57CA527
:100800008DA59EA50F94B2AE6BA77CA78DA79EA7C2
:10081000EFA0F8A409A51AA52BA13CA14DA15EA1AA
:100820006F8D78A189A19AA17F926F92812C912CD2
:10083000A12CA0E4BA2EDE019B966D010F94A00DB1
:100840000F942B740F900F90BECF20E030E04CE857
:1008500052E46BA57CA58DA59EA50F94B2AE6BA7A7
:100860007CA78DA79EA7EFA0F8A409A51AA52BA188
:100870003CA14DA15EA16F8D78A189A19AA17F9223
:100880006F92812C912CB0EAAB2EB1E4BB2EDE012D
:100890009B966D010F94A00D20E030E048E452E4F7
:1008A0006BA57CA58DA59EA50F94B2AE6BA77CA76A
:1008B0008DA79EA7EFA0F8A409A51AA52BA13CA17E
:1008C0004DA15EA16F8D78A189A19AA17F926F92AF
:1008D000812C912CA12CE0E4BE2E0F94A00D6DCFA5
:1008E0000F941D7481E00F94DD596DCF20E030E04E
:1008F00040EA50E46BA57CA58DA59EA50F94B2AEF1
:100900006BA77CA78DA79EA7EFA0F8A409A51AA5A1
:100910002BA13CA14DA15EA16F8D78A189A19AA1C7
:10092000E1E46E2EEBE07E2E7F926F92812C912C73
:10093000A12CF0E4BF2EFE01BB966F010F94A00D19
:10094000A50194016BA57CA58DA59EA50F94B1AEC4
:100950006BA77CA78DA79EA7EFA0F8A409A51AA551
:100960002BA13CA14DA15EA16F8D78A189A19AA177
:100970007F926F92812C912CA8ECAA2EA3E4BA2E20
:100980000F94A00DEFA0F8A409A51AA52D813E8112
:100990004F81588569817A818B819C817F926F928A
:1009A000812C912CB8E4AB2EB2E4BB2E0F94A00D99
:1009B000E984FA840B851C852D813E814F81588501
:1009C00069817A818B819C817F926F92812C912C9D
:1009D000E0E7AE2EE1E4BE2E0F94A00D20E030E063
:1009E00040E050E46BA57CA58DA59EA50F94B2AE0A
:1009F0006BA77CA78DA79EA7E984FA840B851C852D
:100A00002D813E814F81588569817A818B819C81BE
:100A10007F926F92812C912CF8ECAF2EF3E4BF2ED5
:100A20000F94A00DCE010D960F94ED1B8091410205
:100A30009091420280934702909348029F938F9334
:100A400082E79AE09F938F938E01015D1F4F1F9362
:100A50000F930F9404B960E0C8010E94BEB2E3E8AE
:100A6000F6E2859194910F94F1561092860B1092B4
:100A7000840B1092830B0FB6F894DEBF0FBECDBF70
:100A80008091A512882309F444C50E94E8B10F940F
:100A900014270E9458B4811105C00E94ED5A0E948B
:100AA000E8B1F7CF0E9400BA0E94FBB932C580912D
:100AB000F11B9091F21B892B09F02BC585E090E08A
:100AC0009093F21B8093F11B24C58091F11B9091B0
:100AD000F21B892B09F01DC586E090E09093F21B74
:100AE0008093F11B16C50E94F33B13C588E50E9455
:100AF0004736882339F00E94A7360F9411B080E062
:100B00000F948C288AE50E944736882339F00E948A
:100B1000A7360F9411B081E00F948C2885E40E94D1
:100B20004736882309F4F5C40E94A7360F9411B004
:100B300082E00F948C28EDC40F942744EAC488E522
:100B40000E944736882339F00E94A7360F9416B0CA
:100B500080E00F94A54389E50E944736882339F049
:100B60000E94A7360F9416B081E00F94A5438AE542
:100B70000E944736882339F00E94A7360F9416B09A
:100B800082E00F94A54385E40E944736882309F448
:100B9000C0C40E94A7360F9416B083E00F94A543FB
:100BA000B8C488E50E944736882339F00E94A736EA
:100BB0000F9416B080E00F94E64389E50E94473613
:100BC000882339F00E94A7360F9416B081E00F9465
:100BD000E6438AE50E944736882339F00E94A7360B
:100BE0000F9416B082E00F94E64385E40E944736E6
:100BF000882309F48EC40E94A7360F9416B083E0B0
:100C00000F94E64386C40F94324083C481E08093FE
:100C10004D1B0F9427447DC488E50E9447368823E6
:100C200031F00E94A7360F9416B06093A60289E5B2
:100C30000E944736882331F00E94A7360F9416B0E1
:100C40006093A7028AE50E944736882331F00E940C
:100C5000A7360F9416B06093A80285E40E94473629
:100C6000882331F00E94A7360F9416B06093A90232
:100C7000ECEDF4E08191882339F09091C00095FF6C
:100C8000FCCF8093C600F6CF4AE050E06091A60208
:100C90008EE09AE00E94E334EFEEF4E08191882345
:100CA00039F09091C00095FFFCCF8093C600F6CF3D
:100CB0004AE050E06091A7028EE09AE00E94E3349F
:100CC000E2E0F5E08191882339F09091C00095FF32
:100CD000FCCF8093C600F6CF4AE050E06091A802B6
:100CE0008EE09AE00E94E334E5E1F5E0819188230B
:100CF00039F09091C00095FFFCCF8093C600F6CFED
:100D00004AE050E06091A9028EE09AE00E94E3344C
:100D100000C488E50E944736882339F00E94A73630
:100D20000F9416B080E00F94A64189E50E944736E3
:100D3000882339F00E94A7360F9416B081E00F94F3
:100D4000A6418AE50E944736882339F00E94A736DB
:100D50000F9416B082E00F94A64185E40E944736B6
:100D6000882309F4D6C30E94A7360F9416B083E0F7
:100D70000F94A641CEC388E50E944736882339F0F8
:100D80000E94A7360F9416B080E00F94FD4189E5CC
:100D90000E944736882339F00E94A7360F9416B078
:100DA00081E00F94FD418AE50E944736882339F09F
:100DB0000E94A7360F9416B082E00F94FD4185E49F
:100DC0000E944736882309F4A4C30E94A7360F94D3
:100DD00016B083E00F94FD419CC3159881E0809389
:100DE000860B82E090E09093840B8093830BE3E981
:100DF000F7E2859194910F94F15620E030E04CE8B1
:100E000052E46091610B7091620B8091630B909141
:100E1000640B0F94B2AE6093610B7093620B80937E
:100E2000630B9093640BE0905D0BF0905E0B009170
:100E30005F0B1091600B2091590B30915A0B409130
:100E40005B0B50915C0B6091550B7091560B809130
:100E5000570B9091580BE1E46E2EEBE07E2E7F92C3
:100E60006F92812C912CF0ECAF2EF0E4BF2EA1E616
:100E7000CA2EABE0DA2E0F94A00D20E030E048EC53
:100E800051E46091610B7091620B8091630B9091C2
:100E9000640B0F94B2AE6093610B7093620B8093FE
:100EA000630B9093640BE0905D0BF0905E0B0091F0
:100EB0005F0B1091600B2091590B30915A0B4091B0
:100EC0005B0B50915C0B6091550B7091560B8091B0
:100ED000570B9091580B7F926F92812C912CB0E818
:100EE000AB2EBFE3BB2E0F94A00D0F9414270F90D1
:100EF0000F900F900F908091ED1B8823A9F081E057
:100F00000F94DD5982E00F947058E3E8F6E2859182
:100F100094910F94F1561092850B1092860B1092BB
:100F2000840B1092830BF5C28091850B882339F3D3
:100F300007EC602E07E2702EF3018591949141E059
:100F400060E00F94567E91E0811101C090E011E4C1
:100F5000412E1BE0512E9111D2CF81E00F94DD592B
:100F600082E00F94705820E030E048EC51E460914A
:100F7000610B7091620B8091630B9091640B0F94E5
:100F8000B2AE6093610B7093620B8093630B90938E
:100F9000640BE0905D0BF0905E0B00915F0B109185
:100FA000600B2091590B30915A0B40915B0B509183
:100FB0005C0B6091550B7091560B8091570B909183
:100FC000580B5F924F92812C912CA0E8AA2EAFE390
:100FD000BA2EB1E6CB2EBBE0DB2E0F94A00D0F9402
:100FE0001427F3018591949141E060E00F94567EBF
:100FF0000F900F90811183CFB0CF81E08093860B4B
:1010000082E090E09093840B8093830BE1EAF6E218
:10101000859194910F94F15620E030E040EA52E43B
:101020006091610B7091620B8091630B9091640BE6
:101030000F94B1AE6093610B7093620B8093630B5E
:101040009093640BE0905D0BF0905E0B00915F0B52
:101050001091600B2091590B30915A0B40915B0B12
:1010600050915C0B6091550B7091560B8091570B12
:101070009091580BE1E4FBE0FF93EF93812C912CCE
:10108000E8EEAE2EE2E4BE2EF1E6CF2EFBE0DF2E40
:101090000F94A00D0F941427E3E8F6E28591949144
:1010A0000F94F1561092860B1092840B1092830BC2
:1010B0000F900F902EC2E2E6FAE08491882341F06F
:1010C0009091C00095FFFCCF8093C6003196F5CF7C
:1010D0008091C00085FFFCCF8AE08093C60019C2D2
:1010E00084E50E944736882309F4D1C0E091A3101B
:1010F000F091A410319681918032E9F38930D9F3CF
:1011000090ED980F9A30E0F08F33A9F0E2E5FAE025
:101110008491882341F09091C00095FFFCCF80938B
:10112000C6003196F5CF8091C00085FFFCCF8AE0E4
:101130008093C600EEC10F94FFA18093F60A06C00B
:101140000E94A7360F9416B06093F60A2091F60A13
:1011500081E090E0022E01C0880F0A94EAF7909196
:10116000800B982B9093800B222309F442C0EDE36F
:10117000F0E18491882341F09091C00095FFFCCF6D
:101180008093C6003196F5CFE0E5FAE0849188239C
:1011900041F09091C00095FFFCCF8093C60031963E
:1011A000F5CF6091F60A70E04AE050E08EE09AE0F8
:1011B0000E949E348091C00085FFFCCF8AE080931E
:1011C000C600EBE9F7E285919491FC01249122237A
:1011D00041F03091C00035FFFCCF2093C60001964E
:1011E000F4CF8091C00085FFFCCF8AE08093C600D9
:1011F00090C186E40E9447368823D9F00E94A73622
:101200004B015C016093100B7093110B8093120BD8
:101210009093130B20E030E0A9010F94D1B1181680
:1012200044F480920C0290920D02A0920E02B092B1
:101230000F02EDE3F0E18491882341F09091C0002A
:1012400095FFFCCF8093C6003196F5CFE9E4F8E234
:1012500085919491FC012491222341F03091C000AA
:1012600035FFFCCF2093C6000196F4CF6091410B6F
:1012700070E04AE050E08EE09AE00E949E34809157
:10128000C00085FFFCCF8AE08093C60042C184E4A1
:101290000E944736882309F4FBC00E94A7360F94AA
:1012A00011B06630710509F4C5C0ACF46230710547
:1012B000D9F154F461157105A1F16130710509F09E
:1012C00028C10E94ED2D25C16430710581F194F58E
:1012D0000E94C52E1EC16C30710509F455C064F41E
:1012E00068307105C1F0D4F06A30710509F011C1A0
:1012F00086EE0E948D3A0DC1683EF3E07F0709F447
:1013000088C0693E23E0720709F489C0673E7340D4
:1013100009F0FFC048C0E8E2F5E0ACC0E5E3F5E065
:1013200094C00E94D72DF5C00E94042EF2C00E94E6
:101330008F2FEFC063E475E08EE09AE00E94913455
:1013400080E50E944736882341F00E94A7360F941B
:1013500011B07093940A6093930AEDE4F5E08191E3
:10136000882339F09091C00095FFFCCF8093C60090
:10137000F6CF6091930A7091940A4AE050E08EE0B3
:101380009AE00E94A534C5C060E086E69FE00F9415
:1013900042BB60E085E69FE00F9442BB60E084E6DC
:1013A0009FE00F9442BB63E675E08EE09AE00E94F6
:1013B00091340F94142781E00F94DD590F94DA557E
:1013C00082E00F94705886E69FE00F9430BB61E096
:1013D000680F86E69FE00F9442BB81E00F94DD59D1
:1013E00082E00F947058E3E8F6E2859194910F94AF
:1013F000F15661E08AE49AE00E94BEB261E084E4C2
:101400009AE00E94BEB261E08EE39AE00E94BEB212
:1014100080C00E94CB5981E08093A1027AC01092D3
:10142000D60B60E084ED9BE00E9410AC81E08093DD
:10143000A1026FC081E090E00E94973E6AC0909147
:10144000C00095FFFCCF8093C60081918111F7CF3A
:1014500068EC88EC0F9445084AE050E0BC018EE04F
:101460009AE00E94A53455C09091C00095FFFCCF32
:101470008093C60081918111F7CF85E70F94EC2A04
:101480004AE050E0BC018EE09AE00E94A53441C0E1
:10149000EDE3F0E18491882341F09091C00095FF45
:1014A000FCCF8093C6003196F5CFE3EAF6E2859152
:1014B0009491FC012491222341F03091C00035FF2A
:1014C000FCCF2093C6000196F4CFE091AD10F091CF
:1014D000AE10EE54FF4E8191882339F09091C000F8
:1014E00095FFFCCF8093C600F6CFE9E3FAE0849144
:1014F000882341F09091C00095FFFCCF8093C600F7
:101500003196F5CF8091C00085FFFCCF8AE08093B3
:10151000C6000E94B94372C180902C0B90902D0B95
:10152000A0902E0BB0902F0B2091610B3091620B8D
:101530004091630B5091640BC501B4010F94B1AE9F
:101540002DEC3CEC4CEC5DE30F94D1B1181614F08B
:101550000C94B35D8092610B9092620BA092630B2E
:10156000B092640B81E69BE00F94ED1B60E080E09D
:101570000E94DD4743C10E94A7362091490B30915C
:101580004A0B40914B0B50914C0B0F94B2AE6093B1
:10159000550B7093560B8093570B9093580B0C94EC
:1015A000C65E0E94A73620914D0B30914E0B4091A4
:1015B0004F0B5091500B0F94B2AE6093590B709338
:1015C0005A0B80935B0B90935C0B0C94D35E0E9440
:1015D000A7362091510B3091520B4091530B5091F3
:1015E000540B0F94B2AE60935D0B70935E0B8093BF
:1015F0005F0B9093600B0C94D45F711028C0662031
:1016000031F181E08093E6120F9483276B017C0116
:1016100080E00F948327AB01BC019701860186EE21
:1016200092E10E94B0369B01AC0160915D0B70911C
:101630005E0B80915F0B9091600B0F94B1AE609345
:101640005D0B70935E0B80935F0B9093600B8091AA
:10165000ED1B882321F084E190E00F945F561092F7
:10166000C00BE5EAFEE08491882341F09091C00030
:1016700095FFFCCF8093C6003196F5CF0E94CF59DD
:10168000E9E9FEE08491882341F09091C00095FF44
:10169000FCCF8093C6003196F5CF0E94355AEDE815
:1016A000FEE08491882341F09091C00095FFFCCF2B
:1016B0008093C6003196F5CF0E94915A2ACF20E040
:1016C00030E040E85FE36091610B7091620B8091C4
:1016D000630B9091640B0F94B2AE6093610B7093A7
:1016E000620B8093630B9093640BE0905D0BF09022
:1016F0005E0B00915F0B1091600B2091590B3091A4
:101700005A0B40915B0B50915C0B6091550B7091A3
:10171000560B8091570B9091580BE1E4FBE0FF933F
:10172000EF93812C912CA8ECAA2EA3E4BA2EB1E65B
:10173000CB2EBBE0DB2E0F94A00D0F900F900C94DE
:10174000BB6C0F94AA3881E00E94DF4A80E00F94BE
:1017500070580C9404710E947136AB01BC01409327
:10176000720E5093730E6093740E7093750E8DEB22
:101770009DE00E94329ACDCE0E94A7360F9411B000
:101780008B010C9436730F94FF69E5E5F7E28591C0
:1017900094910F94E55BEFEBF7E2859194910E94B1
:1017A0007F3A41E050E062E080E00F94E555EDEBD8
:1017B000F7E2859194910F94626B0C94CE730F9421
:1017C000142788E50E944736882319F0179A10924B
:1017D000460B89E50E944736882319F0169A109225
:1017E000470B8AE50E94473685E40E9447368823E6
:1017F00011F40C949978149A0C949978C75ADF4F85
:101800000FB6F894DEBF0FBECDBFDF91CF911F9111
:101810000F91FF90EF90DF90CF90BF90AF909F908F
:101820008F907F906F905F904F903F902F90089592
:101830000F931F93CF93DF931F92CDB7DEB78091A5
:10184000B90B9091BA0B892BA1F00F94BCA6009113
:10185000F70A1091F80A2091F90A3091FA0A601BF0
:10186000710B820B930B693E73408105910508F063
:10187000B1C08091B90B9091BA0B892B11F41092E1
:10188000C10B8091910B882319F00E940E437EC0FA
:101890000E9461B460E084ED9BE00E941AAB8091ED
:1018A000A9109091AA10892B09F470C01092A81069
:1018B0008091D40B8823B1F00091AD101091AE103F
:1018C0000E541F4E62ED7EE0C8010F942FB8892B95
:1018D00009F5B80184ED9BE00E9469AA8091D50BBF
:1018E000882319F00E94ED5A31C0E7E5F7E28591AF
:1018F0009491FC012491222341F03091C00035FFE6
:10190000FCCF2093C6000196F4CF8091C00085FFE4
:10191000FCCF19C060E084ED9BE00E9410ACE3ECCA
:10192000F7E285919491FC012491222341F03091BA
:10193000C00035FFFCCF2093C6000196F4CF809104
:10194000C00085FFFCCF8AE08093C6008091A8107C
:1019500081111CC08091A9109091AA10892BB1F01F
:10196000F89410E090E0E091AD10F091AE10E155E8
:10197000FF4E8081823011F41181928199830E94FF
:10198000E8B1812F99810F94621C78940F94AA3842
:101990008091EE1B882311F081E001C080E00E945D
:1019A000DF4A0F94F91C80E00F9470580E9445BBE9
:1019B0000F94B2458091331B882319F11092331B89
:1019C00061E08DEC9EE00F90DF91CF911F910F9120
:1019D0000C94BEB281E08093C10B8091B90B9091C1
:1019E000BA0B01979093BA0B8093B90B0F94BCA6D6
:1019F0006093F70A7093F80A8093F90A9093FA0AB1
:101A000038CF0F90DF91CF911F910F9108959F9242
:101A1000AF92BF92CF92DF92EF92FF920F931F93FC
:101A2000CF93DF931F921F92CDB7DEB78DE99FE072
:101A30000F9438BB6093550B7093560B8093570BE4
:101A40009093580B81EA9FE00F9438BB6093590B39
:101A500070935A0B80935B0B90935C0B8DE89FE027
:101A60000F9438BB6B017C0183E79FE00F943DBB73
:101A70008C012FE832EC45EF5FE3C701B6010F940C
:101A8000B2AE6B017C0167E074E0601B710B04E097
:101A9000769567950A95E1F780E090E00F9442B063
:101AA0002091B5193091B6194091B7195091B819D4
:101AB0000F94A9AF9B01AC01C701B6010F94B2AE60
:101AC00060935D0B70935E0B80935F0B9093600B44
:101AD00080E1E5E5FBE0A0E2BBE001900D928A9594
:101AE000E1F7EDE9F8E08491882341F09091C0009E
:101AF00095FFFCCF8093C6003196F5CF0E94CF5959
:101B00000E9413D91092E612A5E7EA2EAFE0FA2E52
:101B1000D12CB3E0BB2EAA24A39417E0C12E8D2DA7
:101B20006B2D0F9460B4082F992E42E050E0B7015E
:101B3000CE0101960F9420BB69817A8161157105F0
:101B400011F0A092E6122C2D020380011124090D40
:101B5000111D97FC1A95000F111F000F111F0A513C
:101B60001D4E882777FD8095982F0F9444B02FE65F
:101B700032E143E85AE30F94A3B2F8016183728320
:101B800083839483D394F2E0EF0EF11C29E0D21208
:101B9000C6CF8091E612882321F086EE92E10F9461
:101BA0008802EBE6F8E08491882341F09091C00030
:101BB00095FFFCCF8093C6003196F5CF0E94915AD5
:101BC0000F947901E0905D0BF0905E0B00915F0B3C
:101BD0001091600B2091590B30915A0B40915B0B87
:101BE00050915C0B6091550B7091560B8091570B87
:101BF0009091580BE1E6CE2EEBE0DE2E0F944E1ABC
:101C000081E08093460B17988093470B169880933A
